:100000000C9456050C949C050C949C050C949C0532
:100010000C949C050C949C050C949C050C949C05DC
:100020000C949C050C94B9180C949C050C949C059C
:100030000C9498320C949C050C949C050C949C0593
:100040000C949C050C949C050C94DC140C949C055D
:100050000C940A0B0C949C050C94D40A0C949C05EB
:100060000C94821B0C949C050C941E2E0C949C05E5
:100070000C9443750C949C050C94B26FA91BAE1B99
:10008000B31BBC1BD31BEA1BFA1B0A1C271C4B1EF1
:10009000EA1BFD1C0E1D3D1D5B1D781DD21D2D1E76
:1000A00057200121902110224822EB22F2245C25C6
:1000B000D6251F2669269726C42627277127BB2702
:1000C000B4283D2E712EB42E242F3C2F7D2F34309A
:1000D000FB30FB30FB30FB30FB30FB30FB30FB30C8
:1000E000FB30FB30FB30B030B230B730CF30D130E6
:1000F0007F652866AD66F26503673367B365216681
:100100000A0D3D3D3D3D3D3D3D3D3D3D3D3D3D3D82
:100110003D3D3D3D3D3D3D3D3D3D3D3D3D3D3D3D0F
:100120003D3D3D3D3D000A0D426174743A0020257D
:10013000642043656C6C732000204C6F77207761DE
:10014000726E696E673A2025642E2564000A0D469A
:100150006F756E6420424C2D4374726C3A200025FA
:1001600064000A0D0A0D2121204D495353494E4781
:1001700020424C2D4354524C3A202564202121002A
:100180000A0D43616C6962726174696E67207072F6
:100190006573737572652073656E736F722E2E00B2
:1001A0004F4B0A0D000A0D466C696768742D74691F
:1001B0006D65202575206D696E20546F74616C3AF1
:1001C0002575206D696E00416E676C654E69636BC5
:1001D00020202020202020416E676C65526F6C6CBF
:1001E000202020202020204163634E69636B202063
:1001F00020202020202020416363526F6C6C20203F
:10020000202020202020205961774779726F2020FC
:1002100020202020202020416C74697475646520A2
:100220005B302E316D5D204163635A2020202020F9
:100230002020202020202047617320202020202003
:1002400020202020202020436F6D70617373205682
:10025000616C7565202020566F6C74616765205B4A
:10026000302E31565D2020526563656976657220B7
:100270004C6576656C20204779726F20436F6D70F6
:10028000617373202020204D6F746F722031202005
:10029000202020202020204D6F746F7220322020DB
:1002A000202020202020204D6F746F7220332020CA
:1002B000202020202020204D6F746F7220342020B9
:1002C0002020202020202031362020202020202007
:1002D00020202020202020313720202020202020F6
:1002E00020202020202020313820202020202020E5
:1002F00020202020202020313920202020202020D4
:1003000020202020202020536572766F202020207E
:1003100020202020202020486F766572676173209E
:100320002020202020202043757272656E74205B8F
:10033000302E31415D202043617061636974792002
:100340005B6D41685D20204865696768742053656E
:1003500074706F696E742032352020202020202098
:100360002020202020202032362020202020202065
:1003700020202020202020436F6D70617373205354
:100380006574706F696E744932432D4572726F7275
:1003900020202020202020424C204C696D697420B0
:1003A000202020202020204750535F4E69636B207F
:1003B000202020202020204750535F526F6C6C205B
:1003C0002020202020202021212120494E434F4D54
:1003D00050415449424C4520212121002E000A0D54
:1003E00020444143206F7220493243204552524FEE
:1003F000522120436865636B204932432C203356D9
:100400007265662C2044414320616E6420424C2D6D
:100410004374726C005B25695D005B25695D002B90
:10042000204D696B726F4B6F70746572202B0048A2
:10043000573A5625642E25642053573A25642E25B5
:100440006425632056340053657474696E673A25D9
:1004500064202573004D69786572204572726F7251
:1004600021004861726477617265204572726F7213
:1004700020313A2564202121004D697373696E672C
:1004800020424C2D4374726C3A25642121002120B6
:100490004E432D4552523A202532642021200049F6
:1004A0003243204552524F5221212100486569674D
:1004B00068743A202025356900536574706F696E41
:1004C000743A2535690050726573737572653A2503
:1004D0003569004F66667365743A202025356900DA
:1004E00048656967687420636F6E74726F6C00444E
:1004F000495341424C4544006163742E206265615A
:1005000072696E67004E69636B3A202020202020BC
:1005100025356900526F6C6C3A2020202020202560
:10052000356900436F6D706173733A202020253563
:1005300069004B25693A25346920204B25693A2505
:10054000346920004E693A2534692020526F3A25DB
:100550003469200047733A253469202047693A25D9
:100560003469200050313A253469202050323A2530
:100570003469200050333A253469202050343A251C
:10058000346920004779726F202D2053656E736F98
:1005900072004E69636B25346920282533692E2546
:1005A000692900526F6C6C25346920282533692E27
:1005B0002569290047696572253469202825336932
:1005C00029004E69636B2025346920282533692E64
:1005D00025782900526F6C6C20253469202825333A
:1005E000692E257829005961772020253469202833
:1005F00025336929004E69636B202534692028253D
:10060000336929282533692900526F6C6C20253401
:1006100069202825336929282533692900596177FC
:100620002020253469202825336929282533692984
:1006300000414343202D2053656E736F72004E6955
:10064000636B2025346920282533692900526F6C9B
:100650006C20253469202825336929005A20202060
:100660002025346920282533692900566F6C746170
:1006700067653A2020202533692E253169560043CD
:10068000757272656E743A2020202533692E2531EB
:10069000694100506F7765723A2020202020253470
:1006A0006957004469736368617267653A2025354C
:1006B000696D4168005265636569766572005243F1
:1006C0002D525353493A20202020253469005243AB
:1006D0002D5175616C6974793A2025346900524353
:1006E0002D4368616E6E656C733A25346900436F03
:1006F0006D70617373004D61676E65743A202020E0
:10070000253569004779726F3A2020202020253551
:100710006900536574706F696E743A2025356900FD
:10072000506F746925693A202025336900506F7431
:100730006925693A202025336900536572766F2058
:100740002000536574706F696E7420202533690032
:10075000506F736974696F6E3A2025336900526176
:100760006E67653A2533692D25336900424C2D4368
:1007700074726C204572726F72732000253364208E
:1007800025336420253364202533642000424C2027
:1007900054656D70657261747572650025336420EF
:1007A00025336420253364202533642000424C2DFA
:1007B0004374726C20666F756E6420002025632080
:1007C0002020256320202025632020202563200071
:1007D0002025632020202563202020256320202041
:1007E000256320002025632020202D2020202D207F
:1007F00020202D2000313000313100313200466C94
:10080000696768742D54696D65202000546F7461A8
:100810006C3A2535756D696E004163743A20202568
:1008200035756D696E0028726573657429000A0D4F
:1008300047656E65726174696E672064656661758F
:100840006C7420506172616D6574657220536574BB
:10085000202564000A0D5573696E6720506172612E
:100860006D6574657220536574202564000A0D4718
:10087000656E65726174696E672064656661756C2A
:1008800074204D69786572205461626C65000A0DB0
:100890004D697865722D436F6E6669673A2027252A
:1008A000732720282575204D6F746F727329000AF5
:1008B0000D414343206E6F742063616C6962726105
:1008C000746564210D0A0000008F001E01AD013B1C
:1008D00002CA025803E603740402058F051B06A72B
:1008E000063307BE074808D2085B09E3096B0AF222
:1008F0000A780BFD0B810C040D860D070E870E0682
:100900000F840F00107B10F5106E11E5115B12CFF4
:10091000124213B31323149214FE146A15D3153B19
:1009200016A11605176717C81727188318DE18377A
:10093000198E19E319361A871AD61A231B6E1BB69D
:100940001BFD1B411C831CC31C001D3C1D751DABE6
:100950001DE01D121E421E6F1E9A1EC31EE91E0DB3
:100960001F2E1F4D1F691F841F9B1FB01FC31FD346
:100970001FE11FEC1FF51FFB1FFF1F00200A0D7753
:1009800077772E4D696B726F4B6F707465722E6442
:10099000652028632920486953797374656D732035
:1009A000476D6248000A0D74686520757365206F95
:1009B00066207468697320736F667477617265204E
:1009C0006973206F6E6C79207065726D69747465DF
:1009D00064200A0D6F6E206F726967696E616C200A
:1009E0004D696B726F4B6F707465722D48617264E4
:1009F00077617265005573657200486F54542056D4
:100A000034004143542044534C004A6574690053F8
:100A100070656B7472756D0050504D000A0D526513
:100A20006365697665723A2000756E6B6E6F776EDE
:100A30002E205573696E672050504D2E2E2E006E5D
:100A40006F7420737570706F7274656420627920A2
:100A5000686172647761726521000A0D466C69678E
:100A60006874436F6E74726F6C0A0D4861726477BC
:100A70006172653A25642E25640A0D536F6674779A
:100A80006172653A5625642E2564256320000A0D9F
:100A9000202D204C4942204E4F5420434F4D504171
:100AA0005449424C452021212121000011241FBE20
:100AB000CFEFD0E1DEBFCDBF11E0A0E0B1E0E0E2DA
:100AC000F0EF02C005900D92A43AB107D9F718E0F3
:100AD000A4EAB1E001C01D92A138B107E1F76AEACA
:100AE000E2E0F0E081E2809357007491AE014F5F45
:100AF0005F4F20EF37EFDA019FE0F9012F5F3F4FA3
:100B000084918D93915097FFF8CF773911F40000BD
:100B1000FECFFA019EE0819168276095915097FF82
:100B2000FACF8889681721F0773911F40000FECFD9
:100B30000E9468060C940F780C94000080E091E00D
:100B40009F938F9380EC91E19F938F93E0917E032D
:100B5000F0917F0309950F900F900F900F900895DB
:100B60008091C905E82FFF27EE0FFF1FE450F94FD2
:100B7000808191818D5E9F4F14F0109202018081DF
:100B800091818A5B9F4FCCF4809102018823A9F464
:100B900081E0809302018091B2038F5F8093B20362
:100BA000853038F088EE93E09093D9018093D80196
:100BB000089566E970E00E94B63408951F93CF93BC
:100BC000DF93182F882389F086E291E09F938F931B
:100BD00080EC91E19F938F93E0917E03F0917F03EE
:100BE00009950F900F900F900F908091EC05823334
:100BF00008F044C084EF91E00E94CF15EC0111236E
:100C000029F0CE010E94D8158823D9F3C2E0D0E0A4
:100C100026E530E080911F01909120018217930713
:100C200030F02196255D3F4FC730D10598F3809174
:100C3000EC059927C89F9001C99F300DD89F300DB2
:100C40001124209300011123D9F068EC70E08C2F5F
:100C50000E94B634DF93CF938EE291E09F938F93FF
:100C600080EC91E19F938F93E0917E03F0917F035D
:100C700009958DB79EB706968DBF02C0809300017F
:100C8000112311F1809100016AE00E946277892F9F
:100C900099279F938F93809100010E9462779927F3
:100CA0009F938F9389E391E09F938F9380EC91E1E1
:100CB0009F938F93E0917E03F0917F0309952DB769
:100CC0003EB7285F3F4F2DBFDF91CF911F91089511
:100CD000CFEFD0E1DEBFCDBF8824992414B815B87A
:100CE0008AE08AB98FE58BB9B7EEEB2EB3E0FB2E25
:100CF0002EEC3FEFE20EF31EF7FEFACF189B06C074
:100D0000199B02C08DE005C08BE003C0199B04C095
:100D100084E18093010107C08AE0809301018EE3A2
:100D20008AB987E48BB981E887B93E9A8FEF88B991
:100D30008BE184B981E085B9469A84B7877F84BF07
:100D4000809160008861809360001092600084EC64
:100D500099E09093D9018093D8011092800210926B
:100D60007F021092010710920007109282021092E7
:100D70008102109284021092830220910101243199
:100D800028F084EC94E0A0E0B0E004C08BE095E0B3
:100D9000A0E0B0E080933C0190933D01A0933E0120
:100DA000B0933F012A3011F0243110F0289801C08F
:100DB000289A2C3010F0273111F4299A01C0299873
:100DC0000E9438160E9409160E94C8110E946F32B4
:100DD0000E943A1A81E00E94D22D0E9411640E9462
:100DE000826D82E00E94FC73809101018C3010F0D2
:100DF000873111F4299A01C0299878940E94F12C26
:100E000080912202826080932202109225020E9429
:100E1000144084EF91E00E94CF157C018091220262
:100E200080FD05C0C7010E94D8158823B9F38DE461
:100E300091E09F938F93A0ECAA2EA1E1BA2EBF92CE
:100E4000AF92E0917E03F0917F03099580EA9FE0E5
:100E50000E94CF157C01C0E0D0E00F900F900F9062
:100E60000F900EE916E0F2E5CF2EF6E0DF2E0E949D
:100E700014408091220280FD05C0C7010E94D81550
:100E80008823B9F3F60180811816ACF40BC00E94D8
:100E900014408091220280FD05C0C7010E94D81530
:100EA0008823B9F3C7010E94D815882321F4F801DB
:100EB0008081882364F7F801808187FF19C021961B
:100EC000DF93CF9321978FE591E09F938F93BF920C
:100ED000AF92E0917E03F0917F0309958091A50187
:100EE0008F5F8093A5012DB73EB72A5F3F4F2DBF7F
:100EF000219684E090E0C80ED91E085F1F4FCC30C9
:100F0000D10508F4B4CFC0E0D0E00BE916E0E2E58B
:100F1000EE2EE6E0FE2EF801838187FD1DC0F7016D
:100F200080811816CCF42196DF93CF93219782E627
:100F300091E09F938F9380EC91E19F938F93E09149
:100F40007E03F0917F03099582E08093D6012DB74F
:100F50003EB72A5F3F4F2DBFF8018381807883839E
:100F6000219624E030E0E20EF31E085F1F4FCC30E4
:100F7000D10588F20E949E059091C7058091A50138
:100F8000981728F48091980380618093980380E8F3
:100F900091E09F938F93C0ECD1E1DF93CF93E091E9
:100FA0007E03F0917F03099588EE93E00E94CF15B0
:100FB0007C010E94401A0F900F900F900F90C70174
:100FC0000E94D8158823D9F380EA91E09F938F93EC
:100FD000DF93CF93E0917E03F0917F03099580E04A
:100FE0000E949A35809101010F900F900F900F9001
:100FF0008A3011F0843110F0289801C0289A80EDD1
:1010000097E09093D9018093D80185E58093B4034C
:101010008EE090E00E94192B9927182F00278FE06F
:1010200090E00E94192B080F111D1093AB01009343
:10103000AA018AE090E00E94192B9927182F002717
:101040008BE090E00E94192B080F111D1093A9014D
:101050000093A8010F5F1F4F39F08091AA01909172
:10106000AB018F5F9F4F41F41092AB011092AA0128
:101070001092A9011092A8018091A8019091A90154
:101080009F938F938091AA019091AB019F938F932F
:1010900085EA91E09F938F93DF93CF93E0917E0356
:1010A000F0917F0309950E94C91F88E893E190930E
:1010B000370180933601C1E0C093B3038C2F0E94A7
:1010C000DE058091EF050E944F730E949E0580ED22
:1010D00097E00E94CF157C018AEF90E00E94CF1527
:1010E00083E0809321051092A401809136062DB7EC
:1010F0003EB7285F3F4F2DBF84FF02C0C093AC01B5
:101100008091AE01882311F04798FECF8091DC01D9
:10111000882309F441C280911101882309F43CC25B
:101120001092DC018091B203882319F00E94B0056F
:1011300002C00E9463430E941440209101012A30A2
:1011400011F0243110F0289801C0289A8091730280
:10115000882331F0809173028150809373020EC016
:1011600080916F00806280936F001092FD06109254
:10117000FC068091980388608093980380913601E3
:1011800090913701019790933701809336018091B8
:10119000360190913701892B21F080912302882319
:1011A000C9F18091360190913701892BD9F40E94C1
:1011B000FC2D85E090E0909337018093360180917B
:1011C0005B0590915C05019690935C0580935B05AF
:1011D00080919803816080939803809122058260BA
:1011E000809322058091090190910A018F5F9F4FA2
:1011F000C1F4809172028823A1F088EA91E690936D
:10120000D9018093D80180E890E090930A018093FF
:10121000090107C02A3011F0243110F0289801C0CC
:10122000289A0E94C9748091DC01882309F0B4C116
:1012300080910F01882311F00E9491160E940C12D8
:101240000E945A0DC7010E94D815882309F4A0C135
:1012500084E190E0E80EF91E0E944F16809123026F
:10126000882349F08091980382608093980380914D
:10127000220582600FC08091D8019091D901892BFD
:1012800059F48091360190913701079728F08091A9
:1012900022058D7F809322058091AC01882361F027
:1012A00080917302873940F01092AC0188E893E195
:1012B0009093D9018093D80180910401882321F073
:1012C0008150809304012EC08093BE031092470288
:1012D000109246021092450210924402109243026C
:1012E00010924202809173028823E1F480910901F7
:1012F00090910A018F5F9F4FA9F42091AC01223099
:1013000089F088E99AE39093D9018093D80180E02D
:101310009CE090930A0180930901222319F082E056
:101320008093AC0180919901893C48F08150809371
:101330009901809198038B7F809398033FC080919F
:10134000DF078823F9F080919803846080939803E5
:1013500089E0809351038091090190910A018F5F88
:101360009F4F81F480917202882361F088E99AE3AB
:101370009093D9018093D80180E098EA90930A0174
:10138000809309011092430310924203109241038B
:101390001092400310923F031092D207109211084E
:1013A0001092100810921308109212088FEF9FEFFE
:1013B00090930F0880930E0810929901809100017C
:1013C000282F332780911F019091200182179307C6
:1013D000CCF480913B02806280933B0280910901B2
:1013E00090910A018F5F9F4FC1F480E797E190933E
:1013F000D9018093D80180E093E090930A01809313
:1014000009010BC08091D8019091D901892B29F451
:1014100080913B028F7D80933B020E94C66884E0EE
:101420008093D7018091AD018F5F8093AD018133AF
:1014300009F065C01092AD0180913B0281FF0AC0A6
:101440008091A6019091A70101969093A7018093A6
:10145000A60104C05AEA852E55E0952E80913C02E3
:1014600090913D028050944008F049C020916A0557
:1014700030916B0540916C0550916D05809117017D
:1014800090911801A0911901B0911A0128173907FC
:101490004A075B0764F480916A0590916B05A091FF
:1014A0006C05B0916D050596A11DB11D20C0209160
:1014B0006A0530916B0540916C0550916D058091E6
:1014C000170190911801A0911901B0911A0182178A
:1014D0009307A407B5079CF480916A0590916B056A
:1014E000A0916C05B0916D050597A109B109809394
:1014F0006A0590936B05A0936C05B0936D050894F5
:10150000811C911C82E788168BE0980609F040C088
:10151000882499242091AA013091AB012F5F3F4F7D
:101520003093AB012093AA018091A8019091A90169
:1015300001969093A9018093A801832F9927682F82
:101540008EE090E00E94212B8091AA019091AB0146
:101550009070682F8FE090E00E94212B8091A8016D
:101560009091A901892F9927682F8AE090E00E9425
:10157000212B8091A8019091A9019070682F8BE098
:1015800090E00E94212B84E190E00E94CF157C0125
:101590000E9416690E94996D8091D701882309F0F5
:1015A000AFCD0E943264ACCD1F920F920FB60F9256
:1015B00011248F939F93EF93FF93809106018823CB
:1015C000E1F48091C8019091C90101969093C901FD
:1015D0008093C801FC01EE58FB4FE081ED3019F01B
:1015E0008F3A910539F41092C9011092C80181E037
:1015F00080930601E093C60004C01092C9011092C6
:10160000C801FF91EF919F918F910F900FBE0F90A6
:101610001F9018951F920F920FB60F9211242F93BF
:101620003F934F935F936F937F938F939F93AF936A
:10163000BF93CF93EF93FF9390E08091AE01813001
:1016400029F48091C6008093CE00CCC08091AE0179
:10165000823029F48091C6008093C103C3C0809179
:10166000C6008093C0015091CE015F3A10F0909374
:10167000CF018091C0018D3009F065C08091CF010C
:10168000823009F060C09093CF01852F99278F5346
:101690009C4FFC01329740812091CA013091CB01CF
:1016A000241B3109DC0111978C91281B3109C901D8
:1016B0009F709093CB018093CA0146E096958795E1
:1016C0004A95E1F7982F935C9093CC012F7330707B
:1016D000235C2093CD018081981729F48C912817E1
:1016E00011F491E006C090E08091BD018F5F80937E
:1016F000BD01C091BF01CC2309F074C0992309F446
:1017000071C081E08093BF01580F5093BC015150CC
:10171000E52FFF27EF53FC4F8DE080838091C303BB
:10172000823509F05FC00E94C91F88E190E02CE07B
:101730000FB6F894A895809360000FBE20936000C8
:10174000C093D6014FC02091CF01822F99278130BD
:101750009105F9F0823091051CF4892B21F040C0ED
:10176000029711F13DC08091C001833239F480911C
:10177000BF01882319F481E08093CF018091C001DB
:101780008093C10381E08093CE018091C0019927AD
:1017900022C02F5F2093CF01E52FFF27EF53FC4F8F
:1017A0008091C001808309C0E52FFF27EF53FC4FD4
:1017B0008091C00180835F3A20F45F5F5093CE0137
:1017C00002C01092CF012091C0018091CA01909176
:1017D000CB01820F911D9093CB018093CA0102C06F
:1017E0001092CF01FF91EF91CF91BF91AF919F9157
:1017F0008F917F916F915F914F913F912F910F90BA
:101800000FBE0F901F901895AC01A0E0B0E09D01B5
:10181000A817B90748F4E2E7F4E08191280F311DD9
:101820001196A417B507C8F33F70FD01EE58FB4FA2
:10183000C90156E0969587955A95E1F7835C8083B8
:101840001196FD01EE58FB4F2F733070822F835C91
:101850008083AD58BB4F8DE08C9310920601809130
:1018600072048093C6000895A0E0B0E0EAE3FCE0D3
:101870000C94DB772C859D850E85BB2483E28093B9
:1018800072049F59909373042093740433E0E32E01
:10189000F12C002309F49EC0CF84D888BE016D5E70
:1018A0007F4FA989BA890150109709F493C0109706
:1018B000B9F0F601EB0DF11DB3949081119791F4FD
:1018C000002349F1FB016E5F7F4FDB01C080D180B7
:1018D0006E5F7F4F0D90BC91A02DBB24015002C0C4
:1018E00090E019C01097B9F0F601EB0DF11DB3941B
:1018F0004081119791F4002341F1FB016E5F7F4F0E
:10190000DB01C080D1806E5F7F4F0D90BC91A02D18
:10191000BB24015002C040E018C01097B1F0F6019E
:10192000EB0DF11DB3941081119781F4002371F038
:10193000FB013296DB01CD90DC90BF016E5F7F4FE3
:10194000A081B181BB24015001C010E0F701EE5825
:10195000FB4F892F86958695835C80830894E11CD4
:10196000F11CF701EE58FB4F892F99278370907077
:1019700024E0880F991F2A95E1F755279A0194E0F2
:10198000369527959A95E1F7822B835C808308949E
:10199000E11CF11CF701EE58FB4F4F705070440FE3
:1019A000551F440F551F812F992726E0969587953F
:1019B0002A95E1F7842B835C80830894E11CF11C59
:1019C000F701EE58FB4F1F73135C10830894E11C62
:1019D000F11C6ACFC7010E94040CE9E00C94F77770
:1019E000A3E07A2F4091BC014650442309F458C02B
:1019F000E72FFF27EF53FC4F80818D537F5FE72F49
:101A0000FF27EF53FC4F20812D537F5FE72FFF27E8
:101A1000EF53FC4F30813D537F5FE72FFF27EF539C
:101A2000FC4F60816D537F5F9927880F991F880F46
:101A3000991F522F52955F70582B822F99278F70C4
:101A40009070F4E0880F991FFA95E1F7232F2695FF
:101A50002695282B832F992783709070E6E0880FB6
:101A6000991FEA95E1F7682B41504F3FC9F0EA2FE3
:101A7000FF27EF53FC4F5083AF5F41504F3F81F042
:101A8000EA2FFF27EF53FC4F2083AF5F41504F3FBA
:101A900039F0EA2FFF27EF53FC4F6083AF5FA5CFEC
:101AA00084EC93E09093BB018093BA01A350A09380
:101AB000B9010895A2E0B0E0E0E6FDE00C94E17722
:101AC0008091BF01882309F457C40E94F00C8091D3
:101AD000C203823609F023C38091C303992780375C
:101AE000910509F4AFC081379105C4F48A36910598
:101AF00009F480C28B36910544F48B34910571F161
:101B00008636910509F45FC10AC38D36910509F443
:101B100069C08E36910509F44DC001C38437910523
:101B200041F1853791054CF48137910509F491C055
:101B30008337910509F4DFC0F2C28737910509F4B4
:101B40001BC2883791052CF48537910509F4D7C15C
:101B5000E6C28937910509F46DC1E1C2E091BA018D
:101B6000F091BB018081918190938B0180938A01D8
:101B7000D6C28091BC01A091BA01B091BB01853160
:101B800040F080E1ECE9F3E00D9001928A95E1F7F5
:101B90000DC08D919D910D90BC91A02D80939C03C3
:101BA00090939D03A0939E03B0939F0380EF809337
:101BB000B7014BC0809106018823E1F38DE490E0EA
:101BC0009F938F9385E496E09F938F9381E08F930B
:101BD0008F938EE48F930E94340C8DB79EB7079637
:101BE0008DBF9DC2A091BA01B091BB011C91113073
:101BF00081F48DE4E5E4F6E00D9001928A95E1F739
:101C00000E942E2C1983809198038F7E80939803D5
:101C100001C01982809106018823E1F381E090E000
:101C20009F938F93CE0101969F938F9381E08F9323
:101C30008F938DE48F930E94340CADB7BEB7179687
:101C4000ADBF6DC281E08093C2018FEF809304012C
:101C500066C2E091BA01F091BB01E0818E2F8A50FB
:101C60008A3058F48983882311F481E003C08630D8
:101C700010F085E0898361E00EC08E2F84518A3098
:101C800070F48983882311F481E003C0863010F05A
:101C900085E0898360E089810E94AE2C12C0E983CF
:101CA000EF3F19F40E94912C89838981882311F4D4
:101CB00081E003C0863010F085E0898389810E942D
:101CC000372B809106018823E1F38CE790E09F9306
:101CD0008F9388EC95E09F938F9381E090E09F93A2
:101CE0008F93CE0101969F938F9382E08F9381E033
:101CF0008F9381E577C12091BA013091BB01D90161
:101D00008C918150853008F045C0F90181818D3575
:101D100009F040C0809172028823E1F52F5F3F4FA8
:101D20008CE7E8ECF5E0D9010D9001928A95E1F796
:101D3000F90182910E94A02B809109069927AA2778
:101D4000BB27BC01CD0124EC39E040E050E00E940B
:101D50004377DC01CB018093820190938301A093B0
:101D60008401B093850180910A069927AA27BB2791
:101D7000BC01CD010E944377DC01CB0180937E0141
:101D800090937F01A0938001B09381010E94912CD8
:101D9000898301C01982809106018823E1F381E0E3
:101DA00090E09F938F93CE0101969F938F9381E054
:101DB0008F938F9383E58F930E94340C8DB79EB7DA
:101DC00007968DBF26C0E091BA01F091BB01E0817A
:101DD0008E2F8150853018F48E2F0E94372B0E9451
:101DE000912C8983809106018823E1F381E090E0C2
:101DF0009F938F93CE0101969F938F9381E08F9352
:101E00008F9386E48F930E94340CADB7BEB71796BC
:101E1000ADBF80917202882329F46EE670E089815B
:101E20000E94B63480E00E94DE058091EF050E949A
:101E30004F7375C1E091BA01F091BB018081992780
:101E400087FD9095909317078093160781819927B6
:101E500087FD9095909319078093180782819927A1
:101E600087FD909590931B0780931A07838199278C
:101E700087FD909590931D0780931C078481992777
:101E800087FD909590931F0780931E078581992762
:101E900087FD90959093210780932007868199274D
:101EA00087FD909590932307809322078781992738
:101EB00087FD909590932507809324078085992727
:101EC00087FD909590932707809326078185992712
:101ED00087FD9095909329078093280782859927FD
:101EE00087FD909590932B0780932A0783859927E8
:101EF00087FD909590932D0780932C0710C1E0915A
:101F0000BA01F091BB0180810E94C8318A83882385
:101F100019F481E0898301C0198280910601882328
:101F2000E1F388E090E09F938F9383E996E09F939D
:101F30008F9321E030E03F932F938091BA019091ED
:101F4000BB019F938F933F932F93CE0102969F9354
:101F50008F933F932F93CE01820F931F9F938F9365
:101F600084E08F9381E08F9385E58F930E94340CFA
:101F7000EDB7FEB773963CC08091B901893008F483
:101F8000CEC02091BA013091BB012F5F3F4F88E056
:101F9000A3E9B6E0F90101900D928A95E1F7D90124
:101FA0008E910E941E318A83882319F481E08983EF
:101FB00001C01982809106018823E1F321E030E01D
:101FC0003F932F93CE0102969F938F933F932F932E
:101FD000CE01820F931F9F938F9382E08F9381E0B6
:101FE0008F9387E58F930E94340CEDB7FEB73B9635
:101FF000EDBF95C080917202882309F090C00E94C5
:1020000006738983823019F0843009F088C020E497
:1020100030E0F8948091C1008F738093C10080916B
:10202000C9008F738093C9008091C100877E80931F
:10203000C1008091C900877E8093C9008091C8004B
:1020400087FF03C08091CE00F9CF8091C00087FF49
:1020500003C08091C600F9CFE091BA01F091BB01B5
:10206000E081E13021F482E08093AE012EC0E436BD
:1020700011F421E830E081E08093AE01832F9927AD
:102080008093CD002093CC008091CD008093C5003B
:102090008091CC008093C4008091CA008F7D809392
:1020A000CA008091CA008F7E8093CA008091C900C7
:1020B0008B7F8093C9008091CA0084608093CA009E
:1020C0008091CA0082608093CA008091CA00877F95
:1020D0008093CA008091C200877F8093C200809164
:1020E000C9008E7F8093C9008091C1008861809370
:1020F000C1008091C90088618093C9008091C100AE
:1021000080688093C1008091C90080688093C90075
:1021100010926E0010926F0010927000789480916F
:10212000C30399278436910509F4BBC08536910510
:10213000ACF48136910509F46FC0823691052CF418
:102140008B34910509F45DC00FC18236910509F405
:1021500070C08336910509F47FC006C18C369105A5
:1021600009F4EDC08D3691054CF48736910509F4DC
:10217000F8C08836910509F4B2C0F6C084379105DD
:1021800029F08637910509F4E8C0EEC08091BC01C2
:10219000A091BA01B091BB01803140F080E1ECE93F
:1021A000F3E00D9001928A95E1F70DC08D919D911C
:1021B0000D90BC91A02D80939C0390939D03A093C0
:1021C0009E03B0939F03809106018823E1F31F9241
:1021D000809103018F9384E58F930E94340C8AEFE2
:1021E0008093B7018FEF8093040180EA9FE00E9403
:1021F000CF159093B0018093AF010F900F900F9087
:10220000B3C0E091BA01F091BB01808191819093BC
:102210008B0180938A01A8C0E091BA01F091BB01C3
:10222000808180930501803298F08FE180930501D1
:102230000FC0A091BA01B091BB018BE0E4EBF3E0D9
:102240000D9001928A95E1F78091BD03809363051B
:102250008FEF8093040188C08091B3019091B40105
:10226000892B89F4E091BA01F091BB01E081EE2362
:1022700051F08AE0E89FC00111240E94CF1590938D
:102280008F0380938E03E091BA01F091BB0190819E
:102290008AE0989FC00111249093B4018093B30108
:1022A00015C08FEF80930401E091BA01F091BB015A
:1022B00090818AE0989FC00111249093B601809389
:1022C000B501892B19F081E08093C40180EA9FE079
:1022D0000E94CF159093B0018093AF0145C08FEF5E
:1022E00080930401E091BA01F091BB01908197FDC8
:1022F00008C082E08093C1011092B2011092B10136
:102300001AC0909580911B02892B80931B029181AA
:102310008AE0989FC00111249093B2018093B1018B
:1023200084E08093C10180EA9FE00E94CF159093E2
:10233000B0018093AF0181E08093C50115C08FEF9C
:1023400080930401E091BA01F091BB0180818093F8
:102350001C0281E08093C60107C081E08093C30125
:1023600003C081E08093C7011092BF011092BB01AE
:102370001092BA011092B901E3E0CE5F0C94FD77A0
:10238000982F8091C00085FFFCCF9093C6000895E0
:102390000F931F9388E18093C1008091C0008260F9
:1023A0008093C0008091C10080688093C1008091BB
:1023B000C10080648093C10000E010E00093C5007C
:1023C0008AE290E08093C4008091B5019091B601BB
:1023D0000E94CF1590939103809390038CED90E031
:1023E0000E94CF159093C0038093BF031092920375
:1023F0008AE58093930386E0809396038BE0809335
:102400009403109295031093BB010093BA011092AC
:10241000B9011F910F910895A0E1B0E0E2E1F2E16E
:102420000C94DE7780910601882309F4C1C2809163
:10243000AF019091B0010E94D815882361F01092ED
:10244000B2011092B1011092B6011092B501109232
:10245000B4011092B3018091B1019091B201892B26
:1024600041F080917004909171040E94D8158823E6
:1024700029F48091C501882309F460C08091060188
:10248000882309F45BC08091C10107E715E084301F
:10249000A8F00E94DF1F80E590E09F938F931F9329
:1024A0000F9381E08F938F9388E48F930E94340C75
:1024B0002DB73EB7295F3F4F2DBF34C010921D028C
:1024C00087EC93E09F938F9382ED9FE19F938F938F
:1024D000E0917E03F0917F03099584E190E09F9362
:1024E0008F931F930F9381E090E09F938F9381ECE4
:1024F00091E09F938F9382E08F9381E08F9388E4A4
:102500008F930E94340C8091C101982F8F5F80932C
:10251000C1012DB73EB7215F3F4F2DBF943010F062
:102520001092C1018091B1019091B2010E94CF152A
:1025300090937104809370041092C5018091C6013C
:10254000882351F180910601882331F10E94DF1F19
:1025500080E590E09F938F9387E795E09F938F931B
:1025600021E030E03F932F9381E291E09F938F939E
:102570003F932F938CE192E09F938F9383E08F930F
:1025800081E08F938CE48F930E94340C1092C601EB
:102590008DB79EB70F968DBF8091C3018823D1F070
:1025A000809106018823B1F08AE090E09F938F9399
:1025B00082E993E09F938F9381E08F938F9386E5D9
:1025C0008F930E94340C1092C3012DB73EB7295F40
:1025D0003F4F2DBF8091C7018823D9F0809106011C
:1025E0008823B9F08BE090E09F938F9384EB93E086
:1025F0009F938F9381E08F93809103018F9387E462
:102600008F930E94340C1092C7018DB79EB7079626
:102610008DBF8091BF039091C0030E94D81588237D
:1026200009F461C080910601882309F45CC080919F
:10263000E4059927880F991F880F991F7C010027AF
:10264000F7FC0095102F8091CD029091CE02A091C1
:10265000CF02B091D002BC01CD01A80197010E9428
:10266000B7773093AD032093AC038091C50290916E
:10267000C602A091C702B091C802BC01CD01A80159
:1026800097010E94B7773093AF032093AE038091F8
:1026900050028093B00380914F028093B10388E091
:1026A00090E09F938F938CEA93E09F938F9381E0C8
:1026B0008F9383E08F938BE68F930E94340C8091ED
:1026C000B2032DB73EB7295F3F4F2DBF853018F0BD
:1026D00086E08093B20383E690E00E94CF1590934A
:1026E000C0038093BF038091B5019091B601892BFF
:1026F00041F080919003909191030E94D815882316
:1027000021F48091C401882339F180910601882346
:1027100019F10E94A03382E490E09F938F9381E2AD
:1027200095E09F938F9381E08F938F9384E48F93B1
:102730000E94340C1092C4018DB79EB707968DBFCE
:102740008091B5019091B601009731F00E94CF15AC
:1027500090939103809390038091B3019091B40181
:10276000892B09F4B8C080918E0390918F030E9449
:10277000D815882309F4AFC080910601882309F495
:10278000AAC08091E4059927880F991F880F991F87
:102790007C010027F7FC0095102F8091CD029091CD
:1027A000CE02A091CF02B091D002BC01CD01A80110
:1027B00097010E94B7773093810320938003809123
:1027C000C5029091C602A091C702B091C802BC0197
:1027D000CD01A80197010E94B7773093830320931E
:1027E00082032091C7073091C8074091C9075091D3
:1027F000CA07DA01C90163E0880F991FAA1FBB1F2E
:102800006A95D1F7820F931FA41FB51F820F931FE4
:10281000A41FB51F20913C0130913D0140913E0124
:1028200050913F01BC01CD010E94B77730938503E1
:10283000209384038091950290919602A091970233
:10284000B091980249E0B595A795979587954A95D7
:10285000D1F7809386038091910290919202A0918A
:102860009302B091940239E0B595A7959795879515
:102870003A95D1F78093870380919D0290919E02B3
:10288000A0919F02B091A00229E0B595A7959795D8
:1028900087952A95D1F7809388038EE090E09F93E7
:1028A0008F9380E893E09F938F9381E08F938F9332
:1028B00083E48F930E94340C8091B3019091B40112
:1028C0000E94CF1590938F0380938E032DB73EB750
:1028D000295F3F4F2DBF809105018F3F71F19927EF
:1028E00004E0880F991F0A95E1F789539E4F40E154
:1028F00050E0BC01CE0101960E94967580E190E007
:102900009F938F93CE0101969F938F9381E090E0E8
:102910009F938F9385E091E09F938F9382E08F93B5
:1029200081E08F9381E48F930E94340C8FEF80932A
:1029300005018DB79EB70B968DBF809163058823E7
:10294000D1F0809106018823B1F081E090E09F935F
:102950008F9383E695E09F938F9381E08F938F937E
:1029600082E48F930E94340C109263052DB73EB71A
:10297000295F3F4F2DBF8091C2018823C9F080910C
:1029800006018823A9F084E390E09F938F938CEF56
:1029900096E09F938F9381E08F938F9380E58F9341
:1029A0000E94340C1092C2018DB79EB707968DBF5E
:1029B000E6E0C05F0C94FA771F920F920FB60F9269
:1029C00011242F933F935F936F937F938F939F93E4
:1029D000AF93BF93EF93FF9320E08091D7018823BB
:1029E00029F08091D70181508093D70180916503B0
:1029F000882319F08150809365038091DF01815015
:102A00008093DF018F3F09F05BC089E08093DF0195
:102A10008091DD019091DE0101969093DE0180931B
:102A2000DD01809110018F5F8170809310018823F8
:102A300019F481E08093DC01349903C081E0809334
:102A4000E0018091D8019091D901892B21F18091E9
:102A5000D8019091D9010B9750F08091D8019091B5
:102A6000D9010A979093D9018093D80104C010929C
:102A7000D9011092D8018091D8019091D90120916B
:102A8000090130910A0182239323892B11F021E05F
:102A900008C020E006C08FEF9FEF90930A0180935B
:102AA000090180910101222331F08A3011F45A9AF0
:102AB00007C0479A05C08A3011F45A9801C0479858
:102AC0008091E001882309F45AC0209199012223C2
:102AD00009F055C08091B70783FF51C086B199278F
:102AE000FC01E071F07084FF13C08091DA019091D5
:102AF000DB0101969093DB018093DA018091DA018A
:102B00009091DB01895E9340D0F12093E00137C0C2
:102B10008091DA019091DB01892B69F18091DA01D2
:102B20009091DB018A56914030F58091DA019091C5
:102B3000DB0169E270E00E946E778091DA0190918A
:102B4000DB01860F971F9093DB018093DA01809160
:102B5000DA019091DB010B9750F08091DA019091AE
:102B6000DB010A9790938B0180938A0104C0F09354
:102B70008B01E0938A011092DB011092DA01FF9140
:102B8000EF91BF91AF919F918F917F916F915F91E5
:102B90003F912F910F900FBE0F901F90189520918D
:102BA000DD013091DE01280F391FC901019608951A
:102BB0002091DD013091DE01821B930B892F992733
:102BC0008695807490700895CF93DF930E94CF15FF
:102BD000EC01CE010E94D8158823D9F3DF91CF9163
:102BE0000895CF93DF930E94CF15EC0109C0809127
:102BF0001101882329F0909311018FEC80937A00C2
:102C0000CE010E94D815982F882389F3DF91CF91A8
:102C100008959FB7F8945F983E9A469A8091B000C5
:102C20008F708093B0008091B00083608093B0007B
:102C30008091B1008B738093B1008091B1008B6063
:102C40008093B1001092B2008FEF8093B300809117
:102C5000B00080688093B000809170008A7F80937C
:102C60007000809170008260809370009FBF089513
:102C70008AE090E00E94CF159093650580936405EB
:102C800082E085BD83EA84BD17BC84EB88BD86E005
:102C900086BD80916E00816080936E000895809162
:102CA00035062091690182FF30C09091F8058CE3D0
:102CB000989FB00111249091F70580E5989FA0019D
:102CC0001124922F905897FD9D5F9595959586E0DC
:102CD0009802C00111242091070130910801281B9E
:102CE000390B3093080120930701421753072CF04A
:102CF000509308014093070108952617370784F081
:102D000070930801609307010895822F992736E098
:102D1000880F991F3A95E1F7909308018093070176
:102D20000895A0E0B0E0E7E9F6E10C94DD7780914A
:102D3000FF05E82FFF27EE5BFE4F9681D080809144
:102D40000F01A92FBB27A7FDB095CB2FDB2F81301B
:102D500009F017C12091CD023091CE024091CF02EF
:102D60005091D002BD01CE010E94437797FF04C06D
:102D700061587F4F8F4F9F4F7B018C01C7E01595A6
:102D80000795F794E794CA95D1F78D2D992787FD7C
:102D90009095A92FB92F2091C5023091C60240917C
:102DA000C7025091C802BC01CD010E94437797FF32
:102DB00004C061587F4F8F4F9F4FB7E0959587951F
:102DC00077956795BA95D1F7F801E701C61BD70B40
:102DD000E80BF90B20914A0330914B03C901A3E0A2
:102DE000880F991FAA95E1F7821B930BAA2797FDDD
:102DF000A095BA2FC81BD90BEA0BFB0B809167017A
:102E00009927AA27BB27BC01CD019E01AF010E94D3
:102E1000437797FF04C061507E4F8F4F9F4FFC0157
:102E2000EB0179E0F595E795D795C7957A95D1F7B8
:102E300010913506609107017091080112FF05C0DD
:102E400070930E0160930D0118C040910D015091D7
:102E50000E018091FE05282F3327CB01841B950B93
:102E6000B9010E94827780910D0190910E01860F29
:102E7000971F90930E0180930D0110FF14C0809155
:102E80000D0190910E0197FD0F9664E09595879541
:102E90006A95E1F7AA2797FDA095BA2FC80FD91F09
:102EA000EA1FFB1F15C080910D0190910E0197FD47
:102EB0000F9654E0959587955A95E1F7AA2797FDC7
:102EC000A095BA2F8C1B9D0BAE0BBF0BFD01EC0127
:102ED00020913206222321F133278091D201909153
:102EE000D301829FA001839F500D929F500D11240A
:102EF000CA01AA2797FDA095BA2F8C0F9D1FAE1F60
:102F0000BF1F2F5F3F4F442737FD4095542FBC0113
:102F1000CD010E94B7773093D3012093D20104C032
:102F2000D093D301C093D2018091F705282F332786
:102F3000220F331F220F331F8091D2019091D301B2
:102F4000821793077CF08091F805282F3327220FF2
:102F5000331F220F331F8091D2019091D301281784
:102F6000390724F43093D3012093D20180910101D9
:102F7000843108F4F7C080910F018F5F80930F01B7
:102F8000F3C02091C5023091C6024091C702509112
:102F9000C802BD01CE010E94437797FF04C061586B
:102FA0007F4F8F4F9F4F7B018C0187E015950795D1
:102FB000F794E7948A95D1F78D2D992787FD909501
:102FC000A92FB92F2091CD023091CE024091CF028E
:102FD0005091D002BC01CD010E9443779B01AC010E
:102FE00097FF04C021583F4F4F4F5F4FC7E05595A3
:102FF000479537952795CA95D1F72E0D3F1D401F50
:10300000511F809166019927AA27BB27BC01CD01DA
:103010000E94437797FF04C061507E4F8F4F9F4FB0
:10302000FC01EB01B9E0F595E795D795C795BA9501
:10303000D1F7809168019927A6E0880F991FAA957A
:10304000E1F740910B0150910C012091FE053327CF
:10305000841B950BB9010E94827780910B0190919E
:103060000C01860F971F90930C0180930B018091A8
:10307000350681FF14C080910B0190910C0197FDE2
:103080000F9674E0959587957A95E1F7AA2797FDB5
:10309000A095BA2FC80FD91FEA1FFB1F15C080913A
:1030A0000B0190910C0197FD0F9664E09595879523
:1030B0006A95E1F7AA2797FDA095BA2F8C1B9D0B67
:1030C000AE0BBF0BFD01EC0120913306222321F151
:1030D00033278091D0019091D101829FA001839FDD
:1030E000500D929F500D1124CA01AA2797FDA0955B
:1030F000BA2F8C0F9D1FAE1FBF1F2F5F3F4F44275E
:1031000037FD4095542FBC01CD010E94B777309315
:10311000D1012093D00104C0D093D101C093D0013C
:103120008091FB05282F3327220F331F220F331FD7
:103130008091D0019091D101821793077CF080910A
:10314000FC05282F3327220F331F220F331F8091B6
:10315000D0019091D1012817390724F43093D1017F
:103160002093D00110920F01E7E0CDB7DEB70C94A9
:10317000F9771F920F920FB60F9211242F933F935E
:103180004F935F938F939F93EF93FF9380910101F0
:103190009091E101843108F04CC0992309F029C1D4
:1031A0008091B00086FF24C08091B0008F7B809317
:1031B000B0008091D2019091D30187559E4F90939A
:1031C000D5018093D40125E08D3D920718F08CED58
:1031D00095E005C08757914030F487E791E09093E0
:1031E000D5018093D4018091D4019091D501C2C0C2
:1031F0008091B00080648093B0008091FD05282FFD
:1032000033278DED96E0289FA001299F500D389F10
:10321000500D1124CA012091E2013091E301821B7B
:10322000930B9093D5018093D40181E080930F019B
:10323000DDC0992309F0DDC08091B00086FF9FC0FA
:103240008091B0008F7B8093B000E091E4012091E9
:10325000FD05EE23D9F433278DED96E0289FA001DC
:10326000299F500D389F500D1124CA012091E20171
:103270003091E301821B930B9093D5018093D4018D
:103280001092E3011092E201469AB0C02E1738F472
:103290008AE090E09093D5018093D401A7C089EA99
:1032A00093E09093D5018093D4018E2F992783309A
:1032B0009105D9F08430910534F48130910549F0BD
:1032C000029761F020C08430910591F0059799F044
:1032D0001AC08091D2019091D30104C08091D00195
:1032E0009091D10187559E4F1DC08091930705C0D5
:1032F00080916A0702C080919C079927880F991FC7
:10330000880F991FEFCFFF27EE0FFF1FE450F94FF3
:1033100020813181220F331F8091D4019091D501FA
:10332000820F931F9093D5018093D4018091D40193
:103330009091D50155E08D3D950718F08CED95E005
:1033400005C08757914030F487E791E09093D5010D
:103350008093D4012091D4013091D5012C5B304071
:103360003093D5012093D4018091E2019091E30143
:10337000820F931F9093E3018093E20137C0809105
:10338000B00080648093B0008CEB90E09093D50106
:103390008093D4018091E2019091E30184549F4F86
:1033A0009093E3018093E2018091D601882321F07C
:1033B00080917302882321F48091D601823011F428
:1033C000469801C0469A8091E4018F5F8093E401A2
:1033D000282F33278091FD0599270196821793079F
:1033E0002CF481E080930F011092E40181E080933E
:1033F000E1012091D4013091D50141E02F3734070C
:1034000030F08FEF8093B3002F5F30400FC02F3F1D
:103410003105C9F0C0F0A9014F5F50404F37510549
:1034200050F480E88093B300205830403093D501A9
:103430002093D40112C08FEF8093B3005093D50135
:103440004093D4010AC08091D4018093B3001092BC
:10345000D5011092D4011092E101FF91EF919F915B
:103460008F915F914F913F912F910F900FBE0F90D1
:103470001F90189510927C008FEC80937A0008952D
:10348000CF93DF931092ED0183E090E00E94192B1F
:10349000C82FDD27C531D10508F02A97C7BD84E6BE
:1034A00090E00E94F11580911501909116018052D3
:1034B000934010F4C0E0D0E0CA3FD105F8F4C7BD96
:1034C00082E390E00E94F1158CED93E09F938F933F
:1034D00080EC91E19F938F93E0917E03F0917F03C5
:1034E000099580911501909116010F900F900F9002
:1034F0000F908052934010F02196DECFC093740558
:103500006C2F83E090E00E94212B8091D50580FFF5
:103510000AC0809174058A508B3E28F080919703F1
:10352000806480939703C7BD8CE291E00E94F115FF
:10353000DF91CF910895EF92FF921F93CF9310E008
:1035400080ED97E00E94CF157C01CCE8133019F490
:10355000CB3008F0C9E010E08091FC019091FD01B2
:103560008C5F934024F48091140181500AC08091B3
:10357000FC019091FD018750944034F0809114013A
:103580008F5F8093140101C011E08091FA01909146
:10359000FB018C5F934024F48091130181500AC099
:1035A0008091FA019091FB018750944034F0809112
:1035B00013018F5F8093130101C01F5F8091F80199
:1035C0009091F9018C5F934024F480911201815015
:1035D0000AC08091F8019091F90187509440C4F09D
:1035E000809112018F5F8093120113C08EED93E0E2
:1035F0009F938F9380EC91E19F938F93E0917E0353
:10360000F0917F0309950F900F900F900F905FC07E
:103610001F5F82E180932802809122028E7F809337
:10362000220285EA8093BC00809114018A3040F424
:10363000809197038160809397038AE080931401BF
:1036400080911401863F40F08091970381608093C0
:10365000970385EF80931401809113018A3040F421
:10366000809197038260809397038AE0809313018F
:1036700080911301863F40F0809197038260809390
:10368000970385EF80931301809112018A3040F4F3
:10369000809197038460809397038AE0809312015E
:1036A00080911201863F40F080919703846080935F
:1036B000970385EF8093120180912802882339F0C7
:1036C000C7010E94D815882309F090CFF5CF10923A
:1036D00011018FEC80937A00809111018823E1F32E
:1036E000CA3020F48AE090E00E94F115C15009F040
:1036F0002DCF86E490E00E94F115CF911F91FF90AD
:10370000EF9008951F920F920FB60F921124EF922F
:10371000FF920F931F932F933F934F935F936F935A
:103720007F938F939F93AF93BF93EF93FF9380917A
:103730000502282F3327442755278F5F80930502E2
:10374000F9012231310508F0FFC3E25CFF4F0C9410
:103750000978809178009091790046C08091780036
:103760009091790054C18091780090917900909364
:103770000902809308027FC18091D7029091D802FC
:103780002091780030917900821B930B909367050C
:10379000809366058091660590916705909313026A
:1037A0008093120286C180917800909179002091D7
:1037B000D9023091DA02821B930B909373058093A8
:1037C0007205809172059091730590931502809314
:1037D0001402BCC380910C0290910D0220917800DC
:1037E00030917900820F931F90930D0280930C0209
:1037F00081E0ADC380910A0290910B022091780084
:1038000030917900820F931F90930B0280930A02EC
:1038100084E09DC380911F01909120019C01220FA3
:10382000331F280F391F809178009091790063E051
:1038300070E00E946E77260F371F369527953695D4
:1038400027953093200120931F0185E080C380914C
:103850007800909179009093690580936805809134
:103860006805909169054091D3025091D402841B60
:10387000950B2091D202332727FD3095821B930BA5
:103880009093F3018093F20180913302882309F031
:103890006DC08091F2019091F30102977CF122E0DA
:1038A0004E3E52070CF062C0209106023091070292
:1038B0002B5F3F4F30930702209306022550304084
:1038C00080913C0290913D02845F914030F4215FF1
:1038D0003F4F309307022093060280910602909199
:1038E0000702853691050CF441C04F5F5F4F50933E
:1038F000D4024093D3028456904034C08091F201A8
:103900009091F3018F5F9F4F8CF562E0473256072D
:103910006CF120910602309107022550304030931F
:103920000702209306022B5F3F4F80913C0290914B
:103930003D02845F914030F42F50304030930702B5
:103940002093060280910602909107022FEF8C3996
:10395000920764F4415050405093D4024093D302F4
:103960008C599F4F90930702809306028091F20139
:103970009091F3019C01442737FD4095542F80918D
:103980008D0290918E02A0918F02B0919002820FD1
:10399000931FA41FB51F80938D0290938E02A09356
:1039A0008F02B093900220918D0230918E0240914F
:1039B0008F025091900257FF04C021503C4F4F4F4F
:1039C0005F4F6AE055954795379527956A95D1F7EA
:1039D00080918D0290918E02A0918F02B091900201
:1039E000821B930BA40BB50B80938D0290938E02D8
:1039F000A0938F02B09390022EC180910A02909101
:103A00000B022091780030917900820F931F9093E0
:103A10000B0280930A02109204029BC28091010162
:103A20008A3071F480917800909179002091080299
:103A300030910902820F931F01969695879517C0C2
:103A40004091080250910902843158F02091780089
:103A500030917900240F351F8FEF97E0821B930B75
:103A600006C08091780090917900840F951F909303
:103A7000F9018093F80186E06AC28091D7029091A3
:103A8000D8022091780030917900821B930B90939B
:103A90006705809366058091660590916705209182
:103AA000120230911302820F931F9093F7018093BB
:103AB000F60187E04CC280917800909179002091C6
:103AC000D9023091DA02821B930B90937305809395
:103AD00072058091720590917305209114023091C6
:103AE0001502820F931F9093F5018093F4012EC26B
:103AF00020910C0230910D02809178009091790014
:103B0000280F391F30930D0220930C028091010180
:103B10008A3019F4220F331F04C0220F331F220FE3
:103B2000331F30930D0220930C0220910C02309130
:103B30000D02C90137FD079603E0959587950A9513
:103B4000E1F79093FD018093FC0180910E0290912A
:103B50000F02820F931F97FD01969595879590937D
:103B60000F0280930E022091E3023091E402821B47
:103B7000930B90931E0180931D01209102023091BE
:103B8000030280911D0190911E01280F391F37FFFC
:103B900002C02F5F3F4F3595279530930302209346
:103BA000020226CE20910A0230910B028091780009
:103BB00090917900280F391F30930B0220930A024D
:103BC000809101018A3019F4220F331F04C0220FA3
:103BD000331F220F331F30930B0220930A022091D0
:103BE0000A0230910B02C90137FD0796F3E0959563
:103BF0008795FA95E1F79093FB018093FA01809104
:103C0000100290911102820F931F97FD01969595D6
:103C1000879590931102809310022091E1023091D8
:103C2000E202821B930B90931C0180931B01209155
:103C300000023091010280911B0190911C01280F1C
:103C4000391F37FF02C02F5F3F4F359527953093BF
:103C500001022093000283E07AC180916D0290916D
:103C60006E02A0916F02B09170028093E501909373
:103C7000E601A093E701B093E8011092050281E00C
:103C8000809311018091E9019091EA01019690934E
:103C9000EA018093E90180917800909179009093F6
:103CA0001601809315018091150190911601AA27A4
:103CB000BB272091160230911702409118025091B3
:103CC0001902280F391F4A1F5B1F209316023093D9
:103CD0001702409318025093190280911A028F5FC5
:103CE00080931A02803108F431C1809117019091BC
:103CF0001801A0911901B0911A017C018D0163E0B6
:103D0000EE0CFF1C001F111F6A95D1F7E81AF90A83
:103D10000A0B1B0BE20EF31E041F151F8091ED0111
:103D2000992787FD9095A92FB92FBC01CD0120EBD4
:103D300030E240E050E00E944377DC01CB01E81A1A
:103D4000F90A0A0B1B0BD801C7010496A11DB11D6E
:103D5000B7FF05C0D801C7010B96A11DB11D23E017
:103D6000B595A795979587952A95D1F780931701D3
:103D700090931801A0931901B0931A01E0906A057D
:103D8000F0906B0500916C0510916D058091170105
:103D900090911801A0911901B0911A01E81AF90A3D
:103DA0000A0B1B0BE0926D02F0926E0200936F0201
:103DB000109370022091EE013091EF014091F001DB
:103DC0005091F10157FF04C0215F3F4F4F4F5F4FAC
:103DD00084E055954795379527958A95D1F7809139
:103DE000EE019091EF01A091F001B091F101821BE1
:103DF000930BA40BB50B8093EE019093EF01A0936E
:103E0000F001B093F1018091EE019091EF01A0914A
:103E1000F001B091F1018E0D9F1DA01FB11F809385
:103E2000EE019093EF01A093F001B093F101809126
:103E3000EE019091EF01A091F001B091F101B7FF77
:103E400003C00F96A11DB11D14E0B595A7959795D8
:103E500087951A95D1F720916D0230916E02281B3B
:103E6000390B64E0213036071CF020E034E006C056
:103E70008CEF2030380714F420E03CEF8091EB0108
:103E80009091EC018091EB019091EC0197FF03C0C0
:103E9000909581959F4FA901F3E0440F551FFA9526
:103EA000E1F78D5B9240C4F08091EB019091EC01C1
:103EB0009C01E4E0220F331FEA95E1F7281B390B40
:103EC000240F351F37FF02C0215F3F4F74E0359547
:103ED00027957A95E1F717C08091EB019091EC015D
:103EE0009C0165E0220F331F6A95E1F7281B390B0F
:103EF000240F351F37FF02C0215E3F4F45E0359547
:103F000027954A95E1F73093EC012093EB018091DE
:103F1000160290911702A0911802B0911902B7FFF2
:103F200003C00196A11DB11DB595A79597958795DD
:103F30008093160290931702A0931802B09319026F
:103F400088E080931A0202C01092050282E08093FA
:103F500004028091040280937C00809105028823F2
:103F600019F08FEC80937A00FF91EF91BF91AF91A0
:103F70009F918F917F916F915F914F913F912F9181
:103F80001F910F91FF90EF900F900FBE0F901F9019
:103F9000189590E2E7E7F5E08FE49193815087FF71
:103FA000FCCF089590911D02903540F4E92FFF2732
:103FB000E958FA4F80839F5F90931D020895AF9256
:103FC000BF92CF92DF92FF920F931F93CF93DF9315
:103FD00020911B0220FF0AC080911C02882311F04F
:103FE000815002C08091210180931C0221FF0CC0EE
:103FF00090911C0280912101981719F410921C02D3
:1040000003C09F5F90931C02822F992780FF04C0FA
:1040100081FF02C010921C020E94C91F80911C02E5
:10402000282F332792EDC92E9FE1D92EC0917E0310
:10403000D0917F038A3098F481E180931D023F93F1
:104040002F9385E194E09F938F93DF92CF92FE01AF
:1040500009952DB73EB72A5F3F4F2DBF11C080E1B4
:1040600080931D023F932F938AE194E09F938F9357
:10407000DF92CF92FE0109958DB79EB706968DBF50
:1040800020911C02822F9927AA27BB27FC01419768
:1040900010F00C941429E05BFF4F02EDC02E0FE1ED
:1040A000D02EC0917E03D0917F030C94097810929A
:1040B0001D028FE194E09F938F9302ED1FE1DF9249
:1040C000CF92FE01099584E180931D020F900F901D
:1040D0000F900F9087E690E09F938F938AE590E092
:1040E0009F938F931F921F92809101016AE00E941B
:1040F0006277892F99279F938F93809101010E9466
:10410000627799279F938F938FE294E09F938F9389
:10411000DF92CF92E0917E03F0917F03099588E2D0
:1041200080931D02EDB7FEB73E96EDBF86E496E0A4
:104130009F938F930E94912C99279F938F9387E44D
:1041400094E09F938F93DF92CF92E0917E03F09162
:104150007F030995809198032DB73EB7285F3F4FA5
:104160002DBF84FF06C08CE380931D0285E594E09B
:10417000D2C090919703992351F08CE380931D0254
:10418000892F99279F938F9382E694E03BC190916A
:1041900023029923B1F08CE380931D02892F992784
:1041A0009F938F9389E794E09F938F931F930F932F
:1041B000E0917E03F0917F030995EDB7FEB7369647
:1041C00079C490915103992371F08CE380931D027F
:1041D000892F99279F938F938EE894E09F938F93D5
:1041E0001F930F93D9C480913601909137010697A0
:1041F00010F00C941D298CE380931D028FE994E04C
:10420000A5C78091B70712EDC12E1FE1D12EC09135
:104210007E03D0917F0380FF6BC010921D028091BE
:104220006D0290916E02A0916F02B0917002BC017C
:10423000CD0125E030E040E050E00E94B7773F93A9
:104240002F938CEA94E09F938F93DF92CF92FE019D
:10425000099584E180931D028DB79EB706968DBFA8
:104260008091690290916A02A0916B02B0916C02F8
:10427000BC01CD0125E030E040E050E00E94B7777E
:104280003F932F9389EB94E09F938F93DF92CF928C
:10429000E0917E03F0917F03099588E280931D02EF
:1042A000EDB7FEB73696EDBF8091150190911601DE
:1042B0009F938F9386EC94E09F938F93DF92CF929E
:1042C000E0917E03F0917F0309958CE380931D02BA
:1042D0002DB73EB72A5F3F4F2DBF87B599279F93D4
:1042E0008F9383ED94E09F938F93DF92CF928EC054
:1042F00010921D0280EE94E09F938F93DF92CF92F5
:10430000FE01099584E180931D020F900F900F909C
:104310000F908FEE94E09F938F93DF92CF921AC706
:1043200010921D0288EF94E09F938F9302ED1FE19E
:10433000DF92CF92FE01099584E180931D020F90D8
:104340000F900F900F908091CD029091CE02A0918E
:10435000CF02B091D002B7FF04C081509C4FAF4F45
:10436000BF4FCAE0B595A79597958795CA95D1F7A0
:10437000BF93AF939F938F9385E095E09F938F9327
:104380001F930F93E0917E03F0917F03099588E2DC
:1043900080931D02EDB7FEB73896EDBF8091C50240
:1043A0009091C602A091C702B091C802B7FF04C0A5
:1043B00081509C4FAF4FBF4FFAE0B595A7959795A9
:1043C0008795FA95D1F7BF93AF939F938F9384E12D
:1043D00095E09F938F931F930F93E0917E03F0914D
:1043E0007F0309958CE380931D022DB73EB7285FAC
:1043F0003F4F2DBF80917207909173079F938F93CA
:1044000083E295E09F938F931F930F93E0917E0338
:10441000F0917F0309958DB79EB706968DBF0DC7A6
:10442000E1E0FE2EC1E0D0E00EEF16E09F2D969564
:1044300084E1989FC001112480931D02F8018281BC
:1044400093819F938F932196DF93CF9321978081C0
:1044500091819F938F93DF93CF9382E395E09F9316
:104460008F9382ED9FE19F938F93E0917E03F09174
:104470007F0309952DB73EB7245F3F4F2DBF32E034
:10448000F30E22960C5F1F4F88E08F1578F6D5C685
:1044900010921D028091CA05E82FFF27EE0FFF1F23
:1044A000E450F94F808191819F938F938091C9054A
:1044B000E82FFF27EE0FFF1FE450F94F8081918115
:1044C0009F938F9384E495E09F938F93DF92CF9295
:1044D000FE01099584E180931D02EDB7FEB7389681
:1044E000EDBF8091CC05E82FFF27EE0FFF1FE450B2
:1044F000F94F808191819F938F938091CB05E82F15
:10450000FF27EE0FFF1FE450F94F80819181815802
:104510009F4F9F938F9384E595E09F938F93DF92B6
:10452000CF92E0917E03F0917F03099588E280931A
:104530001D022DB73EB7285F3F4F2DBF8091CE059E
:10454000E82FFF27EE0FFF1FE450F94F8081918184
:1045500081589F4F9F938F938091CD05E82FFF2720
:10456000EE0FFF1FE450F94F8081918181589F4FDA
:104570009F938F9384E695E09F938F93DF92CF92E2
:10458000E0917E03F0917F0309958CE380931D02F7
:104590008DB79EB708968DBF8091D005E82FFF2775
:1045A000EE0FFF1FE450F94F8081918181589F4F9A
:1045B0009F938F938091CF05E82FFF27EE0FFF1F6A
:1045C000E450F94F8081918181589F4F9F938F9341
:1045D00084E795E063C210921D0284E895E09F9302
:1045E0008F9302ED1FE1DF92CF92FE01099580913A
:1045F00001010F900F900F900F908A3009F09DC02D
:1046000084E180931D028091E3029091E4029C0179
:1046100097FF02C0295F3F4F287F821B930B9F9318
:104620008F938091E3029091E40297FD079673E0E7
:10463000959587957A95E1F79F938F932091E30263
:104640003091E40237FF02C0295F3F4F63E03595A8
:1046500027956A95E1F78091FC019091FD01821BFD
:10466000930B9F938F9382E995E09F938F931F9372
:104670000F93E0917E03F0917F03099588E2809388
:104680001D022DB73EB7265F3F4F2DBF8091E1023F
:104690009091E2029C0197FF02C0295F3F4F287F63
:1046A000821B930B9F938F938091E1029091E20282
:1046B00097FD079653E0959587955A95E1F79F9357
:1046C0008F932091E1023091E20237FF02C0295F0F
:1046D0003F4F43E0359527954A95E1F78091FA01E0
:1046E0009091FB01821B930B9F938F9383EA95E03C
:1046F0009F938F931F930F93E0917E03F0917F031D
:1047000009958CE380931D028DB79EB70A968DBFE5
:104710008091DF029091E0029F938F938091DF025E
:104720009091E0022091F8013091F901821B930BE6
:104730009F938F9384EB95E0ADC08B3019F084315B
:1047400008F4ADC084E180931D028091E302909152
:10475000E4029C0197FF02C0215F3F4F207F821B34
:10476000930B97FD0196959587959F938F938091D5
:10477000E3029091E40297FD0F9624E095958795CA
:104780002A95E1F79F938F932091E3023091E40201
:1047900037FF02C0295F3F4FC3E035952795CA9583
:1047A000E1F78091FC019091FD01821B930B9F9397
:1047B0008F9382EC95E09F938F931F930F93E091DB
:1047C0007E03F0917F03099588E280931D022DB747
:1047D0003EB7265F3F4F2DBF8091E1029091E202EC
:1047E0009C0197FF02C0215F3F4F207F821B930BEC
:1047F00097FD0196959587959F938F938091E10200
:104800009091E20297FD0F96A4E095958795AA9561
:10481000E1F79F938F932091E1023091E20237FFFD
:1048200002C0295F3F4FF3E035952795FA95E1F7F0
:104830008091FA019091FB01821B930B9F938F93C0
:1048400084ED95E09F938F931F930F93E0917E03E8
:10485000F0917F0309958CE380931D028DB79EB77D
:104860000A968DBF8091DF029091E00297FD01963C
:10487000959587959F938F938091DF029091E002A9
:104880002091F8013091F901821B930B9F938F9334
:1048900086EE95E09F938F931F930F9303C18D3006
:1048A00009F0CBC484E180931D0280911401992703
:1048B0009F938F938091E3029091E40297FD0F966E
:1048C00074E0959587957A95E1F79F938F93209162
:1048D000E3023091E40237FF02C0295F3F4F63E0FB
:1048E000359527956A95E1F78091FC019091FD013E
:1048F000821B930B9F938F9385EF95E09F938F93EC
:104900001F930F93E0917E03F0917F03099588E256
:1049100080931D022DB73EB7265F3F4F2DBF80917C
:10492000130199279F938F938091E1029091E20266
:1049300097FD0F9654E0959587955A95E1F79F93CB
:104940008F932091E1023091E20237FF02C0295F8C
:104950003F4F43E0359527954A95E1F78091FA015D
:104960009091FB01821B930B9F938F9389E096E0BC
:104970009F938F931F930F93E0917E03F0917F039A
:1049800009958CE380931D028DB79EB70A968DBF63
:104990008091120199279F938F938091DF029091CC
:1049A000E00297FD0196959587959F938F9380914F
:1049B000DF029091E0022091F8013091F901821B11
:1049C000930B9F938F938DE196E09F938F931F930B
:1049D0000F93E0917E03F0917F030995EDB7FEB749
:1049E0003A9668C010921D0281E396E09F938F93E0
:1049F000DF92CF92FE01099584E180931D020F9012
:104A00000F900F900F908091D9029091DA029F93AE
:104A10008F938091F4019091F5019F938F938EE392
:104A200096E09F938F93DF92CF92E0917E03F09177
:104A30007F03099588E280931D022DB73EB7285F5A
:104A40003F4F2DBF8091D7029091D8029F938F93B3
:104A50008091F6019091F7019F938F938DE496E0FA
:104A60009F938F93DF92CF92E0917E03F0917F032B
:104A700009958CE380931D028DB79EB708968DBF74
:104A80008091D3029091D4029F938F938091F201F1
:104A90009091F3019F938F938CE596E09F938F9372
:104AA000DF92CF92E0917E03F0917F030995EDB7FD
:104AB000FEB73896EDBFC1C310921D0280911F0151
:104AC000909120016AE070E00E9482779F938F931B
:104AD00080911F01909120016AE070E00E9482772E
:104AE0007F936F938BE696E09F938F93DF92CF92A5
:104AF000FE01099584E180931D022DB73EB7285F22
:104B00003F4F2DBF80915708909158086AE070E0A0
:104B10000E946E779F938F938091570890915808C9
:104B20006AE070E00E946E777F936F938FE796E064
:104B30009F938F93DF92CF92E0917E03F0917F035A
:104B4000099588E280931D028DB79EB708968DBFA8
:104B50008091590890915A089F938F9383E996E02A
:104B60009F938F93DF92CF92E0917E03F0917F032A
:104B700009958CE380931D02EDB7FEB73696EDBF25
:104B800080915B0890915C089F938F9383EA96E0F5
:104B90009F938F93DF92CF92E0917E03F0917F03FA
:104BA00009952DB73EB72A5F3F4F4FC110921D02A6
:104BB00085EB96E09F938F93DF92CF92FE0109954C
:104BC00084E180931D020F900F900F900F908091C1
:104BD000FC069091FD069F938F938EEB96E09F933A
:104BE0008F93DF92CF92E0917E03F0917F0309953E
:104BF00088E280931D028DB79EB706968DBF809187
:104C0000730299279F938F938EEC96E09F938F93D7
:104C1000DF92CF92E0917E03F0917F0309958CE3C0
:104C200080931D02EDB7FEB73696EDBF8091FB066F
:104C3000992701979F938F938EED96E0A9CF1092BD
:104C40001D028EEE96E09F938F93DF92CF92FE012E
:104C5000099584E180931D020F900F900F900F90A3
:104C600080918A0190918B019F938F9386EF96E0BC
:104C70009F938F93DF92CF92E0917E03F0917F0319
:104C8000099588E280931D028DB79EB706968DBF69
:104C900080917207909173079F938F9384E097E0C0
:104CA0009F938F93DF92CF92E0917E03F0917F03E9
:104CB00009958CE380931D02EDB7FEB73696EDBFE4
:104CC00080918B0290918C029F938F9382E197E069
:104CD0005FCFC4E7CC2EC2E0DC2E20E030E0E9015B
:104CE000B3E0FB2EC0931D02F60181916F0199275D
:104CF0009F938F9389010F5F1F4F1F930F9380E244
:104D000097E09F938F9382ED9FE19F938F93E09124
:104D10007E03F0917F0309952DB73EB7285F3F4F83
:104D20002DBFFA9464969801F7FEDCCF86C2A8E7FF
:104D3000CA2EA2E0DA2EC0E0D0E08E01F3E0FF2E12
:104D400000931D02F60181916F0199279F938F9324
:104D50002596DF93CF938DE297E09F938F9382ED1B
:104D60009FE19F938F93E0917E03F0917F030995DC
:104D70002DB73EB7285F3F4F2DBFFA940C5E1F4FF3
:104D80002497F7FEDDCF59C210921D028AE397E007
:104D90009F938F9302ED1FE1DF92CF92FE01099561
:104DA00084E180931D020F900F900F900F908091DF
:104DB000690199279F938F9382E497E09F938F9344
:104DC000DF92CF92E0917E03F0917F03099588E214
:104DD00080931D028DB79EB706968DBF8091D2013C
:104DE0009091D30197FD0396959587959595879515
:104DF0009F938F9380E597E09F938F931F930F93DB
:104E0000E0917E03F0917F0309958CE380931D026E
:104E1000EDB7FEB73696EDBF8091F80599279F93C1
:104E20008F938091F70599279F938F938EE597E055
:104E30009F938F931F930F93E0917E03F0917F03D5
:104E400009952DB73EB7285F3F4F2DBFF6C1109291
:104E50001D028CE697E09F938F9372EDA72E7FE162
:104E6000B72EDF92CF92FE0109950F900F900F9011
:104E70000F90CBE9D6E000E010E062E0F62E802F44
:104E80008C5E80931D028B8D99278F7790709F93F6
:104E90008F938B8999278F7790709F938F938B85B2
:104EA00099278F7790709F938F938B8199278F7716
:104EB00090709F938F938CE797E09F938F93BF920F
:104EC000AF92E0917E03F0917F0309958DB79EB775
:104ED0000C968DBFFA940C5E1F4FA096F7FECFCFB5
:104EE000ACC110921D028DE897E09F938F9352ED15
:104EF000A52E5FE1B52EDF92CF92FE0109950F90AE
:104F00000F900F900F90CBE9D6E000E010E042E068
:104F1000F42E802F8C5E80931D028F8D992787FD44
:104F200090959F938F938F89992787FD90959F9355
:104F30008F938F85992787FD90959F938F938F816E
:104F4000992787FD90959F938F938CE997E09F9386
:104F50008F93BF92AF92E0917E03F0917F0309950A
:104F6000EDB7FEB73C96EDBFFA940C5E1F4FA096CE
:104F7000F7FECFCF62C110921D028DEA97E09F939A
:104F80008F9302ED1FE1DF92CF92FE01099584E13C
:104F900080931D020F900F900F900F908091B60696
:104FA000881F8827881F97E0899FC00111248D964C
:104FB0009F938F938091AE06881F8827881F96E065
:104FC000899FC00111248D969F938F938091A6068F
:104FD000881F8827881F95E0899FC00111248D961E
:104FE0009F938F9380919E06881F8827881F9927FB
:104FF000880F991F880F991F8D969F938F938CEB25
:1050000097E09F938F93DF92CF92E0917E03F09190
:105010007F03099588E280931D022DB73EB7245F78
:105020003F4F2DBF8091D606881F8827881F9BE0A1
:10503000899FC00111248D969F938F938091CE06F6
:10504000881F8827881F9AE0899FC00111248D96A8
:105050009F938F938091C606881F8827881F99E0A9
:10506000899FC00111248D969F938F938091BE06D6
:10507000881F8827881F992723E0880F991F2A9562
:10508000E1F78D969F938F9380ED97E09F938F9399
:10509000DF92CF92E0917E03F0917F0309958CE33C
:1050A00080931D028DB79EB70C968DBF8091DE0652
:1050B000881F8827881F9CE0899FC00111248D9636
:1050C0009F938F9384EE97E09F938F93DF92CF927D
:1050D000E0917E03F0917F0309958091E606EDB79C
:1050E000FEB73696EDBF87FF12C080E480931D02A5
:1050F00085EF97E09F938F93DF92CF92E0917E03AD
:10510000F0917F0309950F900F900F900F90809171
:10511000EE0687FF12C084E480931D0288EF97E0BB
:105120009F938F931F930F93E0917E03F0917F03E2
:1051300009950F900F900F900F908091F60687FFC2
:105140007CC088E480931D028BEF97E09F938F9340
:105150001F930F93E0917E03F0917F0309950F90C9
:105160000F900F900F9069C010921D028EEF97E084
:105170009F938F93DF92CF92FE01099584E18093F4
:105180001D020F900F900F900F908091A8019091A9
:10519000A9019F938F938CE098E09F938F93DF9268
:1051A000CF92E0917E03F0917F03099588E280938E
:1051B0001D022DB73EB72A5F3F4F2DBF8091AA0138
:1051C0009091AB019F938F9389E198E09F938F9388
:1051D000DF92CF92E0917E03F0917F03099589E4FD
:1051E00080931D028DB79EB706968DBF86E298E02C
:1051F0009F938F93DF92CF92E0917E03F0917F0394
:10520000099580911B020F900F900F900F9083FFD4
:1052100014C01092AB011092AA0160E070E08EE021
:1052200090E00E94322B09C080912101281719F4C7
:1052300021502093210110921C0210921B02DF9139
:10524000CF911F910F91FF90DF90CF90BF90AF90C3
:105250000895F999FECF92BD81BDF89A80B599273E
:105260000895F999FECF1FBA92BD81BD60BD0FB6FA
:10527000F894FA9AF99A0FBE08954AEA20E030E0CD
:105280002617370740F4FC018191480F2F5F3F4FED
:1052900026173707C8F3842F99270895EAEA40E0D4
:1052A00050E04617570778F49C01F999FECF32BDBC
:1052B00021BDF89A80B5E80F4F5F5F4F2F5F3F4FDA
:1052C0004617570790F38E2F9927089581E0809312
:1052D000CB0582E08093CA0583E08093C90584E012
:1052E0008093CC0585E08093CD0586E08093CE0544
:1052F00087E08093CF0588E08093D00589E0809394
:10530000D1058AE08093D2058BE08093D3058CE0B1
:105310008093D40508958DE58093C8058CE0E8E37B
:10532000F6E011928A95E9F780910101843150F0FD
:105330008AE08093E80510920C068BE18093E405E7
:105340008EE40AC083E08093E80580E280930C0637
:105350008EE18093E40585E58093090680930A0633
:1053600080E280930B06109234068AE68093D5057E
:1053700082E28093360680E48093370666E060938D
:10538000EF0510922C061092290648E04093E205A2
:1053900056EE5093E3058093E5059EE19093D60584
:1053A0008FEF8093D8052FE02093D9059093D705F0
:1053B0001092DB054093DC0584E18093DD051092BB
:1053C000DE052093DA051092F1051092F205109295
:1053D000F3051092F40510920E0610920F0610922B
:1053E00010061092110690E89093F50532E3309381
:1053F000F60582E0809335062093F7055093F80573
:1054000084E08093FD052DE720930006209301069C
:10541000209302069093F90555E55093FA0586E42A
:105420008093FB058CED8093FC058CE38093FE0557
:105430001092FF058FE58093120683EF8093140688
:105440008AEA809316068093170688E280931306F3
:105450008093150610921806309303069AE59093F0
:105460000406309305068EEF8093190684E6809338
:105470001A0690931B0690931C0690931D068BE4CE
:1054800080931E0650931F068093200610922106DB
:105490006093220640932306909324068AE2809329
:1054A000250685EF809326068CE88093270685E005
:1054B0008093280610922A0610922B0681E2809390
:1054C000EC0581E48093ED059093EE0510922D0696
:1054D00010922E0610922F0686E9809330062093B4
:1054E000060684E380930706109231061092320676
:1054F0001092330608950E948B298AE08093DF057D
:1055000080E18093E00526E02093E1059AE5909301
:10551000E60588E78093E7059093E9058093EA051F
:105520002093EB0580E28093F0058CE380930806DE
:105530008BE480930D0686E491E6A3E7B4E78093BD
:10554000380690933906A0933A06B0933B066CE771
:1055500070E088EC95E00E943D2980934406089510
:10556000CF93DF930E948B2988E08093DF0530E1A1
:105570003093E00526E02093E10594E69093E6055C
:1055800088E78093E7059093E9058093EA052093E7
:10559000EB053093F00586E48093080680930D06B2
:1055A000A8E3B6E0E2E2F1E0ED01019009922A956C
:1055B000E1F76CE770E0CD01805790400E943D29F3
:1055C00080934406DF91CF9108950E948B2926E0B5
:1055D0002093DF058AE08093E00584E08093E10575
:1055E00094E69093E60588E78093E7059093E905B4
:1055F0008093EA052093EB0580E18093F00586E433
:105600008093080680930D0685E491E6A3E7B9E749
:105610008093380690933906A0933A06B0933B06E0
:105620006CE770E088EC95E00E943D298093440689
:105630000895F999FECF92BD81BDF89A80B599275A
:105640000895F999FECF1FBA92BD81BD60BD0FB616
:10565000F894FA9AF99A0FBE089569E279E20E94E5
:10566000D175089541E359E20E940B760895EF92B7
:10567000FF920F931F93CF93C82F8150853008F06E
:10568000C3E08DE7C89F8001112487EEE82E8FEFDD
:10569000F82EE00EF11E6CE770E0C7010E944E2963
:1056A000682F98012D593F4F8FB39927AC01427055
:1056B000507081FDF9CF32BD21BDF89A80B58617B3
:1056C00011F0CA0121C08FB399279C01227030705C
:1056D00081FDF9CFF2BCE1BCF89A80B58D3511F0AF
:1056E000C90112C08DE7C89FC0011124499729E262
:1056F00039E24DE750E0BC0188EC95E00E94AC75C2
:105700000E94076981E090E0CF911F910F91FF9077
:10571000EF900895282F863010F025E003C08823ED
:1057200009F421E0F999FECF1FBA82E090E092BD22
:1057300081BD20BD0FB6F894FA9AF99A0FBE08956C
:10574000CF93C82F8091C8058D3509F04FC0C63062
:1057500010F0C5E003C0CC2309F448C00E94B37424
:105760008091370682FF07C08091ED05843618F0DE
:1057700080E58093ED056CE770E088EC95E00E9491
:105780003D29809344068DE7C89FC001112421E381
:1057900039E24DE750E068EC75E049970E94E97501
:1057A00021E339E24CE050E069EC75E080E590E0FF
:1057B0000E94E9756CE070E089EC95E00E943D295B
:1057C000282FF999FECF1FBA8CE590E092BD81BDDC
:1057D00020BD0FB6F894FA9AF99A0FBE8C2F0E944A
:1057E0008A2B0E94076981E090E002C080E090E08F
:1057F000CF9108956DE470E088EE93E00E944E2909
:10580000482F8FB399279C012270307081FDF9CF0A
:1058100085E394E092BD81BDF89A80B5841779F450
:105820008FB399279C012270307081FDF9CF88EEEB
:1058300093E092BD81BDF89A80B5813011F0C90125
:10584000089529E239E24EE450E068EE73E085E421
:1058500096E00E94AC7581E090E008958091450645
:105860008130A9F46DE470E085E496E00E943D2962
:105870008093920621E339E24EE450E065E476E05D
:1058800088EE93E00E94E97581E090E0089580E061
:1058900090E00895CF93DF9381E080934506E5E49F
:1058A000F6E08FE0158616861786108A81503496AA
:1058B00087FFF8CF80E480935206809353061092BE
:1058C0005406809355068093560690EC90935706A5
:1058D000109258068093590680935A0610925B06E0
:1058E00090935C0690935D0680935E0610925F062F
:1058F0008093600690936106A6E4B6E08CE0E9E24E
:10590000F1E0ED01019009928A95E1F76DE470E014
:10591000CD0101970E943D2980939206DF91CF919E
:105920000895F999FECF82E090E092BD81BDF89A8A
:1059300080B5282F863078F023E0322FF999FECFFA
:105940001FBA82E090E092BD81BD30BD0FB6F894E1
:10595000FA9AF99A0FBE822F992708951F93CF9331
:10596000C82F162F863010F0C5E003C0882309F435
:10597000C1E08C2F99278230910541F08330910549
:1059800044F4019731F40E947B2A05C00E94B02A9A
:1059900002C00E94E52A1123E1F06CE070E080E58E
:1059A00090E00E944E29282FF999FECF8CE590E0D7
:1059B00092BD81BDF89A80B5821759F429E239E287
:1059C0004CE050E060E570E089EC95E00E94AC7539
:1059D00002C00E9466298C2F0E94A02BCF911F919C
:1059E0000895DF92EF92FF920F931F93CF93FF24BE
:1059F000DF2CEF2C81E090E00E94192B8B3211F00C
:105A000031E0E32E6CE070E080E590E00E944E29EA
:105A1000C82FF999FECF8CE590E092BD81BDF89A30
:105A200080B58C1711F421E0D22EC1E001E010E026
:105A3000EE2029F48C2F0E94372B8823C9F591E0A2
:105A4000F92E1F930F938EE298E09F938F9380EC33
:105A500091E19F938F93E0917E03F0917F030995ED
:105A60002DB73EB72A5F3F4F2DBF0230110549F0D9
:105A7000033011054CF40130110531F40E947B2AEA
:105A800005C00E94B02A02C00E94E52ADD2059F01C
:105A900029E239E24CE050E060E570E089EC95E005
:105AA0000E94AC7502C00E9466298C2F0E94A02B18
:105AB000CF5F0F5F1F4FC63008F4BACFFF2019F039
:105AC00083E00E948A2B0E94912CC82F0E94372BC2
:105AD0008C2F99279F938F9384E598E09F938F93C2
:105AE00000EC11E11F930F93E0917E03F0917F038F
:105AF000099581E090E00E94192B2DB73EB72A5FEF
:105B00003F4F2DBF8F3F21F00E94FA2B882399F43D
:105B10008DE698E09F938F931F930F93E0917E0300
:105B2000F0917F0309950E944A2C0E942E2C0F9021
:105B30000F900F900F90EE2029F06BE281E090E043
:105B40000E94212B1092C70590E0E2E5F6E0CFE03D
:105B50008081349618160CF49F5FC150C7FFF8CFB0
:105B60009093C705892F99279F938F9386E496E09A
:105B70009F938F938EE898E09F938F931F930F933B
:105B8000E0917E03F0917F0309950E949E058DB7F9
:105B90009EB708968DBFCF911F910F91FF90EF9008
:105BA000DF900895982F2FB7F8943998389A88B1D4
:105BB000836088B98091B9008C7F8093B9008AE2B4
:105BC0008093B800109228021092260210922502AB
:105BD000992379F0EBE9F6E08BE0108211821282D2
:105BE000138214821582168217828150389687FF9D
:105BF000F4CF78942FBF08951092280284E98093FF
:105C0000BC0080E88093BC001092BD001092BA00E6
:105C10001092BB001092B9001092B80010922402AA
:105C200080E00E94D22D1092BB0085E88093BC00DA
:105C30008091220282608093220208951F920F9227
:105C40000FB60F9211242F933F934F935F938F932F
:105C50009F93EF93FF9380912802282F33274427A7
:105C600055278F5F80932802F9012731310508F00D
:105C7000C2C2EF59FF4F0C94097881E0809324024F
:105C800009C0809126028C3090F4809126028F5FAB
:105C90008093260280912602E82FFF27EE0FFF1F38
:105CA000EE0FFF1FEB5BF94F8585181654F78091B7
:105CB00026028C3070F01092210210922002109275
:105CC000260285E08093280280912502880F8D5A54
:105CD00004C080912602880F8E5A8093BB0085E80D
:105CE0007FC280912602E82FFF2783E0EE0FFF1F7F
:105CF0008A95E1F7E556F94F81818093BB0085E8ED
:105D00008093BC0080912602E82FFF27EE0FFF1F33
:105D1000EE0FFF1FEE0FFF1FE556F94F808180FF4A
:105D200091C080912602E82FFF27EE0FFF1FEE0F94
:105D3000FF1FEE0FFF1FE556F94F8281882329F0E0
:105D40008091C705873008F46CC280912002909141
:105D50002102892B09F065C280911E0290911F02D9
:105D6000892B09F05EC26EC08091260221E030E0EE
:105D700002C0220F331F8A95E2F780911E02909194
:105D80001F0228233923232B79F080912602E82F44
:105D9000FF27EE0FFF1FEE0FFF1FEE0FFF1FE55651
:105DA000F94F80E184830DC080912602E82FFF2700
:105DB000EE0FFF1FEE0FFF1FEE0FFF1FE556F94F0F
:105DC000148280912602E82FFF2753E0EE0FFF1F79
:105DD0005A95E1F7E556F94F8481282F332743E0A0
:105DE000220F331F4A95E1F780912602E82FFF2703
:105DF00093E0EE0FFF1F9A95E1F7E556F94F828188
:105E00008770822B8093BB0085E88093BC00209133
:105E1000260281E090E002C0880F991F2A95E2F7E0
:105E2000209120023091210282239323892B51F06B
:105E300083E996E090932C0280932B0288E0809374
:105E40002D02EFC184E089C1E0912B02F0912C0278
:105E500081918093BB0085E88093BC00F0932C0275
:105E6000E0932B0280912D02815080932D02882394
:105E700009F4D7C183E071C18091B900803351F535
:105E800080912902882329F4809126028F5F8093D4
:105E9000290280912602E82FFF2783E0EE0FFF1FE3
:105EA0008A95E1F7E556F94F838199278F779070AE
:105EB0008F3791057CF480912602E82FFF27EE0FA3
:105EC000FF1FEE0FFF1FEE0FFF1FE556F94F8381F7
:105ED0008F5F83831092280284E98093BC008AE05C
:105EE00090E09093370180933601809126028F5F76
:105EF00080932602109228026DC18091B9008034EF
:105F0000C9F180912502E82FFF27EE0FFF1FEE0F4A
:105F1000FF1FEE0FFF1FE556F94F83818F778383B5
:105F2000809125028F5F80932502809125028C301D
:105F3000A0F01092250210921F0210921E02809172
:105F40002A028F5F80932A028C3038F010922A0246
:105F5000809122028D7F80932202809122028160B3
:105F6000809322021092280284E98093BC00109250
:105F7000240273C080912502E82FFF27EE0FFF1F38
:105F8000EE0FFF1FEE0FFF1FE556F94F838180686C
:105F9000838380912502E82FFF27EE0FFF1FEE0F6E
:105FA000FF1FEE0FFF1FE556F94F808180FF2FC0C6
:105FB00080912502E82FFF2753E0EE0FFF1F5A952F
:105FC000E1F7E556F94F84819927009751F0409702
:105FD000D9F583E996E090932C0280932B0288E018
:105FE00031C080912502992743E0880F991F4A9577
:105FF000E1F78056994F90932C0280932B02909159
:10600000250280912A029817E1F483E01BC0809159
:106010002502992733E0880F991F3A95E1F78056BA
:10602000994F90932C0280932B028091220281FD44
:1060300006C09091250280912A02981711F482E0FF
:1060400001C081E080932D0280912D02813011F4F6
:1060500085E801C085EC8093BC0080912902809383
:10606000230210922902DDC0E0912B02F0912C0254
:106070008091BB00808380912B0290912C0201962D
:1060800090932C0280932B0280912D02815080935B
:106090002D02823010F085EC5DC0813011F485E86E
:1060A00059C08091220281FF2DC080913B0280FD6A
:1060B0001DC080912502E82FFF2723E0EE0FFF1F70
:1060C0002A95E1F7E556F94F86818A3F79F4809168
:1060D0002502E82FFF2793E0EE0FFF1F9A95E1F7C7
:1060E000E556F94F8081816080830CC08091250244
:1060F000E82FFF2783E0EE0FFF1F8A95E1F7E556B3
:10610000F94F1082809125028F5F80932502809144
:1061100025028C30A0F01092250210921F021092DE
:106120001E0280912A028F5F80932A028C3038F001
:1061300010922A02809122028D7F80932202109277
:10614000280284E98093BC008091220281608093C0
:10615000220265C08093BC0086E08093280261C063
:1061600088E9BBCD80912702880F805FB6CD8091F2
:10617000270299278130910561F0823091051CF446
:10618000892B21F04EC0029739F04BC08091140149
:10619000A4CD80911301A1CD809112019ECD80E804
:1061A0009CCD1092280284E98093BC0010922402B6
:1061B0008AE090E090933701809336018091270226
:1061C000823088F4809127028F5F8093270282E1DA
:1061D00080932802809122028E7F8093220285EA9A
:1061E0008093BC001EC01092270280912202816021
:1061F0008093220216C01092280284E98093BC008A
:10620000809122028160809322028AE090E0909344
:1062100037018093360110922602109225021092C7
:106220002402FF91EF919F918F915F914F913F9148
:106230002F910F900FBE0F901F9018951F93CF9323
:10624000DF93182F80917202882321F48091B70187
:10625000882319F081E090E097C01D3008F092C0CB
:106260001123B1F0E12FFF2723E0EE0FFF1F2A9546
:10627000E1F7E556F94F35978081359688230CF084
:1062800081C03897808180FD03C083E090E07CC0AE
:1062900080919306823019F084E090E075C067E049
:1062A00070E083E996E00E943D2990919A06891753
:1062B00019F085E090E068C080ED97E00E94CF156E
:1062C000EC018091220280FD05C0CE010E94D8150C
:1062D0008823B9F3112319F48FEF90E00BC0212F1D
:1062E00033272150304081E090E002C0880F991F91
:1062F0002A95E2F79093210280932002A1E0B0E07A
:10630000EBE9F6E040E050E06BE0CD01042E02C086
:10631000880F991F0A94E2F7209120023091210200
:1063200082239323892B11F01182128261504F5FD7
:106330005F4F389667FFE9CF10922602109228022D
:10634000809122028E7F8093220285EA8093BC0096
:106350008091220280FD05C0CE010E94D8158823BD
:10636000B9F38091200290912102892B29F0CE016E
:106370000E94D815882311F3809120029091210268
:10638000009711F082E090E0DF91CF911F91089586
:106390000F931F93CF93DF93982F809172028823DE
:1063A00021F48091B701882319F081E090E092C038
:1063B0009D30A0F4992319F486E090E08BC0C92F9A
:1063C000DD27FE0133E0EE0FFF1F3A95E1F7E556BA
:1063D000F94F35978081359687FD03C082E090E0C4
:1063E00079C03897808180FD03C083E090E072C05F
:1063F00080ED97E00E94CF158C018091220280FDF4
:1064000005C0C8010E94D8158823B9F3219721E05F
:1064100030E0C90102C0880F991FCA95E2F7909336
:106420001F0280931E02D901EBE9F6E040E050E044
:106430006BE0CD01042E02C0880F991F0A94E2F789
:1064400020911E0230911F0282239323892B11F089
:106450001182128261504F5F5F4F389667FFE9CF1C
:10646000109225021092930610929A06109228021A
:10647000809122028E7F8093220285EA8093BC0065
:106480008091220280FD05C0C8010E94D815882392
:10649000B9F380911E0290911F02892B29F0C80147
:1064A0000E94D815882311F380919306823019F049
:1064B00084E090E00FC067E070E083E996E00E941E
:1064C0003D2990919A06891719F085E090E002C065
:1064D00080E090E0DF91CF911F910F910895CF93CD
:1064E000DF9380E021E83FEFC0E3D7E0ECEFF6E098
:1064F000DF01853020F411961C921E9202C0318378
:1065000020831982188222968F5F129632968A31E2
:1065100080F31092E0021092DF021092E2021092D9
:10652000E1021092E4021092E302DF91CF9108950C
:106530001F920F920FB60F9211240F931F932F9358
:106540003F934F935F936F937F938F939F93AF93FB
:10655000BF93CF93DF93EF93FF93409186005091C9
:10656000870080912F0290913002481B590B809137
:106570008600909187009093300280932F02CA0189
:106580008D549440A0913102B0913202835F9A41C0
:1065900078F4809131028093FB06149714F01092E6
:1065A0003A0181E090E09093320280933102B3C0CF
:1065B000AD30B1050CF0AFC0CA018B5F9040845B79
:1065C000914008F085C08091380190913901481BB5
:1065D000590BE0913106EE2351F0FF27EE0FFF1F1C
:1065E000E450F94F8081918184369105ECF4FD01EE
:1065F000EA0FFB1FE450F94F80819181FA01E81BFB
:10660000F90BCF01F7FF03C0909581959F4F069737
:106610005CF480917302883C20F480917302865F61
:1066200001C088EC80937302FD01EA0FFB1FE45068
:10663000F94F808191819C01220F331F280F391F50
:10664000240F351F37FF02C02D5F3F4FE901D5955D
:10665000C795D595C795CA0101968C179D0714F467
:10666000219706C041505040C417D5070CF421961D
:1066700080917302833CD8F08D010A0F1B1FF80133
:10668000E450F94F808191819E01281B390BC9018B
:1066900063E070E00E948277CB01880F991F860F1C
:1066A000971F005D184FF8019183808307C0AA0FE0
:1066B000BB1FA05DB84F11961C921E92E091310253
:1066C000F0913202EE0FFF1FE450F94FD183C083E7
:1066D00020913102309132022F5F3F4F30933202CE
:1066E00020933102809101018431A8F425303105D5
:1066F00011F45D9A01C05D9880913102909132024F
:106700008630910511F45C9A01C05C98079711F4EA
:106710005B9A01C05B98FF91EF91DF91CF91BF91A0
:10672000AF919F918F917F916F915F914F913F9129
:106730002F911F910F910F900FBE0F901F901895E2
:10674000EF92FF920F931F938091E4059927880F92
:10675000991F880F991F7C010027F7FC0095102FC7
:106760008091CD029091CE02A091CF02B091D00243
:10677000BC01CD01A80197010E94B7773093240591
:10678000209323058091C5029091C602A091C70273
:10679000B091C802BC01CD01A80197010E94B77752
:1067A00030932605209325058091BB079091BC0767
:1067B00097FD0396959587959595879590932805D0
:1067C000809327058091CB079091CC0797FD039686
:1067D000959587959595879590932A05809329059A
:1067E0008091DF029091E0022091F8013091F9014F
:1067F000821B930B90932C0580932B0580916D0247
:1068000090916E02A0916F02B0917002BC01CD0117
:106810002AE030E040E050E00E94B77730932E0548
:1068200020932D058091680590916905909330051E
:1068300080932F0580918A0190918B01909334056C
:106840008093330580911F0190912001909336052C
:106850008093350580917302992790933805809332
:106860003705809172079091730790933A05809352
:10687000390580919C06992790933C0580933B05B0
:106880008091A406992790933E0580933D058091C1
:10689000AC0699279093400580933F058091B406FC
:1068A000992790934205809341058091D201909160
:1068B000D30190934C0580934B058091570890919C
:1068C00058089093500580934F0580915B089091F4
:1068D0005C089093520580935105809169029091D4
:1068E0006A02A0916B02B0916C02BC01CD012AE05A
:1068F00030E040E050E00E94B77730935405209399
:10690000530580918B0290918C0290935A0580934D
:10691000590580915D08992790935E0580935D05E8
:1069200080914203909143039093600580935F05AB
:10693000809140039091410390936205809361059B
:1069400080919703882321F480919803882321F074
:1069500080912205816003C0809122058E7F809303
:1069600022051F910F91FF90EF900895EF92FF92F3
:106970001F93CF93DF93182F7B018091720288239E
:1069800091F5809101018C3010F0873111F4299834
:1069900001C0299A11501F3FE9F0F092D901E0920D
:1069A000D801E7018091D8019091D901892B11F488
:1069B000209781F38091DC018823A1F31092DC0100
:1069C0008091D8019091D901892B09F421970E94D7
:1069D000C974E8CF809101018C3010F0873111F437
:1069E000299A01C02998DF91CF911F91FF90EF90D4
:1069F0000895CF93DF93809101018D3011F40E94AF
:106A00009B1A10927A008091FC019091FD01909365
:106A10007E0780937D078091FA019091FB0190930E
:106A20006E0780936D078091F8019091F901909322
:106A3000C1078093C0072091F4013091F501C9018D
:106A4000880F991F880F991F820F931F820F931F22
:106A50009093BC078093BB072091F6013091F7011A
:106A6000C901880F991F880F991F820F931F820FEA
:106A7000931F9093CC078093CB078FEC80937A0081
:106A8000A4E7B2E0CDECD5E097E08991E82FFF27AD
:106A9000EE0FFF1FE450F94F0190F081E02DE15817
:106AA000FF4F1E161F061CF0E0E0F0E005C0EF3FB0
:106AB000F10514F0EFEFF0E08C91282F3327E21767
:106AC000F30714F4815004C02E173F0714F48F5FAE
:106AD0008C939150119697FFD8CF809109069927F2
:106AE000AA27BB27BC01CD0124EC39E040E050E0EF
:106AF0000E944377DC01CB01809382019093830154
:106B0000A0938401B093850180910A069927AA2752
:106B1000BB27BC01CD010E944377DC01CB018093F0
:106B20007E0190937F01A0938001B0938101DF915A
:106B3000CF910895A0E0B0E0E0EAF5E30C94D777B8
:106B4000882E71E0772E00E010E078015801E8010E
:106B5000109297031093DA020093D9021093D8028F
:106B60000093D7021093D4020093D3021092D20262
:106B70001093E4020093E3021093E2020093E10217
:106B80001093E0020093DF021092640110926301FF
:106B90001092ED010E94F93484E690E00E94F11514
:106BA0000E94F9348091D50580FF10C080911501B5
:106BB00090911601875B934038F480911501909174
:106BC00016018E5E924010F40E94401A6FE1C62EAC
:106BD0008AE090E00E94F1158091F8019091F9010E
:106BE000080F191F8091FC019091FD01E80EF91E1C
:106BF0008091FA019091FB01A80EB91E8091680561
:106C000090916905C80FD91FCA94C7FEE1CF9701BB
:106C1000205F3F4F36952795369527953093E402B0
:106C20002093E302C50140969695879596958795A2
:106C30009093E2028093E102005F1F4FB5E016954A
:106C40000795BA95E1F71093E0020093DF02609692
:106C5000A5E0D695C795AA95E1F7D093D402C09345
:106C6000D3029093DE028093DD023093DC02209306
:106C7000DB0282E08816C9F58091BB079091BC07C2
:106C800097FF03C0909581959F4F6CE070E00E9444
:106C900082779B017093DA026093D9028091CB07CF
:106CA0009091CC0797FF03C0909581959F4F6CE022
:106CB00070E00E9482777093D8026093D702B90186
:106CC00084E090E00E94322B6091D7027091D8024C
:106CD00086E090E00E94322B6091D3027091D40242
:106CE00088E090E00E94322B4FC084E090E00E9448
:106CF0002D2B9093DA028093D90286E090E00E94D7
:106D00002D2B9C019093D8028093D7028091D902B9
:106D10009091DA028150984018F421503840A0F147
:106D20008FEA98E09F938F9380EC91E19F938F93EC
:106D3000E0917E03F0917F0309958091BB079091CC
:106D4000BC0797FF03C0909581959F4F6CE070E062
:106D50000E9482777093DA026093D9028091CB0708
:106D60009091CC0797FF03C0909581959F4F6CE061
:106D700070E00E9482777093D8026093D7027724E4
:106D80000F900F900F900F9010927E0710927D073A
:106D900010926E0710926D071092C1071092C007F3
:106DA00084E690E00E94F1158091F4019091F50144
:106DB0009C01220F331F220F331F280F391F280F6A
:106DC000391F3093BC072093BB078091F601909147
:106DD000F7018C01000F111F000F111F080F191F61
:106DE000080F191F1093CC070093CB078091E4057F
:106DF000C82EDD24EE24FF24442737FD4095542F70
:106E0000C701B6010E9443774B015C016093CD023C
:106E10007093CE028093CF029093D00298014427C2
:106E200037FD4095542FC701B6010E944377DC011E
:106E3000CB018093C5029093C602A093C702B09382
:106E4000C8028092AD029092AE02A092AF02B092C0
:106E5000B0028093A5029093A602A093A702B093DC
:106E6000A80210929D0210929E0210929F02109210
:106E7000A0028091170190911801A0911901B09181
:106E80001A0180936A0590936B05A0936C05B093EB
:106E90006D051092EC011092EB011092EE01109230
:106EA000EF011092F0011092F10110928D021092F8
:106EB0008E0210928F021092900200918A0110911E
:106EC0008B0110938C0200938B0284E690E09093E8
:106ED00087018093860182E390E09093D9018093AB
:106EE000D801809109069927AA27BB27BC01CD01AB
:106EF00024EC39E040E050E00E944377DC01CB0114
:106F00008856954CAF4FBF4F809382019093830179
:106F1000A0938401B093850180910A069927AA273E
:106F2000BB27BC01CD010E944377DC01CB01885611
:106F3000954CAF4FBF4F80937E0190937F01A093FC
:106F40008001B09381011092410110924001C8016B
:106F5000AA2797FDA095BA2F20913C0130913D01C1
:106F600040913E0150913F01BC01CD010E94437709
:106F7000DC01CB018093C7079093C807A093C90792
:106F8000B093CA0710928802109287020E94076984
:106F900080913B02846080933B028FEF809347088F
:106FA0001092480880E280934908C4E7D2E0ADEC33
:106FB000B5E077E0C72E8D91E82FFF27EE0FFF1F7A
:106FC000E450F94F8081918181588993CA94C7FE1A
:106FD000F2CF84E6809373028091D601882311F06A
:106FE000579A06C080E091E19093080180930701D1
:106FF00088E090E00E942D2B9093D4028093D302DE
:107000008091E3029091E40280569940815C9B421A
:1070100028F0809197038160809397038091E1022B
:107020009091E20280569940815C9B4228F08091C9
:1070300097038260809397038091DF029091E00232
:107040008C5291408957954028F080919703846035
:10705000809397038091D9029091DA028C529140EB
:10706000835C914028F08091970388608093970318
:107070008091D7029091D8028C529140835C9140CC
:1070800028F0809197038061809397038091D302C9
:107090009091D402805092408355914028F0809185
:1070A00097038062809397038091970381117724DF
:1070B00086E480937901872D9927EDE0CDB7DEB77F
:1070C0000C94F377A3E1B0E0E8E6F8E30C94D27710
:1070D0008091DF029091E0022091F8013091F90156
:1070E000821B930B9093C1078093C007809102028B
:1070F0009091030297FD07969C0153E035952795E3
:107100005A95E1F730937E0720937D078091000226
:107110009091010297FD079643E0959587954A95D2
:10712000E1F790936E0780936D0730938B07209360
:107130008A0790938107809380078091BB07909185
:10714000BC07AC01440F551F480F591F2091F40193
:107150003091F501C901880F991F880F991F820F7F
:10716000931F820F931F480F591F57FF02C04D5F97
:107170005F4F55954795559547955093BC0740935C
:10718000BB078091CB079091CC07AC01440F551FF2
:10719000480F591F2091F6013091F701C901880F5E
:1071A000991F880F991F820F931F820F931F480FFB
:1071B000591F57FF02C04D5F5F4F55954795559535
:1071C00047955093CC074093CB072091F401309121
:1071D000F501C901880F991F880F991F820F931F0E
:1071E000820F931F9C01442737FD4095542F8091B7
:1071F000BD029091BE02A091BF02B091C002820F69
:10720000931FA41FB51F8093BD029093BE02A0934D
:10721000BF02B093C0022091F6013091F701C9017D
:10722000880F991F880F991F820F931F820F931F3A
:107230009C01442737FD4095542F8091B9029091CD
:10724000BA02A091BB02B091BC02820F931FA41F8F
:10725000B51F8093B9029093BA02A093BB02B0937A
:10726000BC0280919407909195072091F401309190
:10727000F501820F931F9093950780939407809157
:10728000C3079091C4072091F6013091F701820F56
:10729000931F9093C4078093C3078091D502909168
:1072A000D60201969093D6028093D502809168050C
:1072B000909169052091D3023091D402821B930BE7
:1072C0009C01442737FD4095542F8091B502909141
:1072D000B602A091B702B091B802820F931FA41F0B
:1072E000B51F8093B5029093B602A093B702B093F6
:1072F000B8028FEC80937A00109211012091A502C0
:107300003091A6024091A7025091A80229873A879E
:107310004B875C8729543B46414050402CF028E481
:107320003BE641E050E00DC089859A85AB85BC8580
:10733000885B9449AE4FBF4F4CF428EB34E94EEFD5
:107340005FEF2D833E834F83588708C089859A85D8
:10735000AB85BC858D839E83AF83B8872091AD02BA
:107360003091AE024091AF025091B0022D873E871E
:107370004F87588B29543B46414050402CF028E41D
:107380003BE641E050E00DC08D859E85AF85B88914
:10739000885B9449AE4FBF4F4CF428EB34E94EEF75
:1073A0005FEF29833A834B835C8308C08D859E857C
:1073B000AF85B88989839A83AB83BC83A091C007CA
:1073C000B091C107BB8BAA8BFD01CF01AA2797FD06
:1073D000A095BA2FA0909D02B0909E02C0909F02EF
:1073E000D090A002A80EB91ECA1EDB1EA0929D025C
:1073F000B0929E02C0929F02D092A002E090C70776
:10740000F090C8070091C9071091CA07E80EF91E4D
:107410000A1F1B1FE092C707F092C8070093C90715
:107420001093CA07F0915602F98BFF2309F098C117
:1074300080915502882309F093C18091B70786FF98
:107440008FC180916D0790916E07AA2797FDA09537
:10745000BA2FBC01CD0129813A814B815C810E9408
:1074600043779B01AC0197FF04C02150384F4F4F29
:107470005F4F6BE055954795379527956A95D1F7FE
:1074800080916301682E772488249924CA01B90168
:10749000A40193010E944377DC01CB018093EF02AA
:1074A0009093F002A093F102B093F202B7FF04C0F0
:1074B0008150904FAF4FBF4F1C012D013CE05594C0
:1074C0004794379427943A95D1F72092EF0230925F
:1074D000F0024092F1025092F20280917D07909169
:1074E0007E07AA2797FDA095BA2FBC01CD012D815B
:1074F0003E814F8158850E94437797FF04C06150B9
:10750000784F8F4F9F4F2BE095958795779567958F
:107510002A95D1F7A40193010E944377DC01CB01A6
:107520008093F3029093F402A093F502B093F602D5
:10753000B7FF04C08150904FAF4FBF4F9C01AD01CA
:107540008CE055954795379527958A95D1F72093E7
:10755000F3023093F4024093F5025093F6028091C7
:10756000EF029091F00290936507809364078091F9
:10757000F3029091F40290936907809368072219AF
:107580003309440955092093F3023093F4024093E0
:10759000F5025093F602E20EF31E041F151FE0924F
:1075A000C707F092C8070093C9071093CA078091D4
:1075B00062018823B1F457FF04C02F5F3F4F4F4F44
:1075C0005F4F5595479537952795A21AB30AC40A78
:1075D000D50AA0929D02B0929E02C0929F02D092C4
:1075E000A0022A893B8979010027F7FC0095102F1A
:1075F0008091F3029091F402A091F502B091F6020D
:10760000E80EF91E0A1F1B1FC801B70129813A8124
:107610004B815C810E9443779B01AC0197FF04C0C2
:107620002150384F4F4F5F4FBBE0559547953795E9
:107630002795BA95D1F780916401A82EBB24CC245C
:10764000DD24CA01B901A60195010E944377DC013E
:10765000CB018093E7029093E802A093E902B093F4
:10766000EA02B7FF04C08150904FAF4FBF4F3C01BB
:107670004D01ACE09594879477946794AA95D1F7DF
:107680006092E7027092E8028092E9029092EA0228
:10769000C801B7012D813E814F8158850E944377F3
:1076A00097FF04C06150784F8F4F9F4FFBE0959537
:1076B000879577956795FA95D1F7A60195010E9470
:1076C0004377DC01CB018093EB029093EC02A09313
:1076D000ED02B093EE02B7FF04C08150904FAF4F60
:1076E000BF4FAC01BD01ECE0759567955795479587
:1076F000EA95D1F74093EB025093EC026093ED02D0
:107700007093EE022A893B8937FF03C0309521959B
:107710003F4F21343105E4F1D401C30197FE07C086
:10772000B095A095909581959F4FAF4FBF4F8138F1
:107730009105A105B10584F4DB01CA0177FF07C0FB
:10774000B095A095909581959F4FAF4FBF4F8138D1
:107750009105A105B105E4F081E08093890218C08C
:1077600010926907109268071092650710926407DB
:107770001092EB021092EC021092ED021092EE02C7
:107780001092E7021092E8021092E9021092EA02C7
:107790008091EB029091EC02A091ED02B091EE028B
:1077A000BC01CD0124E630E040E050E00E94B77714
:1077B000E090E702F090E802E21AF30AF0927C0708
:1077C000E0927B078091E7029091E802A091E902A4
:1077D000B091EA02BC01CD0124E630E040E050E087
:1077E0000E94B777DA01C9012091EB023091EC02D7
:1077F0008C01021B130B1093700700936F0780918D
:107800003C0190913D01A0913E01B0913F01BC012E
:10781000CD0128E631E040E050E00E94437720911E
:10782000C7073091C8074091C9075091CA0726176A
:1078300037074807590764F0261B370B480B590BCD
:107840002093C7073093C8074093C9075093CA07CE
:107850002091C7073091C8074091C9075091CA07C6
:1078600057FF0CC0260F371F481F591F2093C7070B
:107870003093C8074093C9075093CA0760916D07BA
:1078800070916E076E0D7F1D9B01442737FD40955B
:10789000542F8091A1029091A202A091A302B091D5
:1078A000A402820F931FA41FB51F8093A10290937F
:1078B000A202A093A302B093A40280915B029091D4
:1078C0005C02681B790BCB01AA2797FDA095BA2F04
:1078D00029853A854B855C85820F931FA41FB51FB0
:1078E0008093A5029093A602A093A702B093A8024A
:1078F000C0907E01D0907F01E0908001F0908101E6
:10790000C816D906EA06FB06C4F488EA91E6A0E0A8
:10791000B0E08C199D09AE09BF098093A502909330
:10792000A602A093A702B093A8028093A10290930D
:10793000A202A093A302B093A40222273327A90195
:107940002C193D094E095F098091A5029091A6026C
:10795000A091A702B091A80282179307A407B507C8
:10796000B4F4D701C601885A9146A040B040809334
:10797000A5029093A602A093A702B093A8028093B9
:10798000A1029093A202A093A302B093A4026091DB
:107990007D0770917E07600F711F9B01442737FDA3
:1079A0004095542F8091A9029091AA02A091AB0218
:1079B000B091AC02820F931FA41FB51F8093A90240
:1079C0009093AA02A093AB02B093AC0280915902AB
:1079D00090915A02681B790BCB01AA2797FDA095BD
:1079E000BA2F2D853E854F855889820F931FA41F7E
:1079F000B51F8093AD029093AE02A093AF02B093F7
:107A0000B002E0908201F090830100918401109116
:107A10008501E816F9060A071B07C4F488EA91E60F
:107A2000A0E0B0E08E199F09A00BB10B8093AD02CE
:107A30009093AE02A093AF02B093B0028093A902DC
:107A40009093AA02A093AB02B093AC0222273327F3
:107A5000A9012E193F09400B510B8091AD02909165
:107A6000AE02A091AF02B091B00282179307A407B3
:107A7000B507B4F4D801C701885A9146A040B04078
:107A80008093AD029093AE02A093AF02B093B00288
:107A90008093A9029093AA02A093AB02B093AC0288
:107AA00080919D0290919E02A0919F02B091A002B0
:107AB0008093B1029093B202A093B302B093B40248
:107AC0008091AD029091AE02A091AF02B091B00250
:107AD0008093CD029093CE02A093CF02B093D002B8
:107AE0008091A5029091A602A091A702B091A80250
:107AF0008093C5029093C602A093C702B093C802B8
:107B00008091A9029091AA02A091AB02B091AC021F
:107B10008093C9029093CA02A093CB02B093CC0287
:107B20008091A1029091A202A091A302B091A4021F
:107B30008093C1029093C202A093C302B093C40287
:107B400080911D0190911E0197FD079633E0959558
:107B500087953A95E1F790937E0780937D07809112
:107B60001B0190911C0197FD079623E09595879541
:107B70002A95E1F790936E0780936D078091FC0141
:107B80009091FD010F9734F488E19CEF90937E076C
:107B900080937D078091FC019091FD01079734F45B
:107BA00080E398EF90937E0780937D0720910101F9
:107BB0002A30A9F48091FC019091FD01835F9340EC
:107BC00034F088EE93E090937E0780937D07809158
:107BD000FC019091FD018A5F9340DCF014C080911C
:107BE000FC019091FD01815D974034F088EE93E0B7
:107BF00090937E0780937D078091FC019091FD0119
:107C0000805E974034F080ED97E090937E078093FC
:107C10007D078091FA019091FB010F9734F488E180
:107C20009CEF90936E0780936D078091FA0190917D
:107C3000FB01079734F480E398EF90936E078093ED
:107C40006D072A30A9F48091FA019091FB01835FBE
:107C5000934034F088EE93E090936E0780936D0725
:107C60008091FA019091FB018A5F9340DCF014C08F
:107C70008091FA019091FB01815D974034F088EE8C
:107C800093E090936E0780936D078091FA01909135
:107C9000FB01805E974034F080ED97E090936E0793
:107CA00080936D0760917001662309F4AFC0409125
:107CB0001D0150911E018091F7029091F802481B1E
:107CC000590B5093FE024093FD0220911D0130910B
:107CD0001E01280F391F37FF02C02F5F3F4F359518
:107CE00027953093F8022093F702413851051CF094
:107CF00080E890E005C040585F4F34F480E89FEF83
:107D00009093FE028093FD0240911B0150911C0153
:107D10008091F9029091FA02481B590B5093FC0292
:107D20004093FB0220911B0130911C01280F391F49
:107D300037FF02C02F5F3F4F359527953093FA02EA
:107D40002093F902413851051CF080E890E005C00D
:107D500040585F4F34F480E89FEF9093FC0280938B
:107D6000FB02462F55278091FD029091FE02849FD1
:107D7000B001859F700D949F700D11249B0177FFBA
:107D800002C0215F3F4F04E0359527950A95E1F742
:107D900080917D0790917E07820F931F90937E07BD
:107DA00080937D078091FB029091FC02849FD0011B
:107DB000859FB00D949FB00D1124AD019D01B7FFBB
:107DC00002C0215F3F4F14E0359527951A95E1F7E2
:107DD00080916D0790916E07820F931F90936E07AD
:107DE00080936D0780911D0190911E01860F971F52
:107DF00090931E0180931D0180911B0190911C01A5
:107E0000840F951F90931C0180931B0100918007A4
:107E100010918107809164079091650710161106F3
:107E20005CF59C0197FF04C022273327281B390BE0
:107E3000C901AA2797FDA095BA2F20916201332787
:107E400044275527BC01CD010E9443779B01AC011B
:107E500097FF04C0215C3F4F4F4F5F4FB6E05595F1
:107E6000479537952795BA95D1F780917B079091E3
:107E70007C07820F931F27C097FF03C090958195C1
:107E80009F4FAA2797FDA095BA2F20916201332713
:107E900044275527BC01CD010E9443779B01AC01CB
:107EA00097FF04C0215C3F4F4F4F5F4FA6E05595B1
:107EB000479537952795AA95D1F780917B079091A3
:107EC0007C07821B930B90937C0780937B07E09049
:107ED0008A07F0908B0780916807909169071E14BC
:107EE0001F045CF59C0197FF04C022273327281B41
:107EF000390BC901AA2797FDA095BA2F20916201DD
:107F0000332744275527BC01CD010E9443779B01AD
:107F1000AC0197FF04C0215C3F4F4F4F5F4FF6E02D
:107F20005595479537952795FA95D1F780916F0725
:107F300090917007820F931F27C097FF03C0909501
:107F400081959F4FAA2797FDA095BA2F2091620196
:107F5000332744275527BC01CD010E9443779B015D
:107F6000AC0197FF04C0215C3F4F4F4F5F4FE6E0ED
:107F70005595479537952795EA95D1F780916F07E5
:107F800090917007821B930B9093700780936F07FB
:107F90008091B70787FF44C0B989BB2309F040C06F
:107FA000809155028823E1F5E1E0EE16E1E0FE065E
:107FB0004CF080917D0790917E078E0D9F1D805023
:107FC00091400DC0F0E0EF16FFEFFF0664F48091E2
:107FD0007D0790917E078E0D9F1D80509F4F90933F
:107FE0007E0780937D0721E0013012074CF08091DD
:107FF0006D0790916E07800F911F805091400CC0CB
:108000003FEF0030130764F480916D0790916E0785
:10801000800F911F80509F4F90936E0780936D0744
:10802000E2E1CD5E0C94EE7780917202882329F50F
:1080300080913B028C7F80933B0280913A028F7D3E
:1080400080933A02ACE9B3E0EBE9F6E09BE0809183
:10805000B701882309F48C938D918183128291500A
:10806000389697FFF4CF8091B701882359F080911B
:10807000B70181508093B70105C080913B028160B8
:1080800080933B0280912402882319F010922402ED
:1080900008958093260280932802809122028E7F89
:1080A0008093220285EA8093BC000895CF93DF93EA
:1080B000A4E7B2E0CDECD5E057E09991E92FFF2796
:1080C000EE0FFF1FE450F94F0190F081E02DE158D1
:1080D000FF4FEF3FF10521F01CF0EFEFF0E004C09F
:1080E000F7FF02C0E0E0F0E0993111F4EC931BC01F
:1080F0004C91242F3327E217F307A9F0CF01821BFD
:10810000930B97FD03969595879595958795242FC5
:10811000280F2C93822F9927E817F90714F4215080
:1081200001C02F5F2C935150119657FFC6CF8091FD
:10813000D705883F38F0EFEFF0E0E81BF109EC5885
:10814000FD4F80818093760180917601882329F00C
:10815000843618F084E6809376018091D905883FB3
:1081600038F0EFEFF0E0E81BF109EC58FD4F8081AB
:108170008093740180917401882329F0843618F06B
:1081800084E6809374018091E605883F38F0EFEF34
:10819000F0E0E81BF109EC58FD4F808180936F01FE
:1081A00080916F018B3010F48AE002C08F3F11F490
:1081B00080936F0180911306883F38F0EFEFF0E075
:1081C000E81BF109EC58FD4F808180939607809160
:1081D0009607863010F485E002C08F3F11F480933B
:1081E000960780911506883F38F0EFEFF0E0E81B26
:1081F000F109EC58FD4F80818093BE078091BE0746
:10820000863010F485E002C08F3F11F48093BE07E2
:1082100080910006873F19F4429905C006C0863F49
:1082200031F4439B02C08CE80BC086E409C0883F50
:1082300038F0EFEFF0E0E81BF109EC58FD4F8081DA
:108240008093930780910106873F19F4429905C0F6
:1082500006C0863F31F4439B02C08CE80BC086E425
:1082600009C0883F38F0EFEFF0E0E81BF109EC5867
:10827000FD4F808180936A0780910206883F38F025
:10828000EFEFF0E0E81BF109EC58FD4F808180939F
:108290009C078091D805883F38F0EFEFF0E0E81BAD
:1082A000F109EC58FD4F8081809375018091DB05C9
:1082B000883F38F0EFEFF0E0E81BF109EC58FD4F94
:1082C0008081809373018091DD05883F38F0EFEF66
:1082D000F0E0E81BF109EC58FD4F808180937101BB
:1082E0008091E505883F38F0EFEFF0E0E81BF109F9
:1082F000EC58FD4F8081809372018091E705883FA3
:1083000038F0EFEFF0E0E81BF109EC58FD4F808109
:1083100080936E018091E805883F38F0EFEFF0E040
:10832000E81BF109EC58FD4F80818093700180912A
:10833000E905883F38F0EFEFF0E0E81BF109EC5871
:10834000FD4F808180936D018091EA05883F38F070
:10835000EFEFF0E0E81BF109EC58FD4F80818093CE
:108360006C018091F005883F38F0EFEFF0E0E81BFA
:10837000F109EC58FD4F808180936A018091F105ED
:10838000883F38F0EFEFF0E0E81BF109EC58FD4FC3
:108390008081809350028091F205883F38F0EFEFA2
:1083A000F0E0E81BF109EC58FD4F808180934F020B
:1083B0008091F305883F38F0EFEFF0E0E81BF1091A
:1083C000EC58FD4F808180934E028091F405883FE8
:1083D00038F0EFEFF0E0E81BF109EC58FD4F808139
:1083E00080934D0280910E06883F38F0EFEFF0E069
:1083F000E81BF109EC58FD4F808180934C0280917D
:108400000F06883F38F0EFEFF0E0E81BF109EC5879
:10841000FD4F808180934B0280911006883F38F099
:10842000EFEFF0E0E81BF109EC58FD4F80818093FD
:108430004A0280911106883F38F0EFEFF0E0E81B28
:10844000F109EC58FD4F8081809349028091F50538
:10845000883F38F0EFEFF0E0E81BF109EC58FD4FF2
:108460008081809369018091F905883F38F0EFEFB2
:10847000F0E0E81BF109EC58FD4F80818093680122
:108480008091F605883F38F0EFEFF0E0E81BF10946
:10849000EC58FD4F8081809367018091FA05883FF9
:1084A00038F0EFEFF0E0E81BF109EC58FD4F808168
:1084B0008093660180910306883F38F0EFEFF0E08B
:1084C000E81BF109EC58FD4F808180936501809194
:1084D0000606883F38F0EFEFF0E0E81BF109EC58B2
:1084E000FD4F80818093640180910706883F38F0BA
:1084F000EFEFF0E0E81BF109EC58FD4F808180932D
:10850000630180910806883F38F0EFEFF0E0E81B48
:10851000F109EC58FD4F8081809362018091300613
:10852000883F38F0EFEFF0E0E81BF109EC58FD4F21
:1085300080818093790790914C03992321F0809159
:108540007907981720F080917907882311F4909388
:1085500079078091D5058093B7078091360680937F
:108560009B0780910D06883F38F0EFEFF0E0E81BA5
:10857000F109EC58FD4F80818093610180912906BB
:10858000883F38F0EFEFF0E0E81BF109EC58FD4FC1
:1085900080818093CE0780916A01282F33272F5F37
:1085A0003F4F8CE398E2B9010E9482777093780183
:1085B000609377018091E3058093BF078091E20586
:1085C0008093820790912B069333E0F181E08093B2
:1085D0004802983F58F0EFEFF0E0E91BF109EC5842
:1085E000FD4F8081823310F410924802809179010E
:1085F000209148028217B1F0833088F4222319F0C9
:108600008CED95E002C088EC90E09093D9018093C6
:10861000D80185E080935D022093790103C08150E9
:108620008093790180910E0890910F0897FF0FC0F9
:1086300080914802882359F0809197038068809345
:10864000970305C0109248028AE0809379018091D7
:108650000E0890910F0897FF1DC080917202882329
:10866000C9F0809148028823A9F080910901909176
:108670000A018F5F9F4F71F488E99AE39093D901C3
:108680008093D80180E094EA90930A0180930901D5
:108690001092480280914802882369F080913A0242
:1086A000816080933A0280916401823D48F4825E49
:1086B0008093640105C080913A028E7F80933A02D4
:1086C000DF91CF910895A7E1B0E0E9E6F3E40C94DF
:1086D000D2770E94623880913B0299278471907012
:1086E000892B91F58091370682FF27C08091570230
:1086F000909158020097F1F002E088359007D4F489
:108700009C0197FF02C02D5F3F4F3595279535950A
:1087100027958091ED059927289FA001299F500D4D
:10872000389F500D1124CA0164E670E00E948277E0
:10873000CB0106C08DE290E003C08091ED05992742
:10874000909339028093380220913602309137029B
:1087500055E72033350759F410927E0210927D02BE
:108760008091820799279093390280933802609113
:108770007D0270917E027A836983809182079927B6
:108780000A966817790714F49A8389838091730293
:10879000843608F06AC080913A0282FD66C08091FA
:1087A000130390911403009731F0019790931403F1
:1087B000809313030BC01092720290933D0280933A
:1087C0003C0280913B028D7E80933B0280910101AF
:1087D0008A3011F0843110F0289A01C028988091D5
:1087E0003C0290913D02895E9340E0F180915D08EA
:1087F0008536C0F180913802909139029A8389833D
:1088000080913B02806180933B028091C905A82F33
:10881000BB27AA0FBB1FFD01E05DF84F118210823C
:108820008091CA05282F3327220F331FC901805D8D
:10883000984FFC0111821082A450B94F11961C92DE
:108840001E922450394FD90111961C921E9280918C
:10885000CC05E82FFF27EE0FFF1FE450F94F1182E0
:1088600010829FC3109272029CC3809173028D3854
:1088700008F46DC380913B028F7E80933B02909100
:10888000EE0582E3989FC001112490931403809316
:108890001303E981FA81B9978CF0809172028823E1
:1088A00069F080913C0290913D02FFEF8F3F9F075E
:1088B00029F0019690933D0280933C0220913C0266
:1088C00030913D022F3F310509F030F510929502AD
:1088D00010929602109297021092980210929102B2
:1088E0001092920210929302109294021092FF0240
:1088F00010920003109201031092020310929D0245
:1089000010929E0210929F021092A00280913A0251
:10891000806280933A0244C080913B0282608093DF
:108920003B0280913A0285FF3BC080916D0290919D
:108930006E02A0916F02B0917002825A9E4FAF4FAB
:10894000BF4F855F9140A040B04020F48091B707B1
:1089500080FD05C080913A028F7D80933A0210928B
:10896000950210929602109297021092980210921D
:10897000910210929202109293021092940210921D
:108980009D0210929E0210929F021092A002295EF8
:10899000334030F088EE93E090933D0280933C02A8
:1089A0008091CB05E82FFF27EE0FFF1FE450F94F12
:1089B00080819181813591050CF434C1209172023E
:1089C000222309F02FC18091CC05E82FFF27EE0F5D
:1089D000FF1FE450F94F808191818C3491050CF494
:1089E000FFC0809115038F5F80931503893C08F4C5
:1089F00019C12093150310923D0210923C02309150
:108A0000C905E32FFF27EE0FFF1FE450F94F8081C8
:108A1000918187349105B4F48091CA05E82FFF272E
:108A2000EE0FFF1FE450F94F808191810190F0819A
:108A3000E02DF7FF03C0F095E195FF4FE734F10516
:108A40000CF478C041E02091CA05A22FBB27AA0FE1
:108A5000BB1FA450B94F8D919C91119787349105FC
:108A600044F0E32FFF27EE0FFF1FE450F94F808102
:108A700091818D919C918734910574F08091C90505
:108A8000E82FFF27EE0FFF1FE450F94F80819181FF
:108A9000873491050CF042E0E22FFF27EE0FFF1F15
:108AA000E450F94F808191818634910574F480916E
:108AB000C905E82FFF27EE0FFF1FE450F94F808113
:108AC0009181873491050CF043E0E22FFF27EE0FF0
:108AD000FF1FE450F94F808191818A5B9F4F74F4AE
:108AE0008091C905E82FFF27EE0FFF1FE450F94FD3
:108AF00080819181873491050CF044E0E22FFF27BB
:108B0000EE0FFF1FE450F94F808191818A5B9F4FE8
:108B100074F48091C905E82FFF27EE0FFF1FE45082
:108B2000F94F80819181863491050CF445E0842FC2
:108B30000E948A2B8091CA05E82FFF27EE0FFF1FA6
:108B4000E450F94F808191810190F081E02DF7FF91
:108B500003C0F095E195FF4F7E97CCF48091C90555
:108B6000E82FFF27EE0FFF1FE450F94F808191811E
:108B70008A5B9F4F64F481E08093B20310925E029F
:108B800088EE93E09093D9018093D8014BC00E9466
:108B9000912C0E94372B80E00E94DE058091EF052A
:108BA0000E944F738091B70780FF10C0809115011C
:108BB00090911601875B934038F480911501909154
:108BC00016018E5E924010F40E94401A81E00E94CD
:108BD0009A3580935E0281E08093D601579A19C03E
:108BE00080819181855B9F4FDCF4809115038F5FBD
:108BF00080931503893CB0F02093720220931503F3
:108C000010923D0210923C0282E00E949A358093BD
:108C10005E020E94912C68E770E00E94B63402C0A8
:108C2000209315038091CB05E82FFF27EE0FFF1F40
:108C3000E450F94F808191818B5A9F4F0CF080C195
:108C400020912C06E22FFF27EF77F070EE0FFF1F29
:108C5000E05DF84F80819181069714F084E606C0AC
:108C6000808191818B5F9F4F1CF48CE98093180366
:108C700080917202E091CC05882309F00FC1FF2793
:108C8000EE0FFF1FE450F94F80819181855B9F4F6C
:108C90009CF48091370683FD0BC0E22FFF27EE0F77
:108CA000FF1FE450F94F80819181855B9F4FDCF07D
:108CB00080912C068823B9F08091370683FFEBC0A2
:108CC00080912C06E82FFF27EE0FFF1FE450F94F8D
:108CD00080819181875F9F4F0CF4DDC080911803E4
:108CE000843609F0D8C020915E02222329F08091B9
:108CF0003B02886080933B0280911701909118019C
:108D0000A0911901B0911A0180936A0590936B05A7
:108D1000A0936C05B0936D051092E5011092E601E9
:108D20001092E7011092E80110926D0210926E020B
:108D300010926F02109270021092EE011092EF01E9
:108D40001092F0011092F101809116038F5F8093D1
:108D500016038E3F08F4E6C0109216038091970325
:108D6000882309F091C0222309F48EC08091510319
:108D7000882309F089C081E090E090933D028093C0
:108D80003C0281E0809372021092FF021092000375
:108D9000109201031092020310929D0210929E0203
:108DA00010929F021092A0021092990210929A02C1
:108DB00010929B0210929C028091E405E82EFF2401
:108DC000002711278091BB079091BC079C01442785
:108DD00037FD4095542FC801B7010E944377DC014D
:108DE000CB018093AD029093AE02A093AF02B093FB
:108DF000B0028091CB079091CC079C01442737FDAE
:108E00004095542FC801B7010E944377DC01CB0184
:108E10008093A5029093A602A093A702B093A80204
:108E20008091CD029091CE02A091CF02B091D0025C
:108E30008093A9029093AA02A093AB02B093AC02D4
:108E40008091C5029091C602A091C702B091C8025C
:108E50008093A1029093A202A093A302B093A402D4
:108E60001092950210929602109297021092980218
:108E70001092910210929202109293021092940218
:108E800084E680935D024EC08CED95E09093D9010D
:108E90008093D80147C01092160344C0FF27EE0FFD
:108EA000FF1FE450F94F808191818C3491059CF033
:108EB0008091370683FD0BC0E22FFF27EE0FFF1FC7
:108EC000E450F94F80819181855B9F4FCCF0809178
:108ED0002C068823A9F08091370683FF21C080915A
:108EE0002C06E82FFF27EE0FFF1FE450F94F80817B
:108EF00091818E5C9F4FA4F4809118038C3981F48A
:108F0000809117038F5F809317038B3F58F0109267
:108F100072021092170310923D0210923C0202C09E
:108F200010921703809136029091370253E0883EE9
:108F30009507B8F50196909337028093360231C0B9
:108F40001092180310923702109236022AC02E5E39
:108F5000324038F18091D6079091D70780599140DF
:108F600000F580916D0290916E02A0916F02B09118
:108F700070028C5D9540A040B0409CF480E395E782
:108F8000909337028093360280913C0290913D028B
:108F90008A5E934030F089EE93E090933D02809397
:108FA0003C0280913A01815080933A0180913A01CC
:108FB0008F3F21F080913B0284FFA9C30E9456405D
:108FC000B090DF0580912103909122039C01220F34
:108FD000331F280F391FC090C905AC2DBB27AA0F1E
:108FE000BB1FFD01E450F94F4B2D55278081918126
:108FF000849F7001859FF00C949FF00C11242E0D1E
:109000003F1D37FF02C02D5F3F4FB9017595679532
:1090100075956795A05DB84F8091E005082F1127E1
:109020008D919C91809F9001819F300D909F300D7C
:109030001124620F731F70932203609321038091A8
:109040002303909124039C01220F331F280F391F03
:10905000D090CA05AD2DBB27AA0FBB1FFD01E45060
:10906000F94F80819181849FF001859FF00D949F3D
:10907000F00D11242E0F3F1F37FF02C02D5F3F4F11
:10908000A9015595479555954795A05DB84F8D9188
:109090009C91809F7001819FF00C909FF00C112497
:1090A0004E0D5F1D5093240340932303809148028B
:1090B000882309F448C0CB0177FD0396DC01B59500
:1090C000A795B595A795CA0157FD0396FC01F5959F
:1090D000E795F595E79580919A01682F772767FDC9
:1090E00070956A9F90016B9F300D7A9F300D11240F
:1090F00080915303482F552747FD50954E9FC0013F
:109100004F9F900D5E9F900D1124280F391F37FF40
:1091100002C0295F3F4F93E0359527959A95E1F777
:1091200030938402209383026E9F90016F9F300DD5
:109130007E9F300D11244A9FC0014B9F900D5A9F76
:10914000900D11243FC080912A06E82FFF27EE5B87
:10915000FE4F868180939A01908190935303A82FAC
:10916000BB27A7FDB095A69F9001A79F300DB69F86
:10917000300D1124E92FFF27E7FDF095E49FC00192
:10918000E59F900DF49F900D1124280F391F37FF94
:1091900002C0295F3F4F83E0359527958A95E1F717
:1091A0003093840220938302A49F9001A59F300DE9
:1091B000B49F300D1124E69FC001E79F900DF69FEC
:1091C000900D1124281B390B37FF02C0295F3F4F38
:1091D00003E0359527950A95E1F7309382022093B5
:1091E00081028091CC05E82FFF27EE0FFF1FE4508E
:1091F000F94F80819181909581959F4F9093800246
:1092000080937F028530910514F0049705C00FEF1D
:109210008C3F900734F404969093800280937F02F1
:1092200004C01092800210927F0280913F03882335
:1092300009F43EC0282F3327809183029091840245
:1092400097FD079613E0959587951A95E1F7289F66
:10925000A001299F500D389F500D1124CA0157FDC0
:109260000F96B4E095958795BA95E1F790938402AF
:1092700080938302809181029091820297FD0796EC
:10928000A3E095958795AA95E1F7289FB001299FBE
:10929000700D389F700D1124CB0177FD0F96F4E00F
:1092A00095958795FA95E1F79093820280938102D4
:1092B00080908302909084028091420390914303B6
:1092C000881A990A90928402809283020091810206
:1092D000109182028091400390914103081B190B69
:1092E00010938202009381028091CB05E82FFF2723
:1092F000EE0FFF1FE450F94FE080F1808FE790E020
:10930000E80EF91EF0927E02E0927D0280916F01DC
:109310009927AA2797FDA095BA2FBC01CD010E94DD
:10932000B776DC01CB0120E030E040E251E4BC0143
:10933000CD010E942576DC01CB01BC01CD010E944C
:109340008976DC01CB018093C50780916E01809303
:109350009D0780916D019927AA2797FDA095BA2FA7
:10936000BC01CD010E94B776DC01CB0120E030E0EA
:1093700040E251E4BC01CD010E942576DC01CB0125
:10938000BC01CD010E948976DC01CB01809374077A
:1093900080916C0180938C078091BE0380FF59C03F
:1093A0008091CE07813808F454C08091B703992783
:1093B00087FD90952B2D3327829FD001839FB00D81
:1093C000929FB00D11248A0E9B1E9092840280926F
:1093D00083028091B803992787FD9095829FF001C1
:1093E000839FF00D929FF00D11240E0F1F1F1093FD
:1093F0008202009381028091B903282F332727FD31
:10940000309580917F0290918002820F931F9093FC
:10941000800280937F028091BB03282F332727FD92
:1094200030958091DA059927289F8001299F100D9A
:10943000389F100D11241093410100934001809139
:10944000BA0399278E159F0524F490937E0280938A
:109450007D0280917D0290917E0297FF04C0109260
:109460007E0210927D028091B70782FF02C01092A7
:109470009D074091830250918402CA0157FD0396D3
:109480009C01359527953595279537FF03C0309575
:1094900021953F4F8091400290914102821793079E
:1094A000B4F4CA0157FF03C0909581959F4F97FD73
:1094B000039695958795959587959093410280930E
:1094C00040028536910544F084E690E001C00197A2
:1094D0009093410280934002409181025091820218
:1094E000CA0157FD03969C0135952795359527951B
:1094F00037FF03C0309521953F4F80913E029091F8
:109500003F0282179307B4F4CA0157FF03C0909536
:1095100081959F4F97FD039695958795959587958E
:1095200090933F0280933E028536910544F084E695
:1095300090E001C0019790933F0280933E0280919A
:109540003B0284FF08C01092410210924002109228
:109550003F0210923E02ED2DFF27EE0FFF1FE45059
:10956000F94F40910406242F3327808191812817D9
:10957000390744F48091340682FF04C081E080936F
:10958000540213C0ED2DFF27EE0FFF1FE450F94FDB
:10959000842F992720910506821B91092081318112
:1095A0002817390714F4109254024091CA05E42F89
:1095B000FF27EE0FFF1FE450F94F50910406852F4F
:1095C000992722273327281B390B80819181821705
:1095D000930744F48091340683FF04C081E08093B4
:1095E000530216C080915302882391F0E42FFF2785
:1095F000EE0FFF1FE450F94F809105069927851B58
:109600009109208131818217930714F4109253023B
:10961000EC2DFF27EE0FFF1FE450F94F4091040699
:10962000242F3327808191812817390744F48091B2
:10963000340680FF04C081E08093510217C08091FE
:109640005102882399F0EC2DFF27EE0FFF1FE45005
:10965000F94F842F992720910506821B91092081BB
:1096600031812817390714F4109251024091C9052D
:10967000E42FFF27EE0FFF1FE450F94F509104062F
:10968000852F992722273327281B390B8081918129
:109690008217930744F48091340681FF04C081E06F
:1096A0008093520216C080915202882391F0E42FD9
:1096B000FF27EE0FFF1FE450F94F80910506992711
:1096C000851B9109208131818217930714F4109230
:1096D000520280915402882319F48091530281111F
:1096E00081E08093550280915102882321F480917A
:1096F0005202882351F081E0809356021092550265
:10970000109254021092530202C08093560280912C
:109710005502882321F480915602882369F08091B4
:109720000306992729813A818217930714F49A83B3
:10973000898381E08093890280913A0299279C0174
:109740002470307082FF2DC08091420390914303BA
:10975000909581959F4F909384028093830280918E
:10976000400390914103909581959F4F9093820281
:109770008093810280917C0190917D0190937E0283
:1097800080937D028091B7078B778B668093B707B4
:1097900080919B078C7B80939B0788EC809375015D
:1097A0001EC080913B0284FF1AC030938002209338
:1097B0007F023093840220938302309382022093AD
:1097C00081029AE59093C50788E780939D0790935F
:1097D000740780938C071092550210925602809164
:1097E0008F0790919007A0919107B09192072091D7
:1097F000CD023091CE024091CF025091D002820F23
:10980000931FA41FB51F80938F0790939007A09379
:109810009107B09392078091970790919807A09134
:109820009907B0919A07E090C502F090C6020091A6
:10983000C7021091C802EB82FC820D831E838E0D3D
:109840009F1DA01FB11F8093970790939807A09327
:109850009907B0939A078091840790918507A0910A
:109860008607B0918707E090C902F090CA02009184
:10987000CB021091CC02EF82F88609871A878E0DF1
:109880009F1DA01FB11F8093840790938507A0930D
:109890008607B09387078091750790917607A0910E
:1098A0007707B0917807E090C102F090C202009172
:1098B000C3021091C402EB86FC860D871E878E0DB5
:1098C0009F1DA01FB11F8093750790937607A093EB
:1098D0007707B0937807F0905602FF86FF2029F4AF
:1098E00080915502882309F460C01092BD02109245
:1098F000BE021092BF021092C0021092B9021092E2
:10990000BA021092BB021092BC0210928F07109202
:109910009007109291071092920710929707109259
:1099200098071092990710929A0710928407109244
:10993000850710928607109287071092750710927C
:10994000760710927707109278078091AD02909178
:10995000AE02A091AF02B091B0028093A9029093A1
:10996000AA02A093AB02B093AC028091A5029091A1
:10997000A602A091A702B091A8028093A1029093A1
:10998000A202A093A302B093A4021092EA01109243
:10999000E90110925A021092590210925C02109240
:1099A0005B020F85002309F0D0C180915502882306
:1099B00009F0CBC180916805909169058150924072
:1099C0002CF480917202882309F4BFC1909047085B
:1099D000A090E4052090BB073090BC074090CB07D7
:1099E0005090CC0719140CF0BBC0BB24CC24DD2450
:1099F000CA01B901A60195010E94B77779018A01D0
:109A00008091100890911108281A390AC101AA27DB
:109A100097FDA095BA2FE81AF90A0A0B1B0B6B8168
:109A20007C818D819E81A60195010E94B7775901A5
:109A30006A018091120890911308481A590AC201CC
:109A4000AA2797FDA095BA2FA81AB90ACA0ADB0A55
:109A5000292C332427FC3094432C532CC801B70104
:109A6000A20191010E94437797FF04C061507E4F8D
:109A70008F4F9F4F3B014C0109E095948794779459
:109A800067940A95D1F7C601B501A20191010E9420
:109A9000437797FF04C061507E4F8F4F9F4F5B010C
:109AA0006C0119E0D594C794B794A7941A95D1F78F
:109AB0008091400290914102813491053CF4809163
:109AC0003E0290913F0281349105D4F0D401C3014C
:109AD00097FE03C00196A11DB11D3C014D01959457
:109AE000879477946794D601C501D7FE03C0019689
:109AF000A11DB11D5C016D01D594C794B794A794C5
:109B000080914908282F332727FD3095432F532F65
:109B1000261537054805590514F439014A019927D6
:109B200087FD9095909581959F4FAA2797FDA095C9
:109B3000BA2F681679068A069B0614F43C014D017B
:109B40002A153B054C055D0514F459016A01A81658
:109B5000B906CA06DB060CF0D0C05C016D01CDC0B1
:109B6000EA2CFF2400271127CA01B901A801970197
:109B70000E94B77739014A01C101AA2797FDA09534
:109B8000BA2F681A790A8A0A9B0A6B817C818D81B7
:109B90009E81A80197010E94B77759016A01C2010D
:109BA000AA2797FDA095BA2FA81AB90ACA0ADB0AF4
:109BB000D401C30197FE03C00F96A11DB11D3C0146
:109BC0004D01F4E09594879477946794FA95D1F7D2
:109BD000D601C501D7FE03C00F96A11DB11D5C01C2
:109BE0006D01E4E0D594C794B794A794EA95D1F7B2
:109BF0008091400290914102813491053CF4809122
:109C00003E0290913F0281349105A4F0C401B3015A
:109C100023E030E040E050E00E94B77739014A018C
:109C2000C601B50123E030E040E050E00E94B77784
:109C300059016A018091CC05E82FFF27EE0FFF1F25
:109C4000E450F94F808191810190F081E02DF7FF80
:109C500003C0F095E195FF4F7A97A4F0C401B301DA
:109C600023E030E040E050E00E94B77739014A013C
:109C7000C601B50123E030E040E050E00E94B77734
:109C800059016A0189E18093880121E26216710419
:109C9000810491042CF070E2672E712C812C912CA0
:109CA00030EE63163FEF73063FEF83063FEF9306F8
:109CB00044F460EE662E6FEF762E6FEF862E6FEF18
:109CC000962E41E2A416B104C104D1042CF050E256
:109CD000A52EB12CC12CD12C50EEA5165FEFB506E8
:109CE0005FEFC5065FEFD50644F440EEA42E4FEFBC
:109CF000B42E4FEFC42E4FEFD42E8091AD02909131
:109D0000AE02A091AF02B091B00286199709A809DE
:109D1000B9098093AD029093AE02A093AF02B093C5
:109D2000B0028091A5029091A602A091A702B091E5
:109D3000A8028A199B09AC09BD098093A5029093DA
:109D4000A602A093A702B093A8028091E901909186
:109D5000EA018F3F910509F008F4C4C56F856623B9
:109D600009F04EC580915502882309F049C58091BC
:109D70008902882309F044C570910C06788B7723FB
:109D800009F43EC580918F0790919007A0919107AB
:109D9000B0919207B7FF04C081509F4FAF4FBF4FA4
:109DA000E92EFA2E0B2F112707FD1A95E0928F0747
:109DB000F092900700939107109392078091970774
:109DC00090919807A0919907B0919A07B7FF04C0A6
:109DD00081509F4FAF4FBF4F892F9A2FAB2FBB277B
:109DE000A7FDBA95898B9A8BAB8BBC8B8093970719
:109DF00090939807A0939907B0939A078091E405F0
:109E0000A82EBB24CC24DD242091BD023091BE02BB
:109E10004091BF025091C002C601B5010E94437734
:109E200097FF04C061507F4F8F4F9F4F672E782E52
:109E3000892E992487FC9A946092BD027092BE028A
:109E40008092BF029092C0022091B9023091BA0272
:109E50004091BB025091BC02C601B5010E944377FC
:109E600097FF04C061507F4F8F4F9F4F272E382E92
:109E7000492E552447FC5A942092B9023092BA02D6
:109E80004092BB025092BC028091B5029091B60202
:109E9000A091B702B091B802B7FF04C081509F4FA4
:109EA000AF4FBF4F892F9A2FAB2FBB27A7FDBA9576
:109EB0008093B5029093B602A093B702B093B80214
:109EC000D801C70186199709A809B90980930B031E
:109ED00090930C03A0930D03B0930E0320910B06F7
:109EE000E22EFF2400271127BC01CD01A801970114
:109EF0000E94B77759016A012093190330931A031E
:109F000040931B0350931C0389899A89AB89BC89B0
:109F100082199309A409B50980930F039093100344
:109F2000A0931103B0931203BC01CD01A8019701C6
:109F30000E94B77720931D0330931E0340931F03A5
:109F400050932003D601C501D7FE04C081509F4F16
:109F5000AF4FBF4F892F9A2FAB2FBB27A7FDBA95C5
:109F600090935A028093590257FF04C021503F4FEB
:109F70004F4F5F4FBB2757FDBA95A52F942F832FC7
:109F800090935C0280935B02809140029091410229
:109F900081349105DCF480913E0290913F0281343E
:109FA0009105A4F48091CC05E82FFF27EE0FFF1F49
:109FB000E450F94F808191810190F081E02DF7FF0D
:109FC00003C0F095E195FF4F7A97E4F08091470840
:109FD0008F3FC1F48091590290915A0297FD0196EA
:109FE0009595879590935A028093590280915B02D0
:109FF00090915C0297FD01969595879590935C02F0
:10A0000080935B028091840790918507A0918607D9
:10A01000B0918707B7FF04C081509F4FAF4FBF4F2C
:10A02000892F9A2FAB2FBB27A7FDBA958093840762
:10A0300090938507A0938607B09387078091750753
:10A0400090917607A0917707B0917807B7FF04C089
:10A0500081509F4FAF4FBF4F892F9A2FAB2FBB27F8
:10A06000A7FDBA958093750790937607A09377071D
:10A07000B09378078091CD029091CE02A091CF024B
:10A08000B091D0022F81388549855A85281B390B1C
:10A090004A0B5B0B209303033093040340930503A7
:10A0A000509306038091C5029091C602A091C70209
:10A0B000B091C802EB84FC840D851E85E81AF90A6C
:10A0C0000A0B1B0BE0920703F092080300930903AD
:10A0D00010930A0320930B0330930C0340930D035A
:10A0E00050930E03E0920F03F092100300931103BC
:10A0F000109312038091A9029091AA02A091AB0241
:10A10000B091AC02821B930BA40BB50B8093A902F8
:10A110009093AA02A093AB02B093AC028091A102EB
:10A120009091A202A091A302B091A4028E199F095E
:10A13000A00BB10B8093A1029093A202A093A30263
:10A14000B093A40288898823E1F02091870230919E
:10A150008802213831054CF08091DF029091E002B5
:10A1600001969093E0028093DF0220583F4F4CF419
:10A170008091DF029091E00201979093E00280933A
:10A18000DF02109288021092870281E090E09093A3
:10A19000260380932503E0900B03F0900C030091BD
:10A1A0000D0310910E03D801C70117FF07C08827C0
:10A1B0009927DC018E199F09A00BB10B81509240A9
:10A1C000A040B04034F084E090E090932603809368
:10A1D000250380912B0390912C03A0912D03B09126
:10A1E0002E0320918F073091900740919107509155
:10A1F0009207821B930BA40BB50B815E914BAF4F63
:10A20000BF4F8F539C49A040B04028F08091480830
:10A2100089310CF4FFC021E0E21620E1F20620E0D3
:10A22000020720E012070CF473C0809127038823F3
:10A2300009F46AC0D801C70117FF07C0882799270A
:10A24000DC018E199F09A00BB10B9C01AD01B7FF7A
:10A2500004C021503E4F4F4F5F4FF9E05595479551
:10A2600037952795FA95D1F780912503909126038C
:10A27000820F931F9093260380932503D801C70173
:10A2800017FF03C00796A11DB11DE3E0B595A79583
:10A2900097958795EA95D1F78093190390931A03C0
:10A2A000A0931B03B0931C0389589341A040B04076
:10A2B00064F088E893E1A0E0B0E080931903909304
:10A2C0001A03A0931B03B0931C0320911903309130
:10A2D0001A0340911B0350911C0357FF04C02150E7
:10A2E0003F4F4F4F5F4F232F342F452F552747FDAB
:10A2F0005A958091590290915A02820F931F909320
:10A300005A028093590206C081E08093270302C05D
:10A310001092270340E0E41640EFF4064FEF0407E5
:10A320004FEF14070CF073C080912803882309F4C1
:10A330006AC0D801C70117FF07C088279927DC0129
:10A340008E199F09A00BB10B9C01AD01B7FF04C092
:10A3500021503E4F4F4F5F4F69E0559547953795D8
:10A3600027956A95D1F78091250390912603820F56
:10A37000931F9093260380932503D801C70117FFED
:10A3800003C00796A11DB11D23E0B595A79597952C
:10A3900087952A95D1F78093190390931A03A09378
:10A3A0001B03B0931C0388579C4EAF4FBF4F64F400
:10A3B00088E79CEEAFEFBFEF8093190390931A03E9
:10A3C000A0931B03B0931C032091190330911A032F
:10A3D00040911B0350911C0357FF04C021503F4F75
:10A3E0004F4F5F4F232F342F452F552747FD5A9549
:10A3F0008091590290915A02820F931F90935A02B2
:10A400008093590211C081E0809328030DC01092FF
:10A4100028030AC0109226031092250384E690E0D8
:10A4200090938701809386016889262F3327809136
:10A430002503909126032817390724F43093260327
:10A440002093250310914808112379F0212F3327F9
:10A4500027FD309580912503909126032817390711
:10A4600024F4309326032093250340910B0350914D
:10A470000C0360910D0370910E0341385105610585
:10A48000710574F08091E3029091E402209125031C
:10A4900030912603820F931F9093E4028093E3028E
:10A4A00040585F4F6F4F7F4F74F48091E30290915B
:10A4B000E4022091250330912603821B930B909395
:10A4C000E4028093E30281E090E09093260380937E
:10A4D0002503C0900F03D0901003E0901103F0907B
:10A4E0001203D701C601F7FE07C088279927DC01B0
:10A4F0008C199D09AE09BF0981509240A040B0401F
:10A5000034F084E090E090932603809325038091BB
:10A510002F0390913003A0913103B0913203209129
:10A520009707309198074091990750919A07821B9D
:10A53000930BA40BB50B815E914BAF4FBF4F8F5365
:10A540009C49A040B04018F019310CF4FFC001E064
:10A55000C01600E1D00600E0E00600E0F0060CF4D2
:10A5600073C080912903882309F46AC0D701C6010A
:10A57000F7FE07C088279927DC018C199D09AE09D1
:10A58000BF099C01AD01B7FF04C021503E4F4F4FA2
:10A590005F4F09E055954795379527950A95D1F76F
:10A5A0008091250390912603820F931F9093260399
:10A5B00080932503D701C601F7FE03C00796A11DAE
:10A5C000B11D13E0B595A795979587951A95D1F785
:10A5D00080931D0390931E03A0931F03B093200349
:10A5E00089589341A040B04064F088E893E1A0E02E
:10A5F000B0E080931D0390931E03A0931F03B093BC
:10A60000200320911D0330911E0340911F035091A0
:10A61000200357FF04C021503F4F4F4F5F4F232F60
:10A62000342F452F552747FD5A9580915B02909115
:10A630005C02820F931F90935C0280935B0206C0C2
:10A6400081E08093290302C01092290320E0C21602
:10A6500020EFD2062FEFE2062FEFF2060CF073C0C8
:10A6600080912A03882309F46AC0D701C601F7FE46
:10A6700007C088279927DC018C199D09AE09BF09FD
:10A680009C01AD01B7FF04C021503E4F4F4F5F4FBB
:10A69000E9E05595479537952795EA95D1F780914B
:10A6A000250390912603820F931F90932603809396
:10A6B0002503D701C601F7FE03C00796A11DB11DF2
:10A6C00073E0B595A795979587957A95D1F780937F
:10A6D0001D0390931E03A0931F03B093200388577C
:10A6E0009C4EAF4FBF4F64F488E79CEEAFEFBFEFD7
:10A6F00080931D0390931E03A0931F03B093200328
:10A7000020911D0330911E0340911F03509120039F
:10A7100057FF04C021503F4F4F4F5F4F232F342F1F
:10A72000452F552747FD5A9580915B0290915C0219
:10A73000820F931F90935C0280935B0211C081E0B3
:10A7400080932A030DC010922A030AC01092260398
:10A750001092250384E690E0909387018093860110
:10A760004889242F332780912503909126032817A9
:10A77000390724F430932603209325038091480859
:10A78000882379F0282F332727FD309580912503E2
:10A79000909126032817390724F430932603209339
:10A7A000250340910F0350911003609111037091A4
:10A7B0001203413851056105710574F08091E10281
:10A7C0009091E2022091250330912603820F931F7E
:10A7D0009093E2028093E10240585F4F6F4F7F4FAA
:10A7E000CCF48091E1029091E20220912503309116
:10A7F0002603821B930B9093E2028093E1020AC02E
:10A8000010925C0210925B0210925A02109259024E
:10A810001092890280919D07882341F410925C0276
:10A8200010925B0210925A021092590280918F0787
:10A8300090919007A0919107B091920780932B037C
:10A8400090932C03A0932D03B0932E038091970730
:10A8500090919807A0919907B0919A0780932F0340
:10A8600090933003A0933103B09332031092BD0252
:10A870001092BE021092BF021092C0021092B90252
:10A880001092BA021092BB021092BC021092B50252
:10A890001092B6021092B7021092B80210928F076F
:10A8A00010929007109291071092920710929707BA
:10A8B000109298071092990710929A0710928407A5
:10A8C00010928507109286071092870710927507DD
:10A8D0001092760710927707109278071092EA018B
:10A8E0001092E901E0907F02F0908002C701F7FE2C
:10A8F00004C0882799278E199F0904973CF08091FE
:10A90000B70784FD03C082E380935D021091E105E7
:10A91000A12EBB24CC24DD24B701882777FD8095A8
:10A92000982F9701F7FE04C0222733272E193F09DD
:10A93000442737FD4095542F0E9443779B01AC017B
:10A94000C601B5010E94437797FF04C061507E4F56
:10A950008F4F9F4F59E095958795779567955A95B5
:10A96000D1F79B01812F99278E9DD0018F9DB00D2E
:10A970009E9DB00D1124CD01B7FD03969595879549
:10A9800095958795280F391F80913602909137024F
:10A990008150924010F020E030E080915F02909171
:10A9A0006002280F391F442737FD4095542F20930C
:10A9B000FF02309300034093010350930203809100
:10A9C0009D0290919E02A0919F02B091A002821BD5
:10A9D000930BA40BB50B80939D0290939E02A093C2
:10A9E0009F02B093A0028155934CA040B04064F008
:10A9F00080E593ECA0E0B0E080939D0290939E02EE
:10AA0000A0939F02B093A00280919D0290919E021C
:10AA1000A0919F02B091A002805B9C43AF4FBF4FBB
:10AA200064F480EB9CE3AFEFBFEF80939D029093C3
:10AA30009E02A0939F02B093A00200918A01109100
:10AA40008B0117FDFCC08091B70783FFF8C0809190
:10AA50008901815080938901882309F0F4C08DE039
:10AA6000809389018091CD029091CE02A091CF0276
:10AA7000B091D002B7FF04C081509E4FAF4FBF4F7F
:10AA800039E0B595A795979587953A95D1F77C01CB
:10AA900097FF04C0F094E194F108F3948091C5020B
:10AAA0009091C602A091C702B091C802B7FF04C03E
:10AAB00081509E4FAF4FBF4F29E0B595A795979511
:10AAC00087952A95D1F79C0197FF03C03095219572
:10AAD0003F4FE216F3060CF47901B701F7FE02C00E
:10AAE000695F7F4F2B0183E0559447948A95E1F786
:10AAF00022E030E0420E531E6090C7077090C807F6
:10AB00008090C9079090CA0720913C0130913D0187
:10AB100040913E0150913F01C401B3010E94B777BB
:10AB200059016A013093730720937207021B130BBC
:10AB3000C801845E9D4F68E671E00E9482779C01A7
:10AB4000245B30408091860190918701009731F01D
:10AB5000019790938701809386011BC049E1E41619
:10AB6000F104BCF48091870290918802820F931FB8
:10AB7000909388028093870280915D02882349F038
:10AB8000815080935D02882321F4B0928C02A092C0
:10AB90008B028091860190918701892BF9F4809135
:10ABA00088019927289FB001299F700D389F700D4B
:10ABB0001124CB01B2010E948277CB01AA2797FD15
:10ABC000A095BA2F680E791E8A1E9B1E6092C70739
:10ABD0007092C8078092C9079092CA0780915D025F
:10ABE000882369F580918B0290918C0220917207E5
:10ABF00030917307821B930B845E9D4F68E671E072
:10AC00000E9482779C01245B30408091720186957E
:10AC10009927289FD001299FB00D389FB00D11248E
:10AC20009D01B7FF02C0215F3F4F04E03595279596
:10AC30000A95E1F73093600220935F0204C01092FE
:10AC4000600210925F0280918902882381F0109245
:10AC5000910210929202109293021092940210921A
:10AC60009502109296021092970210929802F0901C
:10AC70005602FF20F1F480919D07282F33274427A7
:10AC800055278091CD029091CE02A091CF02B09134
:10AC9000D002BC01CD010E944377DC01CB01BC0195
:10ACA000CD0128EF3AE240E050E00E94B777390149
:10ACB00002C066247724E0905502EE20F1F48091E2
:10ACC0009D07282F3327442755278091C50290914F
:10ACD000C602A091C702B091C802BC01CD010E947A
:10ACE0004377DC01CB01BC01CD0128EF3AE240E023
:10ACF00050E00E94B777290102C044245524809176
:10AD00006F0790917007893C91051CF088EC90E0EA
:10AD100005C088539F4F34F488E39FEF90937007EA
:10AD200080936F0780917B0790917C07893C910508
:10AD30001CF088EC90E005C088539F4F34F488E302
:10AD40009FEF90937C0780937B0780917D07909184
:10AD50007E07AA2797FDA095BA2F2091C507A22E9E
:10AD6000BB24CC24DD24BC01CD01A60195010E94A9
:10AD700043779B01AC0180916F0790917007AA27E0
:10AD800097FDA095BA2F17E0880F991FAA1FBB1F28
:10AD90001A95D1F7280F391F4A1F5B1F57FF04C0B0
:10ADA000215C3F4F4F4F5F4FA6E055954795379534
:10ADB0002795AA95D1F78301020F131F10937E07E1
:10ADC00000937D0780916D0790916E07AA2797FDEC
:10ADD000A095BA2FBC01CD01A60195010E94437731
:10ADE0009B01AC0180917B0790917C07AA2797FD7E
:10ADF000A095BA2FF7E0880F991FAA1FBB1FFA95DD
:10AE0000D1F7280F391F4A1F5B1F57FF04C0215C71
:10AE10003F4F4F4F5F4FE6E0559547953795279544
:10AE2000EA95D1F74201820E931E90926E078092AE
:10AE30006D078091C0079091C107880F991FAA27BD
:10AE400097FDA095BA2F20917407332744275527E3
:10AE5000BC01CD010E9443775B016C0197FF08C0E4
:10AE60002FE330E040E050E0A20EB31EC41ED51E1A
:10AE700076E0D594C794B794A7947A95D1F780914A
:10AE80008C07282F3327442755278091B1029091B2
:10AE9000B202A091B302B091B402BC01CD010E94F4
:10AEA0004377DC01CB01BC01CD0120EF35E540E06B
:10AEB00050E00E94B777B501620F731F7093C1070E
:10AEC0006093C0070150104134F080E090E190930E
:10AED0007E0780937D0780917D0790917E0780504B
:10AEE000904F34F480E090EF90937E0780937D073D
:10AEF00051E0851650E1950634F080E090E19093A2
:10AF00006E0780936D0780916D0790916E0780505A
:10AF1000904F34F480E090EF90936E0780936D072C
:10AF20006150704134F080E090E19093C1078093CC
:10AF3000C0078091C0079091C1078050904F34F4B2
:10AF400080E090EF9093C1078093C007809100014B
:10AF5000482F552780911F019091200148175907CC
:10AF600094F420911F013091200109811A81049FDE
:10AF7000C001059F900D149F900D1124B9010E94EE
:10AF80006E777A83698329813A81220F331F220FDA
:10AF9000331F3A8329834091B70740FD02C00C94C8
:10AFA0002760EE2011F00C942760FF2011F00C9424
:10AFB0002760882499248091570290915802909399
:10AFC0004E0580934D052091E5023091E602211552
:10AFD000310509F03FC08091150190911601895902
:10AFE000934058F087B5853F20F48091ED01815062
:10AFF00011C081E080933E034EC080911501909175
:10B0000016018436910508F587B58B30D0F0809114
:10B01000ED018F5F8093ED019AE089029001112488
:10B0200080917405821B87BD8CE291E09093D901D9
:10B030008093D8018EE591E09093E6028093E5023B
:10B040002AC081E080933D0326C0F0923D03F09238
:10B050003E0321C09092EC018092EB0180916D0241
:10B0600090916E02A0916F02B091700254E0880F2F
:10B07000991FAA1FBB1F5A95D1F78093EE01909399
:10B08000EF01A093F001B093F101215030403093D3
:10B09000E6022093E5022091750141FF25C022338D
:10B0A000E8F480918C01815080938C018F3FE1F511
:10B0B00010928A0280916D0290916E02A0916F02AF
:10B0C000B09170028093690290936A02A0936B0220
:10B0D000B0936C0281E080938C0126C0273420F16C
:10B0E00088EC80938C011DC08091400190914101BA
:10B0F000820F911D2091DA053327829FA001839F43
:10B10000500D929F500D1124CA01AA2797FDA095BA
:10B11000BA2F8093690290936A02A0936B02B09356
:10B120006C0281E080938A028091CD029091CE02E0
:10B13000A091CF02B091D002E0903C01F0903D018F
:10B1400000913E0110913F01BC01CD01A801970182
:10B150000E94B77759016A018091C5029091C60299
:10B16000A091C702B091C802BC01CD01A80197010E
:10B170000E94B777B901C5010E94AE6E909389070E
:10B1800080938807CC9734F08CE390E09093890704
:10B190008093880780918807909189070E94726D3B
:10B1A000909389078093880780E280933B011092F7
:10B1B00068021092670280918A02882309F4ABC565
:10B1C00080913B0299279C012071307084FDA3C5BA
:10B1D00080913A02826080933A0270919B07872F98
:10B1E000992741E0C42ED12CC822D92280FD04C069
:10B1F0008091B70781FD10C0E980FA803093340355
:10B2000020933303309368022093670280913B02BE
:10B21000806C80933B02DFC280913B0281FFAEC213
:10B2200000917C0110917D01C8010F96A0907D02D4
:10B23000B0907E028A159B050CF06EC080913D0394
:10B24000882309F069C080913503909136034597B2
:10B2500084F08091E5019091E601A091E701B09121
:10B26000E8018093690290936A02A0936B02B09305
:10B270006C0280913B0287FF15C080913B028F7763
:10B2800080933B028091E5019091E601A091E70156
:10B29000B091E8018093690290936A02A0936B02D7
:10B2A000B0936C0280913B02806480933B02E090FB
:10B2B0007907EE20F1F08091690290916A02A091E5
:10B2C0006B02B0916C02BC01CD0124E630E040E09D
:10B2D00050E00E94B7778E2D9927AA27BB278217A7
:10B2E0009307A407B5072CF4D0926802C0926702B6
:10B2F00010C0C501801B910B0F9797FF03C090955D
:10B3000081959F4F90936802809367028BE28093B0
:10B310003B011092610234C1C8010F97A816B9060B
:10B32000C4F520913E032223A1F580913B0286FFC4
:10B3300015C080913B028F7B80933B028091E50199
:10B340009091E601A091E701B091E8018093690234
:10B3500090936A02A0936B02B0936C0280913B02BF
:10B36000806880933B02C501801B910B0F9697FF6D
:10B3700003C0909581959F4F909581959F4F909395
:10B380006802809367028DE280933B012093610203
:10B39000F7C08DE380933B0160916202662371F1F7
:10B3A00020916302309164024091650250916602DF
:10B3B0008091690290916A02A0916B02B0916C0237
:10B3C00082179307A407B507CCF480913B028064F1
:10B3D00080933B02862F992790936802809367029F
:10B3E0008AE0809361028EE580933B0180913B026D
:10B3F00087FFC6C080913B028F7733C0662309F474
:10B4000043C02091630230916402409165025091E3
:10B4100066028091690290916A02A0916B02B091DC
:10B420006C02281739074A075B0774F580913B02C5
:10B43000806880933B02862F9927909581959F4F36
:10B44000909368028093670286EF8093610286E79B
:10B4500080933B0180913B0286FF92C080913B022A
:10B460008F7B80933B028091E5019091E601A09152
:10B47000E701B091E8018093690290936A02A0937A
:10B480006B02B0936C027CC080913B02807C09F41B
:10B4900077C080916102882309F04CC08091E5015A
:10B4A0009091E601A091E701B091E801885C90409D
:10B4B000A040B0402091690230916A0240916B0235
:10B4C00050916C0282179307A407B5076CF0809126
:10B4D000E5019091E601A091E701B091E801885C57
:10B4E0009040A040B0401DC08091E5019091E601E0
:10B4F000A091E701B091E80188539F4FAF4FBF4F34
:10B50000281739074A075B07BCF08091E501909145
:10B51000E601A091E701B091E80188539F4FAF4F3A
:10B52000BF4F8093690290936A02A0936B02B0931D
:10B530006C0202C01092610280913B028F73809373
:10B540003B02109234031092330371FF06C084EF64
:10B5500091E09093D9018093D80180917102882362
:10B5600079F480916D0290916E02A0916F02B0917A
:10B570007002C397A105B1051CF081E080937102B0
:10B580006091330370913403809167029091680257
:10B59000680F791F7093340360933303CB0177FFF7
:10B5A00004C088279927861B970B855F91400CF470
:10B5B000CEC040916102442389F180916302909151
:10B5C00064022091690230916A02821B930B0996F2
:10B5D000439748F48091630290916402A0916502C0
:10B5E000B091660212C0242F332727FD3095432FD8
:10B5F000532F8091690290916A02A0916B02B091E1
:10B600006C02820F931FA41FB51F80936902909351
:10B610006A02A0936B02B0936C0224C08091DA0599
:10B620002091690230916A0240916B0250916C0244
:10B630001616170644F463E00E946277280F311D46
:10B64000411D511D07C063E00E946277281B31092C
:10B65000410951092093690230936A0240936B02B9
:10B6600050936C021092340310923303E0906D02F9
:10B67000F0906E0200916F0210917002D801C70124
:10B6800080509440A040B0402091690230916A02FD
:10B6900040916B0250916C0282179307A407B50783
:10B6A0005CF4D801C70180509C4FAF4FBF4F2817A3
:10B6B00039074A075B0744F08093690290936A0256
:10B6C000A0936B02B0936C0280919B0781FF06C030
:10B6D00084E690E09093D9018093D8018091DE05B3
:10B6E0008823A9F580916202882389F54091570249
:10B6F0005091580257FF02C04D5F5F4F55954795D7
:10B700005595479580911F0190912001209100014E
:10B710003327489FB001499F700D589F700D112429
:10B72000CB01B9010E94827770937D0160937C0107
:10B73000663471051CF486E490E005C06739710534
:10B7400034F086E990E090937D0180937C018091B4
:10B75000E5029091E602892BD1F18091E50190916B
:10B76000E601A091E701B091E8018093690290930E
:10B770006A02A0936B02B0936C0229C080916D02A3
:10B7800090916E02A0916F02B09170028059914029
:10B79000A040B0408093690290936A02A0936B022C
:10B7A000B0936C028091DE05882311F0992702C0C6
:10B7B00088E790E090937D0180937C0189819A8154
:10B7C00090935802809357028EE280933B01E09061
:10B7D0005702F09058028091E5019091E601A09106
:10B7E000E701B091E8012091690230916A0240912D
:10B7F0006B0250916C02281739074A075B0724F047
:10B8000080919B0780FDD3C280913302882309F089
:10B81000CEC28091E5029091E602892B49F0E0903A
:10B820005702F09058021092360310923503E1C08F
:10B830008091E5019091E601A091E701B091E801C6
:10B84000821B930BA40BB50B80930303909304030B
:10B85000A0930503B09306038230E0E89E07EFEF64
:10B86000AE07EFEFBE072CF481E090E8AFEFBFEF3B
:10B8700009C08F5F9F47A040B04064F08FEF9FE703
:10B88000A0E0B0E08093030390930403A09305032A
:10B89000B0930603809103039091040390933603C1
:10B8A0008093350380917401282F3327442755272F
:10B8B0008091030390910403A0910503B0910603C6
:10B8C000BC01CD010E94437797FF04C0615E7F4FAA
:10B8D0008F4F9F4F25E095958795779567952A958A
:10B8E000D1F760930303709304038093050390934F
:10B8F000060365300EEF70070FEF80070FEF90071C
:10B900002CF484E09EEFAFEFBFEF09C060507440AD
:10B910008040904064F080E094E0A0E0B0E080934C
:10B92000030390930403A0930503B0930603809050
:10B930000303909004032091EB013091EC0137FF59
:10B9400002C0295F3F4F03E0359527950A95E1F73F
:10B950004FEF223834071CF421E83FEF05C02038B0
:10B96000310514F020E830E0C901AA2797FDA09521
:10B97000BA2F20917601332744275527BC01CD01EA
:10B980000E94437797FF04C06D5F7F4F8F4F9F4F9B
:10B9900012E095958795779567951A95D1F79B0154
:10B9A0005FEF613075071CF420E03FEF06C06F3F8A
:10B9B000710519F014F020E031E080913B02807CA9
:10B9C00049F0C90137FD03969C01359527953595BA
:10B9D00027950DC080919B0780FF09C0C90137FDE5
:10B9E00007969C01A3E035952795AA95E1F7820E6D
:10B9F000931E20917301222309F454C060918D029B
:10BA000070918E0280918F029091900297FF04C0F6
:10BA100061587F4F8F4F9F4FF7E0959587957795AA
:10BA20006795FA95D1F73327442755270E94437726
:10BA300097FF04C0615E7F4F8F4F9F4FE5E0959564
:10BA4000879577956795EA95D1F76093030370938F
:10BA5000040380930503909306036138AFEF7A07E0
:10BA6000AFEF8A07AFEF9A072CF480E89FEFAFEFB4
:10BA7000BFEF0AC06F3F71058105910569F064F061
:10BA800080E091E0A0E0B0E0809303039093040392
:10BA9000A0930503B09306038091030390910403E0
:10BAA000880E991E80917101282F332780914B08B1
:10BAB000992787FD9095289FF001299FF00D389FC9
:10BAC000F00D11249F01F7FF02C021583F4F220FB4
:10BAD000232F221F330BFFEF21383F071CF420E8F0
:10BAE0003FEF06C02F3F310519F014F020E031E0A0
:10BAF000820E931EC401AA2797FDA095BA2F00912C
:10BB00005702109158029801442737FD4095542F51
:10BB1000BC01CD010E94437797FF04C061507E4F66
:10BB20008F4F9F4F59E095958795779567955A95D3
:10BB3000D1F7E61AF70A8091670290916802892B83
:10BB400009F064C0101611060CF060C02091350396
:10BB500030913603C90137FF03C0309521953F4F1F
:10BB60002D33310540F480918502909186028E1527
:10BB70009F0574F526C02C53304045E03695279537
:10BB80004A95E1F72031310510F02FE030E0409187
:10BB900085025091860218161906E4F480E190E0BF
:10BBA000821B930B489F9001499F300D589F300D89
:10BBB0001124B4E036952795BA95E1F72E153F0587
:10BBC00020F580917A0190917B01E816F906F4F056
:10BBD0007C011CC0205F3F4F80917A0190917B01D6
:10BBE000829FB001839F700D929F700D11249B0165
:10BBF000A4E036952795AA95E1F74E155F0514F058
:10BC00007A0104C0E216F30608F07901C701AA27F9
:10BC100097FDA095BA2FFDE0880F991FAA1FBB1FA3
:10BC2000FA95D1F72091880730918907442737FD8D
:10BC30004095542FBC01CD010E94B7772093070394
:10BC4000309308034093090350930A03E0900703DD
:10BC5000F090080380913703909138039C01220FE4
:10BC6000331F280F391F2E0D3F1D37FF02C02D5FD8
:10BC70003F4FA901559547955595479550933803E2
:10BC8000409337038091D605282F3327220F331F87
:10BC9000220F331F241735076CF48091BF07282F1C
:10BCA0003327220F331F220F331F205530404217F6
:10BCB000530724F0309338032093370380919B0778
:10BCC00080FF14C08091370390913803A981BA8115
:10BCD0008A179B0724F0B0933803A0933703E091B1
:10BCE0003703F0913803FA83E98361C029813A81EF
:10BCF000201B310B37FF02C02D5F3F4F3595279535
:10BD000035952795E0903703F0903803E20EF31E47
:10BD1000FA82E9824CC08091DE05882301F56091AA
:10BD200057027091580277FF02C06D5F7F4F759583
:10BD300067957595679540911F01509120018091FD
:10BD40000001282F3327649FC001659F900D749FC9
:10BD5000900D1124B9010E948277CB0101C099276F
:10BD600090937D0180937C0180917C0190917D0175
:10BD7000873491051CF486E490E005C0863991056E
:10BD800034F086E990E090937D0180937C010981F5
:10BD90001A81109338030093370380913B02806C23
:10BDA00080933B0280913A028D7F80933A0280918A
:10BDB0003B0299279C012270307081FF39C180912C
:10BDC000390390913A03A0913B03B0913C03009753
:10BDD000A105B10521F0809171028130B9F4809103
:10BDE000570290915802AA2797FDA095BA2F1EE0FE
:10BDF000880F991FAA1FBB1F1A95D1F7809339038B
:10BE000090933A03A0933B03B0933C03809171025B
:10BE1000813019F482E08093710229813A8179019D
:10BE20000027F7FC0095102F8091880790918907D3
:10BE30009C01442737FD4095542FC801B7010E944B
:10BE40004377DC01CB018093070390930803A09311
:10BE50000903B0930A03B7FF04C08150904EAF4F5F
:10BE6000BF4F7C018D01ADE015950795F794E794E0
:10BE7000AA95D1F7E0920703F09208030093090313
:10BE800010930A0360913C0270913D023FE0603ADA
:10BE9000730750F58091390390913A03A0913B03C9
:10BEA000B0913C039C01AD01FAE05695479537955A
:10BEB0002795FA95D1F7821B930BA40BB50BA8011C
:10BEC0009701E4E0220F331F441F551FEA95D1F775
:10BED000820F931FA41FB51F8093390390933A03D9
:10BEE000A0933B03B0933C0360547F4118F58091CD
:10BEF000390390913A03A0913B03B0913C039C011C
:10BF0000AD016CE056954795379527956A95D1F721
:10BF1000821B930BA40BB50BA8019701F2E0220F33
:10BF2000331F441F551FFA95D1F7820F931FA41F8B
:10BF3000B51F41C08091EB019091EC018091EB0124
:10BF40009091EC0197FF03C0909581959F4F8436A7
:10BF50009105CCF58091E5019091E601A091E70172
:10BF6000B091E8019C018091690290916A02281BBE
:10BF7000390B37FF03C0309521953F4F2F3F3105D7
:10BF800009F00CF58091390390913A03A0913B039D
:10BF9000B0913C039C01AD01EEE056954795379575
:10BFA0002795EA95D1F7821B930BA40BB50B8E0D49
:10BFB0009F1DA01FB11F8093390390933A03A09354
:10BFC0003B03B0933C038091390390913A03A091D5
:10BFD0003B03B0913C037EE0B695A7959795879576
:10BFE0007A95D1F790935802809357024091DC05DF
:10BFF000442399F055279C01BA010E948277C90118
:10C00000861B970B9093860280938502260F371F1D
:10C0100030937B0120937A011FC010928602109208
:10C0200085028FEF93E090937B0180937A0114C097
:10C03000109271021092390310923A0310923B034E
:10C0400010923C03309358022093570205C0809110
:10C050003B02806C80933B0280914D0381FF37C08F
:10C0600089819A8197FD03969595879595958795F2
:10C0700020913802309139022817390760F48091F5
:10C08000570290915802892B31F0220F331F220F53
:10C09000331F3A8329838091E5019091E601A091B5
:10C0A000E701B091E8018093690290936A02A0933E
:10C0B0006B02B0936C0288E99AE39093D901809364
:10C0C000D80180E09EE090930A01809309012091BD
:10C0D0008207822F9927880F991F880F991F8896AA
:10C0E00069817A818617970714F09A838983709102
:10C0F000BF077D8B872F9927880F991F880F991F5E
:10C1000080559040A981BA818A179B0714F49A83BD
:10C11000898380912302882341F480915D088F3FB9
:10C1200021F4809151038823E9F080913C029091A1
:10C130003D020297C097B0F4E981FA811E161F06EE
:10C140008CF481E090E090933D0280933C02E22EDB
:10C15000FF24EE0CFF1CEE0CFF1C8701085D1F4F37
:10C160001A83098329813A8130933205209331055E
:10C170008091FF0290910003A0910103B09102030E
:10C1800012E0880F991FAA1FBB1F1A95D1F70091C3
:10C19000C0071091C107081B190B213A31058CF01B
:10C1A000C90137FD019695958795801791070CF485
:10C1B0008C01909581959F4F081719076CF48C019D
:10C1C0000BC00135110514F000E510E03FEF003B16
:10C1D000130714F400EB1FEF4D89242F3327220F90
:10C1E000331F220F331FC90169817A81861B970B88
:10C1F000801791070CF48C0189819A81821B930B23
:10C20000081719070CF48C0180917D0790917E0727
:10C210006091830270918402861B970B90938E0726
:10C2200080938D07D0909D072091950230919602C2
:10C230004091970250919802DD2041F0661A770AEA
:10C24000C301AA2797FDA095BA2F04C0AA2797FD7E
:10C25000A095BA2F280F391F4A1F5B1F2093950204
:10C2600030939602409397025093980280919502E2
:10C2700090919602A0919702B091980281509A4FA6
:10C28000A040B04064F080E09AEFA0E0B0E080937E
:10C29000950290939602A0939702B0939802809192
:10C2A000950290919602A0919702B09198028050C9
:10C2B0009640AF4FBF4F64F480E096E0AFEFBFEF22
:10C2C0008093950290939602A0939702B093980260
:10C2D000C090EB0520918D0730918E0778E0E72E16
:10C2E000EC1498F08C2D9927829FA001839F500D0C
:10C2F000929F500D1124CA0157FD07967C0163E0FF
:10C30000F594E7946A95E1F712C08C2D86959927EC
:10C31000829FB001839F700D929F700D1124CB01FD
:10C3200077FD03967C01F594E794F594E794A0904B
:10C330007701B09078019501442737FD4095542F3F
:10C340008091950290919602A0919702B0919802E7
:10C35000BC01CD010E94B777E20EF31E90906101FF
:10C36000692D772788279927980117FF04C022276E
:10C370003327201B310B37FF02C02F5F3F4F35950E
:10C380002795A981BA812A0F3B1F442737FD409585
:10C39000542F0E94437797FF04C0615C7F4F8F4FFB
:10C3A0009F4F26E095958795779567952A95D1F7C4
:10C3B0009B016E157F050CF47B01309521953F4F55
:10C3C000E216F3060CF4790180916D0790916E07E7
:10C3D0006091810270918202861B970B90936C078B
:10C3E00080936B07209191023091920240919302C9
:10C3F00050919402DD2041F0461A570AC201AA2743
:10C4000097FDA095BA2F04C0AA2797FDA095BA2F33
:10C41000280F391F4A1F5B1F20939102309392020D
:10C4200040939302509394028091910290919202D2
:10C43000A0919302B091940281509A4FA040B040D5
:10C4400064F080E09AEFA0E0B0E0809391029093D6
:10C450009202A0939302B0939402809191029091E2
:10C460009202A0919302B091940280509640AF4FF7
:10C47000BF4F64F480E096E0AFEFBFEF809391028E
:10C4800090939202A0939302B093940220916B0731
:10C4900030916C0748E04C1598F08C2D9927829FBD
:10C4A000B001839F700D929F700D1124CB0177FD19
:10C4B00007966C0193E0D594C7949A95E1F712C062
:10C4C000C6948C2D9927829FD001839FB00D929F97
:10C4D000B00D1124CD01B7FD03966C01D594C7941E
:10C4E000D594C7949501442737FD4095542F8091EA
:10C4F000910290919202A0919302B0919402BC019A
:10C50000CD010E94B777C20ED31E692D77278827E9
:10C510009927980117FF04C022273327201B310BCE
:10C5200037FF02C02F5F3F4F35952795E981FA818C
:10C530002E0F3F1F442737FD4095542F0E9443770D
:10C5400097FF04C0615C7F4F8F4F9F4FA6E095958A
:10C55000879577956795AA95D1F79B016C157D0511
:10C560000CF46B01309521953F4FC216D3060CF4A5
:10C57000690180918207282E332450902D06FBE913
:10C580008F2EF6E09F2EE2E5AE2EE6E0BE2E7BE09B
:10C59000472E6EE9662E67E0762ED5012C91121695
:10C5A0000CF029C1203429F4E981FA81FF8BEE8B4C
:10C5B0001FC049815A81CA01AA2797FDA095BA2FA9
:10C5C000332727FD3095432F532FBC01CD010E9407
:10C5D000437797FF04C0615C7F4F8F4F9F4F56E0BA
:10C5E00095958795779567955A95D1F77F8B6E8B43
:10C5F000F5012181203439F42E893F892E0D3F1D0C
:10C600003F8B2E8B2AC0203C39F44E895F894E190E
:10C610005F095F8B4E8B21C0C701AA2797FDA095AC
:10C62000BA2F332727FD3095432F532FBC01CD015F
:10C630000E94437797FF04C0615C7F4F8F4F9F4FED
:10C6400046E095958795779567954A95D1F7AE8998
:10C65000BF89A60FB71FBF8BAE8BF5012281203497
:10C6600039F42E893F892C0D3D1D3F8B2E8B2AC01E
:10C67000203C39F44E895F894C195D095F8B4E8BE4
:10C6800021C0C601AA2797FDA095BA2F332727FD01
:10C690003095432F532FBC01CD010E94437797FF64
:10C6A00004C0615C7F4F8F4F9F4F36E09595879513
:10C6B000779567953A95D1F7AE89BF89A60FB71FD1
:10C6C000BF8BAE8BF5012381203439F42E893F894D
:10C6D000200F311F3F8B2E8B2AC0203C39F44E890E
:10C6E0005F89401B510B5F8B4E8B21C0C801AA276D
:10C6F00097FDA095BA2F332727FD3095432F532F51
:10C70000BC01CD010E94437797FF04C0615C7F4F5D
:10C710008F4F9F4F26E095958795779567952A953A
:10C72000D1F7AE89BF89A60FB71FBF8BAE8BF301C0
:10C73000808191812E893F898217930764F4B90122
:10C74000680F791F77FF02C06F5F7F4F7595679500
:10C750007F8B6E8B1DC0552049F44E895F89440F35
:10C76000551F481B590B5F8B4E8B12C051E055155E
:10C7700078F4252D33276E897F89861B970BB901A5
:10C780000E948277AE89BF89A60FB71FBF8BAE8B81
:10C79000C101880F991F880F991FEE89FF898E1795
:10C7A0009F0764F4FD898F2F9927880F991F880FA1
:10C7B000991F2E893F892817390714F09F8B8E8B7C
:10C7C0008E899F8997FD0396959587959595879571
:10C7D000F4018183880F991F880F991F2E893F8943
:10C7E000281B390BC901880F8283EE89FF89D30189
:10C7F000ED93FC9303C0F401118212824A9422E06B
:10C8000030E0620E731E44E050E0A40EB51E68E0F6
:10C8100070E0860E971E47FEC0CEE2E1C95E0C9422
:10C82000EE7784B1806A84B93D9A82E58CBD1DBCE7
:10C83000459A81E08093D1078AEA8093E20783E8F2
:10C840008093E3078AE08093E4071092E607109252
:10C85000E5071092E8071092E70710924A08109235
:10C86000060808953091D107332309F085C00DB42F
:10C8700007FE82C084E08093D701459A2EB580914F
:10C88000540399278130910589F0823091051CF479
:10C89000892B21F03EC00297B9F03BC030930508C8
:10C8A000209355032138A9F581E008C0253549F4C6
:10C8B00080915503820F8093550382E08093540347
:10C8C00028C03093540325C080910508E82FFF2726
:10C8D000E95DF74F20838F5F8093050890915503A2
:10C8E0008032A0F0291769F480E2A7E2B8E0E7E01F
:10C8F000F8E00D9001928A95E1F781E080930608B7
:10C9000002C0309306081092540303C0920F909314
:10C9100055032091E107223208F028C04598000015
:10C920000000000000000000000000000000000007
:10C9300000000000000000000000000000000000F7
:10C940000000000000000000000000000000E09176
:10C95000DA07F091DB07E20FF11D80818EBD809137
:10C9600003089081890F8093030803C081E08093BE
:10C97000D1072F5F2093E1070895EF92FF920F9365
:10C980001F938091E4059927880F991F880F991F9D
:10C990007C010027F7FC0095102F8091CD0290912B
:10C9A000CE02A091CF02B091D002BC01CD01A8016E
:10C9B00097010E94B7773093E6072093E5078091AF
:10C9C000C5029091C602A091C702B091C802BC01F5
:10C9D000CD01A80197010E94B7773093E807209313
:10C9E000E7072091C7073091C8074091C9075091C8
:10C9F000CA07DA01C90163E0880F991FAA1FBB1F8C
:10CA00006A95D1F7820F931FA41FB51F820F931F42
:10CA1000A41FB51F20913C0130913D0140913E0182
:10CA200050913F01BC01CD010E94B7773093EE07D2
:10CA30002093ED078091DF029091E0022091F801B0
:10CA40003091F901821B930B9093F4078093F307C5
:10CA5000E091D502F091D6028091940790919507CC
:10CA6000BF010E9482779B01220F331F220F331FC9
:10CA7000260F371F260F371F37FF02C02D5F3F4F8E
:10CA800035952795359527953093EA072093E90743
:10CA90008091C3079091C407BF010E9482779B01D8
:10CAA000220F331F220F331F260F371F260F371F6A
:10CAB00037FF02C02D5F3F4F359527953595279558
:10CAC0003093EC072093EB071092D6021092D50218
:10CAD00010929507109294071092C4071092C30702
:10CAE0008091E4079927AA27BB27FC013A97E830F1
:10CAF000F10508F0E8C1E858FF4F0C9409788091DF
:10CB000050028093F70780914F028093F80780913D
:10CB10004E028093F90780914D028093FA0780912D
:10CB20004C028093FB0780914B028093FC0780911D
:10CB30004A028093FD07809149028093FE0780910D
:10CB40003B028093FF0780913B02837F80933B02EF
:10CB50000E94912C8093000880912E0680930108FA
:10CB600080913A02AEC180915708909158089093F5
:10CB7000F8078093F70780915B0890915C08909389
:10CB8000FA078093F90780911F019091200180930B
:10CB9000FB07809100018093FC0780913B0180930B
:10CBA000FD07909156039093FE07E92FFF27A3E01E
:10CBB000EE0FFF1FAA95E1F7E556F94F86818093A6
:10CBC000FF07838180930008878180930108858116
:10CBD00080930208892F8F5F6CE00E9462779093A8
:10CBE000560371C1809119068093F70780911A0648
:10CBF0008093F80780911B068093F90780911C06AB
:10CC00008093FA0780911D068093FB07809121068F
:10CC10008093FC07809122068093FD078091230674
:10CC20008093FE07809126068093FF07809124065B
:10CC30008093000880912506809301088091270643
:10CC400040C1809118068093F7071092F8073BC106
:10CC5000F8948091CB05E82FFF27EE0FFF1FE450DB
:10CC6000F94F0190F081E02DE038F1051CF0EFE77D
:10CC7000F0E006C02FEFE138F20714F4E1E8FFEF2F
:10CC8000E093F7078091CC05E82FFF27EE0FFF1FF9
:10CC9000E450F94F0190F081E02DE038F1051CF0EF
:10CCA000EFE7F0E006C07FEFE138F70714F4E1E8C2
:10CCB000FFEFE093F8078091CA05E82FFF27EE0FFA
:10CCC000FF1FE450F94F0190F081E02DE038F105AD
:10CCD0001CF0EFE7F0E006C08FEFE138F80714F43E
:10CCE000E1E8FFEFE093F9078091C905E82FFF27FE
:10CCF000EE0FFF1FE450F94F0190F081E02DE03876
:10CD0000F1051CF0EFE7F0E006C02FEFE138F20785
:10CD100014F4E1E8FFEF7894E093FA07809174024D
:10CD20008093FB07809175028093FC0780917602C7
:10CD30008093FD07809177028093FE0780917802AF
:10CD40008093FF07809179028093000880917A0296
:10CD50008093010880917B02B4C08091B203863039
:10CD600018F01092B20385E08093F70780912806AF
:10CD70008093F80780916D0290916E02A0916F02EE
:10CD8000B0917002BC01CD0125E030E040E050E000
:10CD90000E94B7773093FA072093F90780916902D0
:10CDA00090916A02A0916B02B0916C02BC01CD011E
:10CDB00025E030E040E050E00E94B7773093FC0778
:10CDC0002093FB0780911E068093FD0780911F062C
:10CDD0008093FE07809120068093FF078091730265
:10CDE000809300088091FC069091FD0680930108D5
:10CDF000809131059091320597FD03969595879521
:10CE0000959587955EC01092F7078AE58093F8079D
:10CE100086E08093F90785E38093FA07809101010A
:10CE20008093FB07809197038093FC079091980370
:10CE30009093FD078F778093970390719093980359
:10CE4000809199038093FE078091B7078093FF0735
:10CE500080919B078093000880912A0680930108A7
:10CE6000809137062EC08091FD058093F707809151
:10CE700035068093F807809169018093F9078091C6
:10CE8000F6058093FA078091F7058093FB07809160
:10CE9000F8058093FC07809168018093FD078091DD
:10CEA000FA058093FE078091FB058093FF07809130
:10CEB000FC058093000880915D08809301088091B3
:10CEC0005B058093020880910608882309F451C10C
:10CED0006091070880919B01681719F08AEF809391
:10CEE000990160939B0181E080938901409108083A
:10CEF00050910908CA0181509E4F8F5F9340B0F452
:10CF000020910A0830910B08C90181509E4F8F5F14
:10CF1000934060F48091D50585FF08C0509343038A
:10CF200040934203309341032093400380910E08C5
:10CF300090910F0821E08936920724F490938B0199
:10CF400080938A0120911808309119088091D801A6
:10CF50009091D9018217930740F48091AC01882306
:10CF600021F43093D9012093D801862F9927883650
:10CF7000910509F468C08936910524F48736910536
:10CF800051F0FFC08936910509F496C08B369105A2
:10CF900009F4E2C0F6C080911A0880934708809196
:10CFA0001B088093490880911C0880934808809151
:10CFB0001D088093880180911E0880934B08809102
:10CFC0001F0880939A0180912008809353038091D9
:10CFD000210880933F03809148028823F9F0209133
:10CFE00022083091230837FD19C030938C0220931A
:10CFF0008B029091FF05992389F08FE0989FC001E3
:10D000001124281B390BC90188599E4F68E671E02D
:10D010000E94827790938C0280938B0220914A0326
:10D0200030914B038091240890912508280F391FD7
:10D0300037FF02C02F5F3F4F3595279530934B0345
:10D0400020934A039EC080911A088093DC07809148
:10D050001B088093DD0780911C088093DE07809178
:10D060001D088093DF0780911E088093E007809160
:10D07000210590911F08892B80932105909122050D
:10D080009370809120088C70982B9093220580914A
:10D090002108809351038091220880938D01809113
:10D0A000230880934A088091240880934D0380913F
:10D0B000250880934C0365C080911A088093D2079D
:10D0C00080911B088093D30780911C088093D4071C
:10D0D00080911D088093D50780911E0890911F08AC
:10D0E0009093D7078093D6078091200890912108CC
:10D0F0009093D9078093D80780912208992787FDBC
:10D10000909590932F0780932E078091230880930A
:10D11000620280912408909125089C01442737FDE4
:10D120004095542FDA01C90163E0880F991FAA1FA7
:10D13000BB1F6A95D1F7820F931FA41FB51F820FE3
:10D14000931FA41FB51F8093630290936402A09362
:10D150006502B093660215C080911A08809350034F
:10D1600080911B0880934F0380911C0880934E038D
:10D1700008C0109243031092420310924103109290
:10D1800040031F910F91FF90EF9008958091D10778
:10D19000882309F43BC0459882EE97E09093DB0723
:10D1A0008093DA0790915203E92FFF27E257FE4F51
:10D1B0009F5F9093520380818093E4079B3010F02F
:10D1C000109252031092D1070E94BD6481E08093B7
:10D1D000E107000000000000000000000000000067
:10D1E000000000000000000000000000000000003F
:10D1F000000000000000000000000000000000002F
:10D2000000008091E207809303088EBD089587B1E6
:10D210008C6087B9429843981092580380E88093B5
:10D220009D011092570380939C01089580915D03A6
:10D23000815080935D038F3F09F055C189E0809351
:10D240005D0380912E0790912F0781589F4F39F0F1
:10D2500080912E0790912F078158809362038091CF
:10D260003B02992780739070892B21F48091980359
:10D2700080FF1DC080911606882351F080916003C5
:10D28000882319F484E08093580381E0809360033D
:10D29000809117068823B9F080916103882319F4DF
:10D2A00084E08093570381E0809361030CC0109267
:10D2B0006003109261038091120680935E03809157
:10D2C000140680935F0380916003882309F073C084
:10D2D00080913406282F332724FF07C080917202E3
:10D2E000882319F425FD80C081C090911306983FD2
:10D2F00048F0809196078D3D28F080915E03882349
:10D300006CF00AC0983F68F080919607853049F428
:10D3100080915E0387FF02C0429801C0429A81E07B
:10D3200032C0809158038150809358038F3F09F099
:10D330005EC08091370685FF29C090916203892FD6
:10D34000869580935803992351F480915E0387FF5B
:10D3500002C0429801C0429A10929D0148C080913B
:10D360009D0190915E03882341F48093620380E8DD
:10D3700080939D019923D4F137C0982311F0429AEC
:10D3800001C04298869580939D0131C08091960797
:10D3900086958093580380919D01813021F41092ED
:10D3A000620380E801C0869580939D0180919D0174
:10D3B00090915E0317C08091580381508093580369
:10D3C0008F3FA9F489E08093580380919D018130BB
:10D3D00011F480E801C0869580939D0180919D01A4
:10D3E00090911606892311F0429A01C042988091CB
:10D3F0006103882309F043C09091340697FF07C06A
:10D4000080917202882319F496FD52C053C0909106
:10D410001506983F48F08091BE078D3D28F0809119
:10D420005F0388236CF00AC0983F78F08091BE07B4
:10D43000853059F480915F0387FF02C0439801C093
:10D44000439A81E080939C0136C0809157038150BC
:10D45000809357038F3F79F58091BE07869580931F
:10D46000570380919C01813011F480E801C08695BA
:10D4700080939C0180919C0190915F0317C08091E3
:10D4800057038150809357038F3FA9F489E080931D
:10D49000570380919C01813011F480E801C086958A
:10D4A00080939C0180919C0190911706892311F033
:10D4B000439A01C04398429B04C080913A0288601D
:10D4C00003C080913A02877F80933A02439B06C053
:10D4D00080913A02806180933A02089580913A02E5
:10D4E0008F7E80933A0208950F931F93CF93DF931B
:10D4F000482FEB0180917302E42FFF27843BD8F083
:10D500008F010E0F1F1FF801E450F94F80819181A8
:10D510009B01281B390BC90163E070E00E948277F0
:10D52000CB01880F991F860F971F005D184FF801D8
:10D530009183808306C0EE0FFF1FE05DF84F1182DC
:10D540001082E42FFF27EE0FFF1FE450F94FD18325
:10D55000C083DF91CF911F910F9108954FB724E1C0
:10D5600030E0F8948091C9008F778093C900809152
:10D57000C9008F7B8093C9008091C9008F7D809303
:10D58000C900832F99278093CD002093CC008091F0
:10D59000C80082608093C80080E18093C9008091B8
:10D5A000CA008F778093CA008091CA008F7B8093D6
:10D5B000CA008091CA008F7D8093CA008091CA0002
:10D5C0008F7E8093CA008091CA00877F8093CA00B3
:10D5D0008091C9008B7F8093C9008091CA008460CC
:10D5E0008093CA008091CA0082608093CA008091B3
:10D5F000C80087FF03C08091CE00F9CF8091C90099
:10D6000080688093C9004FBF0895EF92FF920F93F7
:10D610001F93CF93DF93482F00E010E080919E018D
:10D62000813061F410929E0184E48093650310922E
:10D630006703109266031092680303C2809165032A
:10D64000882319F421E030E001C09801909166032D
:10D65000992371F4232B11F081E010C084E48093AE
:10D660006503909367039093660390936803D2C118
:10D67000913069F4232B09F0C3C182E080936603E3
:10D68000809167038F5F8093670383E0C1C192300D
:10D69000D1F4232B09F0B4C183E080936503409358
:10D6A000680390916703923039F41092690347FF41
:10D6B00003C081E08093690383E0809366039F5FEA
:10D6C00090936703A7C1933009F09AC1232B09F007
:10D6D00097C19093650382E080936603809167030E
:10D6E0008F5F8093670320916803822F9927782F9B
:10D6F0006627842F9927682B792B8091EF0581303D
:10D7000051F47370CB018050924063E070E00E944E
:10D710008277EB0119C0823069F47770CB018050B9
:10D72000944066E070E00E948277EB012695269592
:10D7300026950CC0EB01D370C856D140CE01D7FD61
:10D740000196EC01D595C79526952695022F1127B0
:10D750000F7010700F5F1F4F0D30110508F049C199
:10D760000230110519F404E010E005C00430110581
:10D7700011F402E010E0D801A00FB11FFD01E45048
:10D78000F94F808191819E01281B390BC90137FF18
:10D7900003C0909581959F4F069704F5E09131065F
:10D7A000EE2351F0FF27EE0FFF1FE450F94F808169
:10D7B00091818436910594F480917302883C30F411
:10D7C00080917302865F8093730208C088EC809317
:10D7D000730280916F008F7D80936F00A450B94FCA
:10D7E0008D919C91BC01660F771F680F791F6C0F9C
:10D7F0007D1F77FF02C06D5F7F4F7B01F594E7943B
:10D80000F594E794CE0101968E159F0524F40894B3
:10D81000E108F10808C0CE010197E816F9061CF4EA
:10D820000894E11CF11C0630110509F0CEC0C53684
:10D83000D1050CF4A5C090916403E92FFF27E45BA8
:10D84000F74FE081ED3729F4809163038095809351
:10D850006303963061F480916303882311F0E33809
:10D86000B9F0882309F088C0ED3791F085C0993070
:10D8700009F082C080916303882329F480915508C0
:10D88000833831F079C0809155088D3709F074C024
:10D8900080914D088D3739F480914E08833899F482
:10D8A00063E87FEF0DC0833871F480914E088338B0
:10D8B00019F460E070E004C08D3729F46DE770E082
:10D8C00085E00E94746A80914F08992787FD9095A2
:10D8D000BC0186E00E94746A80915008992787FDF8
:10D8E0009095BC018BE00E94746A80915108992741
:10D8F00087FD9095BC018CE00E94746A809164035E
:10D900008930D1F5809153088D3749F480910C0707
:10D9100090910D070596BC0188E00E94746A809181
:10D9200054088D3749F480910C0790910D070597A5
:10D93000BC0188E00E94746A80910C0790910D07E9
:10D9400083589F4F1CF483E89FEF09C080910C0718
:10D9500090910D078E37910534F08DE790E090930C
:10D960000D0780930C0780915208992787FD9095A9
:10D97000BC018AE00E94746A1092640310926303EF
:10D98000CA30D1055CF4809164038F5F8093640397
:10D99000E82FFF27E45BF74F83E8808380916403DF
:10D9A0008A3011F4109264038FEFCC39D8076CF4ED
:10D9B00080916403E82FFF27E45BF74F8DE78083B6
:10D9C000809163038095809363030530110518F4FB
:10D9D000B701802F0BC00530110519F4BE0187E097
:10D9E00005C007301105B1F4BE0189E00E94746AD8
:10D9F00011C00231110570F081E080939E010AC0D0
:10DA000081E080939E01109267031092690384E481
:10DA10008093650380916703803198F0809169035A
:10DA2000882331F480919E01882311F480933A0178
:10DA300010926703109269031092660384E4809346
:10DA40006503E6E0CDB7DEB70C94FA77CF93FC011F
:10DA500097FF05C0CFEFF095E195FF4F01C0C1E002
:10DA600028E631E0CF01B9010E948277FC018B35B5
:10DA7000910554F08B5590408A35910538F484EB2C
:10DA800090E08E1B9F0BFC0141E00DC0CF01855B38
:10DA900090408A35910518F4E45BF04003C02E1BDA
:10DAA0003F0BF9014FEFEE0FFF1FE953F74F2591A1
:10DAB00034918C2F992787FD9095289FB001299F3D
:10DAC000700D389F700D1124842F992787FD909534
:10DAD000689FA001699F500D789F500D1124CA01C5
:10DAE000CF9108952AE530E0281B390BC9010E9427
:10DAF000266D08950895089508950895089580E085
:10DB000090E00895109258081092570810925C08FF
:10DB100010925B0810925A081092590810925D08F2
:10DB20008AE090E00E94CF1590936B0380936A0384
:10DB30000895CF93DF9380916A0390916B030E94C5
:10DB4000D815882309F4AFC080916A0390916B03C4
:10DB50000A9690936B0380936A03E0E0F0E09F01E4
:10DB600090E05FEFABE9B6E04BE0ED018B8187FF22
:10DB70000BC09F5F8D81E80FF11D8981280F311D3A
:10DB80008E81851708F4582F4150189647FFEDCF26
:10DB900050935D08232B41F5209170033091710360
:10DBA0004091720350917303BB27A52F942F832FAD
:10DBB00090936F0380936E03AA27BB27281B390B12
:10DBC0004A0B5B0BCF01AA27BB27280F391F4A1F1F
:10DBD0005B1F209370033093710340937203509343
:10DBE0007303E5E0F0E013C020916E0330916F0302
:10DBF0002E173F0718F4E21BF30B02C0E0E0F0E041
:10DC0000892F9927880F991FE80FF91F3596F093F0
:10DC10005808E0935708EF3FF10578F480911F0111
:10DC2000909120018E9F90018F9F300D9E9F300D0F
:10DC30001124C90164E670E013C0CF019695879561
:10DC40009695879520911F0130912001289FA00172
:10DC5000299F500D389F500D1124CA0169E170E0D1
:10DC60000E946E7770935A086093590820916C0354
:10DC700030916D032E0F3F1F30936D0320936C0383
:10DC80005EE02131350778F080915B0890915C0867
:10DC9000019690935C0880935B0820513E4030933E
:10DCA0006D0320936C03DF91CF910895089508953B
:10DCB000002422273327442751E0BB27EE27FF27E4
:10DCC000A0E1660F771F881F991F001C221F331FBA
:10DCD000441F660F771F881F991F001C221F331FC8
:10DCE000441F2AF4050E2B1F3E1F4F1F04C0051AA8
:10DCF0002B0B3E0B4F0B550FBB1FEE1F587F556074
:10DD000047FD5250AA95E9F6E695B7955795E695E1
:10DD1000B7955795852F9B2F08952227332741E0EC
:10DD2000552768E0880F991F221F331F880F991FFE
:10DD3000221F331F1AF4240F351F02C0241B350B7A
:10DD4000440F551F487F456037FD42506A9551F793
:10DD50005695479556954795842F0895AA2797FF7E
:10DD600004C0809590958A1F9A1F77FF04C0609524
:10DD700070956A1F7A1F669F9001779FA001679F29
:10DD8000300D411D5A1F300D411D5A1F889FF00153
:10DD9000999F2E0F3F1F401D511D899F300D411D22
:10DDA0005A1F300D411D5A1FCA01B901112480CFDD
:10DDB00090917703933240F4E92FFF27E25AF74F0F
:10DDC00080839F5F909377030895833218F48D5F6B
:10DDD00080937703089590E2E1E6F8E08FE1919374
:10DDE000815087FFFCCF0895CF93CFB723E031E078
:10DDF000F8948091C9008F778093C9008091C90001
:10DE00008F7B8093C9008091C9008F7D8093C9006A
:10DE1000832F99278093CD002093CC008091C80058
:10DE200082608093C80088E18093C9008091CA0015
:10DE30008F778093CA008091CA008F7B8093CA003D
:10DE40008091CA0080628093CA008091CA0080617C
:10DE50008093CA008091CA0088608093CA00809134
:10DE6000C90084608093C9008091CA008460809357
:10DE7000CA008091CA0082608093CA008091C80065
:10DE800087FF03C08091CE00F9CF8091C9008068E0
:10DE90008093C9008091C90080648093C9000E946A
:10DEA000EB6ECFBFCF910895282F99278F70907078
:10DEB000892B31F4209580917603822B8093760311
:10DEC00008958091A101882309F44BC080913B0201
:10DED00085FD04C08091A401882381F082E98093AC
:10DEE0005E0883E280935F088091A401882309F48F
:10DEF00085E5809360081092A40102C080935E08BB
:10DF00008091A2018F3071F4809176030E947F6D21
:10DF1000882341F081E980935E0880935F0881E364
:10DF2000809360081092A1018091C80085FFFCCF0A
:10DF30008091C9008F7E8093C9008091C9008E7F37
:10DF40008093C90080915E08882311F48EEF01C090
:10DF50008EE78093CE00809176038093A201109289
:10DF6000760308951F920F920FB60F9211248F938C
:10DF70009F93EF93FF939091A101992309F040C0E3
:10DF800080917803882361F480915E08882311F4DE
:10DF900083E003C0813999F481E0809378030FC056
:10DFA000833099F480915E08882349F090935E084D
:10DFB0008091C9008E7F8093C9008EEF1EC0809132
:10DFC000C90081608093C9000EC0833261F48091E2
:10DFD000C9008E7F8093C9008FEF8093CE0081E0CF
:10DFE0008093A10118C080917803E82FFF27E25A9F
:10DFF000F74F8F5F8093780380818093CE000BC0B2
:10E00000109278031092790310927A038091C900DC
:10E0100080618093C900FF91EF919F918F910F9044
:10E020000FBE0F901F901895EF92FF920F931F93C2
:10E03000CF93DF937C018B01EA01452B39F0F80186
:10E0400081918F01F70109952197C9F7E6E0CDB7D6
:10E05000DEB70C94FA77EF92FF920F931F93CF9352
:10E06000DF937C018B01EA01452B41F0F8010F5F42
:10E070001F4F8491F70109952197C1F7E6E0CDB7CD
:10E08000DEB70C94FA770F931F93CF938C01C62FB2
:10E09000161634F480E2F8010995C1501C16D4F329
:10E0A000CF911F910F9108950F931F93CF938C01E0
:10E0B000C62F161634F480E3F8010995C1501C16DA
:10E0C000D4F3CF911F910F910895A5E3B0E0EBE653
:10E0D000F0E70C94D2772E96EEADFFAD2E97882404
:10E0E0009924540180917503882321F42C961FAE46
:10E0F0001EAE2C97AEE44A2E512C4C0E5D1E6F01C5
:10E10000B60105C0153239F00894C11CD11CF601C6
:10E1100014911123B9F7A601461B570B31F02C9629
:10E120008EAD9FAD2C970E942B70112309F46AC20B
:10E130000894C11CD11CFF24FDA6FCA67FEFE72E8E
:10E14000F9A6F6010894C11CD11C1491153721F0D1
:10E15000812F80628837B1F4F0FE0AC0F20124E01A
:10E1600030E0420E531E80809180A280B3800AC0AE
:10E17000F20142E050E0440E551E808191814C0135
:10E18000AA24BB24103221F489A58823D1F61DC00E
:10E19000133219F458E0F52AD4CF1A3211F01D3297
:10E1A00091F41A3259F4F20182E090E0480E591EBF
:10E1B000E081ECA7EE232CF6E195ECA790E1F92A9B
:10E1C000AFEDFA22BECF1B3211F419A7BACF1E321F
:10E1D000C1F5F6010894C11CD11C14911A3279F4CE
:10E1E000F20122E030E0420E531E408151813FEFA8
:10E1F0004F3F530714F44FEF5FEFE42EA2CF40E000
:10E2000050E0812F80538A30A0F4CA0163E0880F68
:10E21000991F6A95E1F7840F951F480F591F410F09
:10E22000511D40535040F6010894C11CD11C14915B
:10E23000E8CF8FEF4F3F580714F44FEF5FEFE42E16
:10E2400085CF103329F4F4FC7CCF90E2F92A79CF02
:10E25000812F81538930D8F440E050E0CA0133E087
:10E26000880F991F3A95E1F7840F951F480F591FA2
:10E27000410F511D40535040F6010894C11CD11C60
:10E280001491812F80538A3048F34CA75FCF183602
:10E2900019F4A4E0FA2A55CF1C3619F4B1E0FB2A90
:10E2A00050CF133661F43E010894611C711CF201D9
:10E2B00022E030E0420E531E808189833CC1143439
:10E2C00021F0143611F0193651F5143411F431E0FF
:10E2D000F32AF0FE0AC0F20144E050E0440E551E5D
:10E2E00080809180A280B3800CC0F20182E090E037
:10E2F000480E591E808191814C01AA2497FCA0945C
:10E30000BA2CB7FE0AC0B094A09490948094811C5B
:10E31000911CA11CB11C8DE289A70AE06FC01F34BB
:10E3200011F01F3631F41F3411F491E0F92A08E09E
:10E3300064C0103779F4F201A2E0B0E04A0E5B1E2F
:10E34000808191814C01AA24BB2400E1B0E4FB2A26
:10E3500018E753C01337C1F5F20122E030E0420E56
:10E36000531E608071806114710489F43E01089429
:10E37000611C711C88E289838EE6F301818385E745
:10E380008B838CE68C838D8389E28E831F82E7FCEE
:10E3900013C08E2D992787FD9095AC0160E070E049
:10E3A000C3010E949F75009729F0382E3618E31498
:10E3B0000CF0C3C03E2CC1C0F30101900020E9F76E
:10E3C00031973E2E3618B9C0153511F0153731F496
:10E3D000153511F4F1E0FF2A0AE00FC0183519F0E5
:10E3E000183709F0A0C000E1F3FE07C081149104C2
:10E3F000A104B10411F020E4F22A19A6EDA6E7FC6D
:10E4000002C03FEDF32229E2622E712C6C0E7D1EBC
:10E4100081149104A104B10421F44DA5442309F40D
:10E420007BC0802F9927AA27BB278EA79FA7A8ABC1
:10E43000B9AB202E332490E0891690E0990691E044
:10E44000A90690E0B90648F0C501B4012EA53FA584
:10E4500048A959A90E94957717C0AFEF8A16910471
:10E46000A104B10449F040F0C401B1010E946E77EB
:10E470009B014427552708C0882D602F0E94627792
:10E48000282F3327442755272AAB3BAB4CAB5DAB3A
:10E490000A3059F48AA9880F880F880F9AA9990F12
:10E4A000890F382D381B832F10C0003139F48AA909
:10E4B0008295807F482D481B842F07C08AA9880F2A
:10E4C000880F880F582D581B852F90E02EA53FA54B
:10E4D00048A959A982169306A406B50608F091E04A
:10E4E0008AA89BA8ACA8BDA88A3010F4805D04C09F
:10E4F000895A183509F48F7DD3018E933D019923F4
:10E5000009F099CF083041F4F3FE06C0803321F0C2
:10E5100080E3FD0182933F01CE010196382E36182B
:10E52000F8E23F0E0BC0112309F46CC03E010894C1
:10E53000611C711C198391E0392E19A6032D2DA49D
:10E54000231827FC222489A5882311F00F5F02C01D
:10E55000F6FC0E5F020DEF2CFF24C7018073907054
:10E56000892B49F48CA5801B682F2C968EAD9FAD0E
:10E570002C970E94437089A5882331F041E050E038
:10E58000BE01675D7F4F0AC0E6FE0EC080E38AA72A
:10E590001BA742E050E0BE01665D7F4F2C968EAD1A
:10E5A0009FAD2C970E941470C70180739070809764
:10E5B00049F48CA5801B682F2C968EAD9FAD2C97AF
:10E5C0000E945470622D2C968EAD9FAD2C970E94A8
:10E5D0005470832D992787FD9095AC01B3012C963B
:10E5E0008EAD9FAD2C970E941470E4FE89CD2CA5B2
:10E5F000201B2CA7622F2C968EAD9FAD2C970E94CE
:10E6000043707ECDE2E1CB5C0C94EE772FB740E017
:10E61000F894E0E0F0E081E2809357009491E2E02A
:10E62000F0E0809357003491E4E0F0E080935700ED
:10E6300084912FBF9E3199F4363941F4893011F419
:10E6400041E00DC08A3059F442E009C0373939F44D
:10E65000863011F443E003C0853009F444E0842F90
:10E66000992708959FB7F8948091C900877F809378
:10E67000C9008091C9008F7E8093C9008091C90034
:10E680008F778093C9008091C9008F7B8093C900E8
:10E690008091C9008F7D8093C9009FBF08951F930B
:10E6A000CF93DF93182F80917503882309F4A0C0BE
:10E6B0008091A001181709F49BC0809174038823EE
:10E6C00021F40E9406738093740382ED91E090938D
:10E6D0003901809338018CE19AE09F938F93C0ECCD
:10E6E000D1E1DF93CF93E0917E03F0917F03099511
:10E6F0000F900F900F900F90812F992784309105E4
:10E70000F1F0853091051CF4892B51F00CC0863056
:10E710009105D9F086309105ACF0089741F12AC0F7
:10E7200088E19AE002C08FE09AE09F938F93DF9395
:10E73000CF93E0917E03F0917F03099527C08AE093
:10E740009AE0F3CF82E09AE0F0CF8AEF99E09F93CE
:10E750008F93DF93CF93E0917E03F0917F03099530
:10E7600088ED91E090933901809338010FC085EFD7
:10E7700099E0DBCF89E29AE09F938F93DF93CF9369
:10E78000E0917E03F0917F03099510E00F900F90C8
:10E790000F900F9080917403843011F0823099F4BF
:10E7A0000E943273812F8150833018F40E94AE6A28
:10E7B0001DC0143019F40E94F46E18C01830B1F462
:10E7C0000E94566E13C0112389F08FE39AE09F9345
:10E7D0008F9380EC91E19F938F93E0917E03F09172
:10E7E0007F0309950F900F900F900F901093A00149
:10E7F000DF91CF911F9108951F93CF93DF93182F2F
:10E8000081E08093750340919F01E5EAF9E020E003
:10E8100030E05FE4849199272F5F3F4F829FB001E2
:10E82000839F700D929F700D112446275150319691
:10E8300057FFF0CF40939F01EDE7F9E020E030E093
:10E8400057E2849199272F5F3F4F829FB001839FAA
:10E85000700D929F700D112446275150319657FF2D
:10E86000F0CF40939F0180917403882321F40E948C
:10E8700006738093740380919F01833459F088E17B
:10E8800090E029E20FB6F894A895809360000FBE3F
:10E890002093600085E690E790937F0380937E034A
:10E8A0000E949E0587E690E09F938F938AE590E013
:10E8B0009F938F931F921F92809101016AE00E94A3
:10E8C0006277892F99279F938F93809101010E94EE
:10E8D000627799279F938F938AE59AE09F938F930E
:10E8E000C0ECD1E1DF93CF93E0917E03F0917F0301
:10E8F000099585EA99E09F938F93DF93CF93E091F9
:10E900007E03F0917F0309958DE799E09F938F93A4
:10E91000DF93CF93E0917E03F0917F0309950E94EE
:10E920009E0583EC8093810080916F0080628093CC
:10E930006F008DB79EB746968DBF123081F08EE87E
:10E940009AE09F938F93DF93CF93E0917E03F091B2
:10E950007F0309950F900F900F900F90F0CFDF91EC
:10E96000CF911F91089580912F068D3338F08091BB
:10E97000D20787FD03C08CE380932F068091DE05CC
:10E98000882331F08055853618F08FE78093DE05B7
:10E990000895CF9380917503882309F472C0809104
:10E9A0007B03815080937B03882309F053C089E166
:10E9B00080937B0380912F068E3338F08091D207AD
:10E9C00087FD03C08DE380932F0680917302823808
:10E9D00020F580913C0290913D02805D974020F0AF
:10E9E00080915D08843620F410927D0310927C03A0
:10E9F00080917C0390917D03009739F1019790936A
:10EA00007D0380937C03419728F18091D20784FF96
:10EA100021C080913A0284601BC080917302853BC3
:10EA2000C8F090912F0684E1989FC0011124409670
:10EA300020917C0330917D032817390730F42F5F34
:10EA40003F4F30937D0320937C0380913A028B7F6C
:10EA500080933A02C091A301CC2321F0C150C0930E
:10EA6000A3010FC08BE48093A3018091A0018430A7
:10EA700011F40E94616F80919F01833411F0C09363
:10EA80007503CF9108951F920F920FB60F92112424
:10EA90002F933F934F935F936F937F938F939F93A6
:10EAA000AF93BF93EF93FF932091CE008091AE017F
:10EAB0008823B1F02093C6008091AE01823029F501
:10EAC0002F3F19F58FEF94E3ACE0B0E0C297A109B6
:10EAD000B109B7FFFBCF8091C1038093CE0015C071
:10EAE0009091A001892F8150833020F4822F0E94C1
:10EAF000056B0BC0943021F4822F0E94546F05C027
:10EB0000983019F4822F0E94576EFF91EF91BF91B8
:10EB1000AF919F918F917F916F915F914F913F91B5
:10EB20002F910F900FBE0F901F901895FB01DC01E5
:10EB300002C005900D9241505040D8F70895FC0155
:10EB40004150504030F001900616D1F73197CF0177
:10EB50000895882799270895A0E0B0E0E2EBF5E753
:10EB60000C94DA776C017B01EA01590121978FEF50
:10EB7000CF3FD80789F086010894C11CD11CC7017A
:10EB80000894E11CF11CF5010995F8018083219797
:10EB9000FFEFCF3FDF0779F7EAE0CDB7DEB70C94A0
:10EBA000F677CF92DF92EF92FF920F931F937C0143
:10EBB0006B01FB010995082FC7010196F601099524
:10EBC000182FC8011F910F91FF90EF90DF90CF9009
:10EBD0000895A0E0B0E0EFEEF5E70C94DC778C014F
:10EBE0007B01EA01690121978FEFCF3FD80771F0D0
:10EBF000F70121917F01C8010F5F1F4F622FF601BE
:10EC000009952197FFEFCF3FDF0791F7E8E0CDB7F8
:10EC1000DEB70C94F877CF92DF92EF92FF920F93CA
:10EC20001F936C018B017A01FA010995812F9927B5
:10EC3000682FC6010196F70109951F910F91FF906A
:10EC4000EF90DF90CF9008955058BB27AA270ED0A1
:10EC5000E0C0D1D030F0D6D020F031F49F3F11F495
:10EC60001EF4C6C00EF4E095E7FBBCC0E92FE2D06D
:10EC700080F3BA17620773078407950718F071F4D9
:10EC80009EF5FAC00EF4E0950B2EBA2FA02D0B01C5
:10EC9000B90190010C01CA01A0011124FF27591BE1
:10ECA00099F0593F50F4503E68F11A16F040A22FE7
:10ECB000232F342F4427585FF3CF46953795279558
:10ECC000A795F0405395C9F77EF41F16BA0B620B57
:10ECD000730B840BBAF09150A1F0FF0FBB1F661F9E
:10ECE000771F881FC2F70EC0BA0F621F731F841FE1
:10ECF00048F4879577956795B795F7959E3F08F007
:10ED0000B3CF9395880F08F09927EE0F97958795C5
:10ED1000089598D088F09F5790F0B92F9927B75150
:10ED2000A0F0D1F0660F771F881F991F1AF0BA95CF
:10ED3000C9F712C0B13081F09FD0B1E008959CC0F6
:10ED4000672F782F8827B85F39F0B93FCCF38695C5
:10ED500077956795B395D9F73EF490958095709522
:10ED600061957F4F8F4F9F4F0895E89409C097FB9F
:10ED70003EF490958095709561957F4F8F4F9F4F92
:10ED80009923A9F0F92F96E9BB279395F6958795D6
:10ED900077956795B795F111F8CFFAF4BB0F11F499
:10EDA00060FF1BC06F5F7F4F8F4F9F4F16C0882340
:10EDB00011F096E911C0772321F09EE8872F762F76
:10EDC00005C0662371F096E8862F70E060E02AF0B7
:10EDD0009A95660F771F881FDAF7880F96958795A3
:10EDE00097F9089597F99F6780E870E060E00895CB
:10EDF0009FEF80EC089500240A9416161706180653
:10EE00000906089500240A9412161306140605062E
:10EE10000895092E0394000C11F4882352F0BB0FBF
:10EE200040F4BF2B11F460FF04C06F5F7F4F8F4F22
:10EE30009F4F089557FD9058440F551F59F05F3F5D
:10EE400071F04795880F97FB991F61F09F3F79F00C
:10EE500087950895121613061406551FF2CF46958E
:10EE6000F1DF08C0161617061806991FF1CF869510
:10EE70007105610508940895E894BB2766277727F4
:10EE8000CB0197F90895629FD001739FF001829F93
:10EE9000E00DF11D649FE00DF11D929FF00D839F29
:10EEA000F00D749FF00D659FF00D9927729FB00DC6
:10EEB000E11DF91F639FB00DE11DF91FBD01CF01D9
:10EEC00011240895991B79E004C0991F961708F042
:10EED000961B881F7A95C9F780950895AA1BBB1BBE
:10EEE00051E107C0AA1FBB1FA617B70710F0A61B4A
:10EEF000B70B881F991F5A95A9F780959095BC016B
:10EF0000CD01089597FB092E07260AD077FD04D07E
:10EF1000E5DF06D000201AF4709561957F4F0895C3
:10EF2000F6F7909581959F4F0895A1E21A2EAA1B9E
:10EF3000BB1BFD010DC0AA1FBB1FEE1FFF1FA217A9
:10EF4000B307E407F50720F0A21BB30BE40BF50BA6
:10EF5000661F771F881F991F1A9469F7609570952F
:10EF6000809590959B01AC01BD01CF01089597FB61
:10EF7000092E05260ED057FD04D0D7DF0AD0001C7D
:10EF800038F450954095309521953F4F4F4F5F4F46
:10EF90000895F6F790958095709561957F4F8F4F06
:10EFA0009F4F08952F923F924F925F926F927F9260
:10EFB0008F929F92AF92BF92CF92DF92EF92FF9289
:10EFC0000F931F93CF93DF93CDB7DEB7CA1BDB0B35
:10EFD0000FB6F894DEBF0FBECDBF09942A883988DA
:10EFE00048885F846E847D848C849B84AA84B984E1
:10EFF000C884DF80EE80FD800C811B81AA81B981ED
:10F00000CE0FD11D0FB6F894DEBF0FBECDBFED0100
:10F010000895EE0FFF1F0590F491E02D0994FFCFA6
:10F020005E0A010164FF010020FFFFC01FC01F0135
:10F030000101737373FF03007D0000C409C40964F8
:10F0400000104E6F726D616C0051756164726F00DB
:10F050000000000000006400D20101200B05000048
:10F06000ECFF00020406070808080706040200FE79
:10F07000FCFAF9F8F8F8F9FAFCFE000204060708B1
:10F08000086440415A46553264640A029696969640
:10F090000840403A10FB30380132FF03780090D02E
:10F0A000030090D0030032002064FFFF64200B0AAD
:10F0B0000D0B0C0E0B0F100B11FA206801010170E3
:04F0C000FF010F64D9
:00000001FF
